:020000040800F2
:1000000000CB01207102000845510008254000087E
:1000100095500008410C00086960000800000000CD
:10002000000000000000000000000000B101000816
:10003000950D0008000000000D020008455700085B
:100040008B0200088B0200088B0200088B0200085C
:100050008B0200088B0200088B0200088B0200084C
:100060008B0200088B0200088B0200088B0200083C
:100070008B0200088B0200088B020008450C000868
:100080008B0200088B0200088B02000800000000B1
:100090000000000000000000000000008B020008CB
:1000A0008B0200088B0200086D5800088B020008C4
:1000B0008B0200088B0200088B0200088B020008EC
:1000C0008B0200088B0200088B0200088B020008DC
:1000D0008B0200088B0200088B0200080000000061
:1000E0008B0200088B0200088B0200080000000051
:1000F0000000000000000000000000008B0200086B
:10010000000000008B0200088B0200088B02000830
:1001100000000000000000000000000000000000DF
:10012000510C0008D90C00088B0200088B02000853
:100130008B0200080000000000000000000000002A
:100140000000000000000000000000008B0200081A
:100150008B020008E50C00088B02000829600008EB
:100160008B0200088B020008000000000000000065
:10017000000000000000000000000000000000007F
:10018000000000008B0200080000000000000000DA
:100190008B0200088B020008DFF810D000F01CFC76
:1001A00000480047E13D0208AFF3008000CB01208A
:1001B0002C4B19680868B0E8F04F80F30988BFF34A
:1001C0006F8F4FF0000080F311887047000000002F
:1001D00008480068006880F308884FF0000080F34A
:1001E000148862B661B6BFF34F8FBFF36F8F00DF25
:1001F00000BF00BF08ED00E0DFF80C00016841F42B
:1002000070010160704700BF88ED00E0EFF30980E6
:10021000BFF36F8F134B1A681EF0100F08BF20ED4D
:10022000108A20E9F04F106009B44FF0500080F3BD
:100230001188BFF34F8FBFF36F8F2DF0ABFA4FF0E4
:10024000000080F3118809BC19680868B0E8F04F15
:100250001EF0100F08BFB0EC108A80F30988BFF3BE
:100260006F8F704798020020EFF305807047000001
:100270000648804706480047FEE7FEE7FEE7FEE740
:10028000FEE7FEE7FEE7FEE7FEE7FEE75D58000853
:10029000990100082DE9F05F0546002092469B4633
:1002A00088460646814640241BE02846414647468C
:1002B000224600F08CFA53465A46C01A914110D398
:1002C00011461846224600F073FA2D1A67EB010812
:1002D0004F4622460120002100F06AFA17EB000980
:1002E0004E41201EA4F10104DFDC484631462A4677
:1002F0004346BDE8F09F2DE9F0410024061B25464A
:1003000071F1000605DA01240027D0EB070067EB46
:100310000101161E73F1000605DA0027D2EB070271
:10032000012567EB0303FFF7B5FF86460E46174628
:100330009C46AC4204D00025D0EB050E65EB0106CF
:1003400024B10020D2EB000760EB030C704631466D
:100350003A466346BDE8F08140EA01039B0703D0BB
:1003600009E008C9121F08C0042AFAD203E011F8F4
:10037000013B00F8013B521EF9D27047D2B201E0B6
:1003800000F8012B491EFBD270470022F6E710B59A
:1003900013460A4604461946FFF7F0FF204610BDF3
:1003A000421C10F8011B0029FBD1801A704710B5C0
:1003B000002200E0521C835C8C5CA34201D1002B24
:1003C000F8D1D8B2E1B2401A10BD2DE9FE4F8046F7
:1003D00081EA0300C00F0C46009021F0004123F099
:1003E0000045B8EB0200A94105D24046214690469F
:1003F0001C460B46024623F00040104347D0270D11
:10040000C7F30A00C3F30A510290401A0190402832
:100410006BDAC3F3130040F4801B0098924620B1BE
:100420000023D2EB030A63EB0B0B01985946C0F192
:100430004002504600F0BCF906460D46504659466B
:10044000019A00F0D4F910EB08006141002487EA1A
:10045000115284EAE7731A4340D0009A62B3019ABA
:10046000012A4FEA075215DC001B61EB02014FF035
:10047000004202EA0752CDE90042001C41F580111A
:1004800032462B4600F029FA03B0BDE8F08F404613
:100490002146F9E7001B61EB0201001C41F58013C6
:1004A00000185B412018A2F5001747EB030140EA52
:1004B000D570B6196D4111E06D084FEA360645EA70
:1004C000C0754FEA0752001B61EB0201001C41F5A9
:1004D000801149084FEA30000019514132462B463D
:1004E00003B0BDE8F04F00F0E9B9009801224000E8
:1004F0000023D0EB020263EBE073009821464FEA41
:10050000E074B8EB000061EB0401E9E783F000431D
:100510005BE781F0004158E72DE9FE4F81EA0304D3
:1005200004F0004421F0004100944FF0000B23F050
:10053000004350EA01045ED052EA03045BD0C3F3E7
:100540000A54C1F30A552C44A4F2F3340194A0FBDD
:100550000254C1F3130141F48011C3F3130343F4B4
:10056000801301FB024400FB034E840A970A44EA0D
:10057000815447EA8357A4FB076802958D0A05FB5F
:1005800007854FEA932C04FB0C542705029D4FEA84
:10059000065847EA1637B5EB08056EEB070C870ED1
:1005A000920E47EA811742EA8312A7FB0201B6EBDB
:1005B0000B0164EB00042B0D43EA0C335E1844EB93
:1005C0001C50DA465146E7FB0201C5F313044FEA1B
:1005D0000B3343EA14534FEA0432019C43EA060307
:1005E000A4F10C040294009CCDE900B400F075F96C
:1005F00003B0BDE8F08F00200146F9E72DE9F04D8A
:1006000081EA030404F0004B21F0004514464FF04A
:10061000000A23F0004150EA050220D054EA01020A
:100620001DD0C5F30A570246C5F31303C1F31300E7
:10063000C1F30A5640F4801543F48013A7EB060873
:10064000101BD64608F2FD3873EB050002D308F103
:10065000010801E092185B41B8F1000F03DA0020B5
:100660000146BDE8F08D00204FF480110646844617
:100670000EE0171B73EB050705D3121B63EB050395
:1006800006434CEA010C49084FEA300092185B41DE
:1006900050EA0107EDD152EA030012D082EA0400C9
:1006A00083EA0501084305D0101BAB4106D20122A5
:1006B000002306E000224FF0004302E06FF0010249
:1006C00053101AEB06004CEB085110EB0A0041EBFB
:1006D0000B01BDE8F04D00F0F1B80EB540F233412A
:1006E00002910021CDE900110A460B4600F0F5F811
:1006F00003B000BDC1F30A5210B5C1F3130140F2BB
:10070000FF3341F480119A4201DA002010BD40F21B
:1007100033439A42A2F2334203DC524200F057F8CC
:1007200010BD904010BD00F0004230F000400AD0F3
:10073000C10D01F56071C0F3160042EA0151C20813
:1007400040071143704700200146704701F0004305
:1007500030B421F0004150EA010206D00A0DA2F5A2
:100760006072C1F31301002A02DC30BC0020704724
:10077000440F44EAC104C100E01830BC00EBC25091
:1007800000F047B830B50B46014600202022012476
:1007900009E021FA02F59D4205D303FA02F5491B4F
:1007A00004FA02F52844151EA2F10102F1DC30BD65
:1007B000202A04DB203A00FA02F100207047914021
:1007C000C2F1200320FA03F3194390407047202A16
:1007D00004DB203A21FA02F00021704721FA02F3EB
:1007E000D040C2F120029140084319467047202AA8
:1007F00006DBCB17203A41FA02F043EAE07306E049
:1008000041FA02F3D040C2F1200291400843194658
:1008100070470029A8BF7047401C490008BF20F05E
:100820000100704710B4B0FA80FC00FA0CF050EAF6
:10083000010404BF10BC704749B1CCF1200421FA77
:1008400004F411FA0CF118BF012121430843A3EB72
:100850000C01CB1D4FEA00614FEA102042BF00207F
:1008600010BC704700EBC35010440029A4BF10BC5B
:100870007047401C490008BF20F0010010BC7047C1
:1008800010B541000CD0C0F3C751962908DC7E2971
:1008900009DC06DB410204D000F0004040F07E504D
:1008A00010BD002010BDC1F19604C4F1200100FA72
:1008B00001F1E040FFF7ADFFA04010BD10B5141EE0
:1008C00073F1000408DA401C41F1000192185B4109
:1008D0001A4301D120F0010010BD2DE9F04D9246E0
:1008E0009B4611B1B1FA81F202E0B0FA80F22032F7
:1008F0009046FFF75DFF04460F4640EA0A0041EAD2
:100900000B0153465A46084313D0114653EA0100DF
:1009100019D0C8F140025046FFF759FF05460E4670
:10092000504659464246FFF743FF084305D0012091
:1009300004E020463946BDE8F08D0020054346EA34
:10094000E0762C4337430A986305E40AA0EB0800DD
:100950000022FD0A44EA47540A3002D5002001462D
:10096000E9E7010510196941DDE908450019694108
:10097000BDE8F04DA2E7C1F30A52C1F3130140F202
:10098000FF3341F480119A4202DA00200146704799
:1009900040F233439A42A2F2334202DC5242FFF762
:1009A00016BFFFF705BF000030B5041E71F100044B
:1009B00004DB4FF00044404264EB0101141E73F16C
:1009C000000405DB1C464FF00043524263EB040376
:1009D000994208BF904230BD064C074D06E0E068E2
:1009E00040F0010394E8070098471034AC42F6D376
:1009F000FFF7D6FBB0F20508D0F2050870B58C18E9
:100A000010F8015B15F0070301D110F8013B2A1122
:100A100006D110F8012B03E010F8016B01F8016B0F
:100A20005B1EF9D12B0705D40023521E0DD401F80B
:100A3000013BFAE710F8013BCB1A921C03E013F8D4
:100A4000015B01F8015B521EF9D5A142D8D3002009
:100A500070BD10B50146806B026C12F0500F05D0CE
:100A6000026CD20626D500F04DFF10BD016C41F49A
:100A70000071016401688A6812F0405F17D1027E3C
:100A8000AAB9CA6A12F4700F02D08A6852050ED44D
:100A90004A6822F020024A60016C21F480710164EE
:100AA000016CC90403D4016C41F00101016400F040
:100AB00027FF10BD806BC26CBDE810400846104790
:100AC00010B5806B40210164416C41F00401416428
:100AD00000F018FF10BD10B5806B00F012FF10BDC4
:100AE000464910B54A6822F440324A604A68436871
:100AF0001A434A6001684A6822F480724A600168B9
:100B00004A68036942EA03224A6001684A6822F09F
:100B100040724A6001684A6883681A434A60016803
:100B20008A6822F400628A6001688A68C3681A438E
:100B30008A60816A6FF07062D14201688A6822F02F
:100B400070628A6001688A680CD0836A1A438A607E
:100B500001688A6822F040528A6001688A68C36A24
:100B60001A4301E022F040528A6001688A6822F04C
:100B700002028A6001688A68037E42EA43028A6050
:100B800090F82010002901684A680FD042F40062F2
:100B90004A6001684A6822F460424A6001684A6813
:100BA000174C436A04EB43331A4301E022F400621A
:100BB0004A600168CA6A22F47002CA620168CA6A9D
:100BC000838B104C04EB03531A43CA6201688A6892
:100BD00022F400728A6001688A6890F8303042EA34
:100BE00043228A6001688A6822F480628A60016810
:100BF0008A68406942EA8020886010BD0023014075
:100C000000E0FFFF0000F0FF0EB50A230092CDE9DF
:100C1000011302460123A021014801F039FB0EBD5A
:100C20008C0400200EB50A230092CDE90113024680
:100C30000123A021014801F02DFC0EBD8C040020F1
:100C4000FEE70000014800F0D3BF00005805002077
:100C50007FB51D481E4C1E4900681C4D1C4B603C56
:100C6000B839A84202D9194A543A03E0984203D944
:100C7000164A583A126804E0A04201D94A6800E0D6
:100C80000A6812F0200F19D02022A84202D90F487A
:100C90004C3803E0984203D90C485038026004E015
:100CA000A04201D9CA6000E08A600E220949684664
:100CB000FFF752FB9DE80F0000F04AFC04B0024829
:100CC000BDE8704000F094BF2C040020586402403E
:100CD000B8600240D4030020014800F089BF000042
:100CE000F4060020014800F083BF000054070020F4
:100CF00001681823CAB2103AB2FBF3F2054B6FF346
:100D00000901032A9B5CC36500D9091D816508465A
:100D10007047000038D6050810B5014600208B69E1
:100D20008A6A4FF0C07453B1B3F5005F15D072B149
:100D3000012A0CD0022A0AD0032A09D104E01AB1F0
:100D4000012A06D0022A03D1C96AC90100D50120AF
:100D500010BDC96AA142FAD010BD002AF7D0012AFD
:100D6000F2D0022AF3D0032AF3D010BD30B50468C4
:100D7000256825F480252560046863608368402B1E
:100D8000036803D099600068C26030BD9A60006853
:100D9000C16030BD704708B50A2001F09BF86A4673
:100DA00002210020FFF730FF9DF80000552803D1F5
:100DB0009DF80100AA2821D055208DF80000AA2016
:100DC0008DF801000A2001F085F86A460221002012
:100DD000FFF728FF002000900A2001F07BF86A4608
:100DE00002210020FFF710FF9DF80000552803D1D5
:100DF0009DF80100AA2801D0012008BD002008BDEF
:100E00001CB56A4605211020FFF7FEFE9DF8001074
:100E10000E48642900D93C2101709DF80110012978
:100E200000D9012141709DF80210012900D900214B
:100E30008170BDF8031039B15A2905D0B42903D007
:100E4000B1F5877F00D0B42181801CBD8C020020C9
:100E50001CB50B486A4601788DF8001041788DF872
:100E6000011081788DF8021080888DF80300000A47
:100E70008DF8040005211020FFF7D4FE1CBD0000F2
:100E80008C0200200EB510B107A007C801E009A22E
:100E900007CA8DE807006846FFF782FA81B26A4602
:100EA0002020FFF7BFFE0EBD7570646174650D0AEA
:100EB000000000002D6E6F70652D0D0A000000000F
:100EC00072B6FEE71CB5094BD3E90023CDE9002338
:100ED00090F85020022A03D25DF8222090471CBDD2
:100EE000002180F8501008461CBD000040D60508BF
:100EF00010B578B190F836301C060BD511B1C3F39C
:100F000002130B7022B190F8360000F00F00107041
:100F1000002010BD022010BD11B190F84E300B70B2
:100F200012B190F84F0010700020704710B51346B2
:100F300009B1828A0A8043B1818AC1F302318A00F1
:100F400000F116011846FFF707FA002010BD000057
:100F500070B50446007878B1606878B1A06878B15F
:100F6000012304F1370216461946204625F054F8AD
:100F700050B14AA020612CE04DA002E051A000E059
:100F800057A02061022070BD94F83700000603D4FA
:100F90005AA02061042070BD002084F85000A08277
:100FA000202104F11600FFF7F0F9012584F84150E3
:100FB0002B4604F141020C21204625F043F800287D
:100FC00063D10F2304F136020121204625F024F8D5
:100FD00008B1082070BD032084F83700202084F871
:100FE0003800312084F8390003233246022120469C
:100FF00025F028F8F0BB94F83E00012340F00700EC
:1010000084F83E0004F13E020921204625F01AF83A
:1010100080BB252084F83F00012304F13F020A2110
:10102000204625F00FF828BBE22084F84300012376
:1010300004F143020E21204625F004F8D0B9FE2029
:1010400084F84400012304F144020F21204624F0D7
:10105000F9FF78B994F83B00012320F0200084F8D0
:101060003B0004F13B020621204624F0EBFF08B9C7
:10107000072000E009E084F84000012304F1400269
:101080000B21204624F0DEFF08B1102070BD84F84B
:10109000515006A02061002070BD000044657669B3
:1010A0006365206E6F7420666F756E6400000000CB
:1010B000496E76616C696420693263206164647290
:1010C00065737300496E76616C6964206932635F91
:1010D000726561642066756E6374696F6E000000EE
:1010E000496E76616C6964206932635F77726974F6
:1010F000652066756E6374696F6E0000496E766177
:101100006C696420646576696365207665727369CD
:101110006F6E00002DE9F0410F4600F149020446D0
:1011200001239046402124F077FF58B994F84900F4
:10113000002500F00306012342464021204624F00A
:101140006BFF10B10820BDE8F08194F8490000F071
:101150000300864201D00120F5E76D1CEDB2052D9C
:10116000E9D33E700020EEE770B5044690F85100D8
:101170000D46A84215D094F83F0015B120F080002C
:1011800001E040F0800084F83F00012304F13F02B9
:101190000A21204624F056FF08B1102070BD84F8C3
:1011A0005150002070BDF8B50D460446072300F1EC
:1011B00045023C2124F030FF08B10820F8BD94F826
:1011C0004C0094F84710084384F84C0094F84D0004
:1011D00094F84810084384F84D0094F85110002604
:1011E00031B394F84910090622D4032084F837005B
:1011F000202084F83800312084F83900032304F1DA
:1012000037020221204624F01DFF00BB072084F88E
:101210004000012304F140020B21204624F012FF7C
:10122000A8B984F85060F5B3287840F002004AE08D
:1012300094F84510C9070CD002208DF80000012356
:101240006A460C21204624F0FDFE0028B6D010206E
:10125000F8BDC10708D020F0010084F84D001DB191
:10126000287840F00800287094F84A00800623D4BB
:1012700003236A464321204624F0CEFE70B9BDF810
:101280000100A082C0F30230042101EB800304F1CD
:1012900016024321204624F0BFFE78B194F83C00AA
:1012A00040F0040000E007E08DF8000001236A46EA
:1012B0000721204624F0C6FE0020F8BD002DFBD0FB
:1012C000287840F004002870F6E72DE9F0470D4635
:1012D0000446012300F14902402124F09DFE00282C
:1012E00055D194F84900000678D50F2084F84000C5
:1012F000012304F140020B21204624F0A3FE002824
:101300006AD1E16802208847072684F837604FF0E9
:10131000200884F83880312084F8390004F137023D
:10132000032392460221204624F08CFE90BBE16804
:101330000220884704F14E0702E0E1680220884756
:1013400039462046FFF7E6FE0028F6D10B2784F841
:101350003770012352460221204624F073FEC8B99B
:10136000E1680220884704F14F0902E0E1680220A9
:10137000884749462046FFF7CDFE0028F6D10223D4
:1013800004F147023E21204624F046FE18B1082011
:10139000BDE8F08720E0002084F84C0084F84D0080
:1013A00094F84E0018B184F83760252005E094F8D1
:1013B0004F0028B184F83770262084F8380004E004
:1013C000032084F8370084F83880022352461946F7
:1013D000204624F037FE10B11020D9E707E00120A5
:1013E00084F850001DB1287840F0010028700020DA
:1013F000CEE738B5044690F83E00012340F04000A7
:101400008DF800006A460921204624F01BFE68B9C9
:10141000E1680620884702208DF8000001236A4613
:101420000C21204624F00EFE002800D0102038BDEC
:1014300030B58BB012258DF800508DF801508DF825
:101440000250132504468DF80350C1F302300225E3
:1014500005EB800545F080058DF804508DF80510EA
:10146000090A8DF8061000210DF107030DE020CACE
:1014700003F8015B2D0A03F8015B2D0A03F8025BF8
:101480002D0A491C03F8015CC9B28142EFD3FF2049
:1014900003F8010B142003F8010BFE2003F8020BE4
:1014A000A12003F8010C6846181AC3B26A4643210A
:1014B000204624F0C7FD10B110200BB030BDE1680C
:1014C000022088470020F8E72DE9F04186B014217A
:1014D0006846FEF75AFF1B480024016841F00101ED
:1014E0000160016801F001010591016841F002010C
:1014F00001600068144F00F00200059001220821ED
:10150000384600F0F6FDDFF844804FF40046002234
:101510003146404600F0EDFD082000900125CDE960
:10152000015469463846039400F0E6FC0096CDE984
:10153000015469464046039400F0DEFC06B0BDE865
:10154000F0810000303802400004024000000240F8
:101550002DE9F04FDFF87C8183462DED028B0020D2
:1015600098F800C00E0C140C85B09FB21FFA81FAD7
:1015700095B2BCF1010F06D0BCF1020F05D0BCF151
:10158000030F05D103E0304602E0284600E0204684
:10159000C01B00D540421FFA80F958466CF31F600B
:1015A0008DE80F000E2269464B4802F0FDFC00EE6C
:1015B00010AAF0EE080AB8EE400A20EE200ADFED8D
:1015C000470A98F8000020EE200AF2EE060A0128E9
:1015D00060EE208A04D0022815D0032830D03DE0E8
:1015E00000EE106A00EE907AB8EE400AF8EE600A5B
:1015F00030EE600A10EE100AFFF795F841EC100B80
:101600009FED371B11E000EE105A00EE907AB8EE15
:10161000400AF8EE600A30EE600A10EE100AFFF79A
:1016200082F841EC100B9FED301B51EC100B53EC8A
:10163000112BFEF771FFFFF789F808EE100A0DE095
:1016400000EE104A00EE907AB8EE400AF8EE600A1A
:1016500030EE600ADFED260A20EE208A2548B0EE43
:10166000680A006823F00DFE2348B0EE480A0068BF
:1016700023F007FE0020B9F5F46F0FD998F8012088
:101680004146521CD2B288F8012088F80200082A8C
:1016900016D3487098F80000401C0EE0B9F10F0F07
:1016A000414612D28A78521CD2B28A704870082AF7
:1016B00006D3887098F80000401EC0B20BF042FBC1
:1016C00005B0BDEC028BBDE8F08F487088F80200D1
:1016D000F6E7000088020020AC06002000008039F8
:1016E00000806CF0FFBFD23F008003F5FF4B3D4010
:1016F000001B3745800200208402002070B586B0B0
:101700000D460646144614216846FEF73EFE0020AC
:101710000246059069461F4801F0DAFB002205A940
:101720001C4801F0B3FB9DF8170040F26D1110FB4F
:1017300001F09DF81510C1EB411108449DF81610F9
:1017400008449DF8001000EB400001EBC0004FF48E
:10175000616148439DF80110C1EB011100EB81006C
:101760009DF8021008440C490968431A3C20B3FB59
:10177000F0F100FB11312170B3FBF0F1B1FBF0F29D
:1017800000FB121028704FF46160B3FBF0F0307072
:1017900006B070BDE00400200400002078B50024ED
:1017A000009490F83C20012A19D0012280F83C20B6
:1017B0000A6807230568092A13D9EE680A3A02EB7A
:1017C000420293409E43EE600B788A680A3B03EB2B
:1017D00043039A400368DD682A43DA6010E0022080
:1017E00078BD2E6902EB420293409E432E610B7836
:1017F0008A6803EB43039A4003681D692A431A6110
:101800004A681F23072A13D205686E6B521E02EB2B
:10181000820293409E436E630A8893B20A79521EF5
:1018200002EB820293400268556B2B43536327E01F
:1018300005680D2A12D22E6BD21F02EB8202934052
:101840009E432E630B790A88DB1F92B203EB83035E
:101850009A4003681D6B2A431A6311E0EE6A0D3A41
:1018600002EB820293409E43EE620B790A880D3BA5
:1018700092B203EB83039A400368DD6A2A43DA627B
:101880001B4B0568194A9D420AD10D68122D07D1DC
:10189000556825F400055560556845F48005556088
:1018A00005689D421DD1134D0B68AB4201D0112B31
:1018B00017D1536823F480035360536843F4000343
:1018C00053600968A9420CD10B490C4A0968B1FB65
:1018D000F2F101EB8101490000E0491E009100296D
:1018E000FBD180F83C40002078BD0000002301407F
:1018F00000200140120000109402002040420F001E
:1019000070477047704770B504004FF0000503D072
:10191000206C002610B107E0012070BD204600F0C9
:101920001DF8666484F83C60206CC00610D4206CFE
:1019300020F4885040F0020020642046FFF7D0F8E1
:101940006664206C20F0020040F00100206400E09A
:10195000012584F83C60284670BD000070B586B053
:10196000064614216846FEF710FD24493068884277
:1019700042D123480025016841F48071016000686C
:101980001F4900F4807014390590086840F0010088
:101990000860086800F001000590086840F0020047
:1019A00008600868032400F002000590E0208DE83C
:1019B00031006946134800F09FFA009469461248C6
:1019C000CDE9014500F098FA114C1048C4E9000532
:1019D0000015A560C4E90350400060618000A0616B
:1019E0004011C4E907052046656200F0D1F908B14D
:1019F000FFF766FAB463A66306B070BD002001402D
:101A000044380240000002400004024010640240DA
:101A10002C040020F8B5044600200E46009094F8EF
:101A20003C10012907D0012184F83C1021688B6803
:101A3000DB0702D011E00220F8BD8B6843F0010300
:101A40008B603649364B0968B1FBF3F101EB41017C
:101A500000E0491E00910029FBD121688B68DB055D
:101A600003D58B6823F480738B6021688B68DB0758
:101A700049D0236C40F20165AB4343F48073236487
:101A80004968490505D5216C21F4005141F4805184
:101A90002164216CC90404D5616C21F006016164E4
:101AA00000E0606484F83C00A16B1F481D4DC863D2
:101AB000A16B1E480864A16B1D48C86421686FF0C3
:101AC000220008602068416841F080614160206820
:101AD000816841F4807181602168134632464C313F
:101AE000A06B00F0BFF96868C006206802D01149F9
:101AF000884210D1816811F0405F0CD1816841F0BB
:101B00008041816007E0206C40F010002064606C30
:101B100040F0010060640020F8BD00009402002045
:101B200040420F0000230140530A0008D70A000872
:101B3000C10A0008002001402DE9F0410446876DEC
:101B400000F0DCFA064694F835000025022806D09D
:101B50008020606584F834500120BDE8F081206861
:101B6000016821F0160101602068416921F08001BF
:101B70004161206C08B9A06C20B12068016821F097
:101B8000080101602068016821F0010101600CE09A
:101B900000F0B4FA801B052807D9202060650320D7
:101BA00084F8350084F83450D7E720680068C0070F
:101BB000EED194F85C103F208840B860012084F892
:101BC000350084F834500020C7E790F8351002291A
:101BD00003D08021416501207047052180F8351030
:101BE0000068016821F001010160002070470000D9
:101BF0002DE9F84304464FF00009CDF80090634802
:101C00004FF41651A56D0068B0FBF1F72E6894F8FB
:101C10005C10082000FA01F131420FD021680A68F7
:101C200052070BD50A6822F004020A6094F85C108F
:101C30008840A860606D40F00100606594F85C1019
:101C40004FF0010808FA01F0304208D021684969D4
:101C5000090604D5A860606D40F00200606594F844
:101C60005C1004208840304208D021680968890748
:101C700004D5A860606D40F00400606594F85C10C5
:101C800010208840304218D021680968090714D50F
:101C9000A86020680168490304D50068000308D5DE
:101CA000A16C07E00168C90503D4016821F00801AF
:101CB0000160216C09B12046884794F85C1020200F
:101CC0008840304231D021680968C9062DD5A86006
:101CD00094F8350005282068016806D0490347D5E7
:101CE000006800031DD4616C1CE021F01601016046
:101CF0002068416921F080014161206C08B9A06C25
:101D000020B12068016821F00801016094F85C109E
:101D10003F208840A86084F8358084F83490216D95
:101D20001FE0E16B09B120468847606D00282BD089
:101D3000606DC00714D0052084F835002068016864
:101D400021F0010101600098401C0090B84203D8C6
:101D500020680068C007F6D184F8358084F8349094
:101D6000E16C002910D001B02046BDE8F0430847DF
:101D70000168C905D5D4016821F01001016084F81B
:101D8000358084F83490CCE7BDE8F88394020020D5
:101D90002DE9F041044600F0B1F906465CB102209D
:101DA00084F83500002584F834502068016821F05B
:101DB000010101600DE00120BDE8F08100F09EF915
:101DC000801B052805D920206065032084F8350094
:101DD000F2E720680068C007F0D122681168204847
:101DE0000140D4E901031843D4E9033633431843CF
:101DF00063691843A3691843E3691843236A1843C6
:101E00000843616A042903D1D4E90B131943084339
:101E1000106020684069666A20F0070130460E4372
:101E2000012704280CD1A06A0643E06A40B120468D
:101E3000FEF772FF20B14020606584F83570BAE784
:101E4000206846612046FEF753FF94F85C203F214E
:101E500091408160656584F835700020ACE7000032
:101E60003F8010F02DE9F0410446866D90F8340073
:101E7000002501280DD0012084F8340094F8357035
:101E80000020012F07D084F8340002252846BDE841
:101E9000F0810220FBE7022784F835706065204658
:101EA000FEF764FF94F85C103F208840B060206823
:101EB000016841F016010160206C20B120680168C2
:101EC00041F0080101602068016841F001010160F2
:101ED000DCE7000070B5044600F010F90546601C10
:101EE00002D004480078044400F008F9401BA042E6
:101EF000FAD370BDD00100202DE9F84FDFF8B8A16A
:101F00000022012403254FF00F090AF1040BAAF166
:101F1000040E00BF0B6804FA02F63340B34273D1DB
:101F20000F7907F00307012F01D0022F16D1876820
:101F30004FEA420805FA08FC27EA0C07D1F80CC062
:101F40000CFA08FC4CEA070CC0F808C04768B74315
:101F50000E79C6F3001696403E4346600E79F6436E
:101F6000B6070DD0C768560005FA06FC27EA0C072D
:101F7000D1F808C00CFA06FC4CEA070CC0F80CC0FB
:101F80000E7906F00306022E10D1D60800EB860863
:101F9000D8F8206057074FEAD76C09FA0CF7BE4310
:101FA0000F6907FA0CF73743C8F8207006684FEA44
:101FB000420C05FA0CF7BE430F7907F0030707FA46
:101FC0000CF7374307604E6816F4403F6DD03B4E28
:101FD000376847F480473760366822F0030706F415
:101FE00080460096364E07EB060CDCF8086897072B
:101FF0003F0F09FA07F826EA0806DFF8C8804045CF
:1020000003D14FF000081EE04FE0DFF8BC804045F0
:1020100002D14FF0010816E0DFF8B080404502D150
:102020004FF002080FE0DFF8A880404502D14FF0E2
:10203000030808E0DFF89C80404502D14FF0040817
:1020400001E04FF0070808FA07F848EA0608CCF85C
:102050000888DAF800605746D1F804C09E435FEA6A
:10206000CC2C00D51E433E60DBF800605F46D1F803
:1020700004C09E435FEA8C2C00D51E433E60DEF810
:1020800000607746D1F804C09E435FEA8C3C00D5DF
:102090001E433E60084F083F3E68D1F804C09E438F
:1020A0005FEACC3C00D51E433E60521C102AFFF470
:1020B00031AFBDE8F88F0000083C014044380240D1
:1020C00000300140000002400004024000080240CD
:1020D000000C0240001002400069084000D00120BE
:1020E0007047426921EA02030A4043EA02418161E2
:1020F00070470AB1816170470904FBE701488068B5
:1021000070470000D001002070B5040025D094F87D
:102110003D00002520B984F83C50204600F052FADA
:10212000242084F83D002068016821F0010101604D
:102130002068016841F4004101602068016821F4D1
:102140000041016000F09AFC4D4A6168914201D85B
:102150004C4900E04C49884201D2012070BD4B49F6
:102160002368B0FBF1F15E6826F03F060E435E6027
:102170006368934206D94FF4967359434FF47A73C8
:10218000B1FBF3F12368491C1E6A26F03F06314378
:1021900019626168914210D84900401EB0FBF1F20B
:1021A000521CC2F30B02042A01D2042022E0B0FB2D
:1021B000F1F0401CC0F30B001CE0A268F2B301EB8D
:1021C000C10303EB0116431EB3FBF6F35B1C43F4A0
:1021D00080431B0549D092B301EBC10202EB011110
:1021E000401EB0FBF1F0401CC0F30B0040F48040F7
:1021F00040F400402168CA694CF6FF739A431043CB
:10220000C861D4E9071001432068026822F0C002C7
:1022100011430160D4E9030101432068826848F258
:10222000FF339A4311438160D4E9050108432168D3
:10223000CA6822F0FF021043C86001E00EE016E019
:102240002068016841F0010101602564202084F8C4
:102250003D00256384F83E50002070BD01EB41062F
:10226000431EB3FBF6F35B1CB3E70120C2E701EBAF
:102270004101401EB0FBF1F0401CC0F30B00B7E77A
:10228000A086010080841E0000093D0040420F002E
:102290002DE9FF4F83B09A46DDE911879346044646
:1022A000DDF84090FFF72AFF054694F83D0020280E
:1022B00070D11923012274492046009502F04AF892
:1022C0000028F5D194F83C00012863D0012084F85F
:1022D0003C0020680168C90703D1016841F0010191
:1022E00001602068016821F400610160222084F807
:1022F0003D00402084F83E0000262664C4F8249067
:10230000A4F82A80608D20856048E062CDE90075E0
:1023100053465A462046049901F01EFF002879D101
:10232000208DD0B1012821D00228206824D0416915
:1023300080690090208D032866D801282BD054494D
:1023400002283B464FF00002009557D088462046B1
:1023500002F000F800285DD13AE020684169816907
:102360000091016841F4007101607DE0206801681E
:1023700021F480610160F0E7016821F4806101606F
:102380002068016841F4006101602068416980694A
:10239000009069E075E02A463946204602F080F850
:1023A00088BB54E02068016841F400710160206836
:1023B0000069616A0870606A401C6062218D491E74
:1023C0002185618D491E618521680969017042E09E
:1023D0002068016821F48061016020680069616AF9
:1023E0000870606A401C6062208D401E2085608DF0
:1023F000401E60853B46002241460095204601F084
:10240000A9FF00B9CEE705E02A463946204602F08A
:1024100047F818B1012007B0BDE8F08F20680069C7
:10242000616A0870606A401C6062208D401E81B243
:102430002185608D401E608520684269D243520725
:1024400012D4032903D1016821F48061016020685E
:102450000069616A0870606A401C6062208D401EDD
:102460002085608D401E6085208D00287FF462AF3E
:10247000202084F83D0084F83E6084F83C60002011
:10248000C9E70220C7E70000020010000000FFFFBC
:10249000040001002DE9FF4F83B09A46DDE9119752
:1024A00093460446DDF84080FFF728FE054694F881
:1024B0003D0020287FD11923012240492046009564
:1024C00001F048FF002876D194F83C00012872D032
:1024D000012084F83C0020680168C90703D1016825
:1024E00041F0010101602068016821F40061016090
:1024F000212084F83D00402084F83E000026266418
:10250000C4F82480A4F82A90608D20852C48E062CD
:10251000CDE9007553465A462046049901F09AFECB
:1025200070B930E02A463946204601F0F1FF58B133
:10253000206C042804D12068016841F40071016016
:10254000012007B0BDE8F08F606A2168007808615B
:10255000606A401C6062218D491E89B22185628DAE
:10256000521E628522685369DB435B070BD469B155
:1025700000781061606A401C6062208D401E2085DA
:10258000608D401E6085208D0028CBD12A463946BB
:10259000204601F0B3FE0028CAD154F83D0B016873
:1025A00041F400710160202004F81E09E677667787
:1025B0000020C6E7FFE70220C3E70000020010008A
:1025C0000000FFFF10B586B0044614216846FDF7F1
:1025D000DCFE13492068884220D11248002102689D
:1025E00042F002020260006800F002000590C02084
:1025F00000901220CDE901010320039004200490F3
:1026000069460948FFF778FC06481030016841F434
:1026100000110160006800F40010059006B010BDC4
:1026200000540040303802400004024002488168F3
:102630000278114481607047D00100200B4810B52A
:10264000016841F400710160016841F4806101603A
:10265000016841F480710160032000F099F80F20B7
:1026600000F006F800F04AF8002010BD003C0240DF
:1026700030B505461C4887B00024016841F480212C
:102680000160006806A900F48020009001A800F015
:10269000D5F900F003FA1549154AB0FBF1F11548D8
:1026A000491E026040F2E732C0E90324C0E9011488
:1026B000846100F0F7FE040012D10E4800F064FFC0
:1026C00004000DD11A2000F035F8102D07D2002299
:1026D00029461A2000F03CF80748056000E0012474
:1026E00007B0204630BD00004438024040420F0091
:1026F00000480140B4070020D40100200C4882B0FB
:10270000016841F480410160006800F4804000905D
:102710000748001F016841F08051016000680022F5
:1027200000F0805000900F21901E02B000F010B811
:1027300044380240002809DB00F01F0201219140CB
:102740004009800000F1E020C0F80011704700004F
:10275000F0B40E4B1B680C46C3F30223C3F107050C
:10276000042D00D90425191D072901D2002300E0FA
:10277000DB1E012606FA05F1491E214099409E40C4
:10278000761E16403143F0BC03F0F4BC0CED00E0C3
:10279000064900F0070208684FF6FF03184040EAB8
:1027A0000220034A10430860704700000CED00E06F
:1027B0000000FA052DE9F843044600684FF00109CE
:1027C000C1074FF0000601D1400729D5DFF820816D
:1027D000C8F86860FFF792FC0746464D05E000BF69
:1027E000FFF78CFCC01B022859D828680001F7D4D9
:1027F000A068217B800140EA0170616808433D497F
:1028000084310860C8F86890FFF778FC074604E058
:10281000FFF774FCC01B022841D828680001F7D5D7
:102820002078800752D533484030016841F080510C
:1028300001600068304D00F080500090286840F43E
:1028400080702860FFF75AFC074604E0FFF756FC4B
:10285000C01B022823D82868C005F7D5254D703540
:10286000286810F4407020D0218A01F44071814220
:102870001BD02868214920F44070C1F800900E60F8
:1028800028602868C00710D0FFF738FC064641F2E0
:10289000883707E0FFF732FC801BB84202D90320DB
:1028A000BDE8F88328688007F4D521691148C1F391
:1028B00001220830032A12D0016821F4F8110160C6
:1028C0002868218AC1F30B0108432860207800079B
:1028D00003D50B49207DC1F8E0010020E0E7026844
:1028E000084B22F4F81219400A430260E8E700009E
:1028F000000047420038024000700040400E47424E
:1029000000104742FFFCFF0F2DE9F0470E4605007F
:1029100065D0DFF81481D8F80000F7B200F00700A6
:10292000B04207D288F80070D8F8000000F0070025
:10293000B04254D128683D4C810712D5400703D5D9
:10294000206840F4E05020602878000703D5206814
:1029500040F4604020602068A96820F0F00008433F
:1029600020602878C0072DD03049686808390128D0
:1029700012D0022813D0032811D009688907002932
:102980002DDA216821F0030101432160FFF7B6FB36
:10299000814641F2883A0EE009688903EFE7096849
:1029A0008901ECE7FFF7AAFBA0EB0901514502D929
:1029B0000320BDE8F0872068696800F00C00B0EBE8
:1029C000810FEFD1D8F80010404601F00701B14265
:1029D00007D90770006800F00700B04201D001205D
:1029E000E7E72878400705D52068E96820F4E0503B
:1029F000084320602878000706D52068296920F45C
:102A0000604040EAC100206000F058F82168084AA0
:102A1000C1F30311515CC8400649086006480068CC
:102A2000FFF726FE0020C4E7003C024008380240C1
:102A300011DB050894020020D40100200F2202605F
:102A40000C4A136803F003034360136803F0F003B8
:102A50008360136803F4E053C36012684FF4E053DB
:102A600003EAD20202610448006800F0070008602F
:102A70007047000008380240003C02400448054905
:102A800000680968044AC1F38221515CC84070475C
:102A9000940200200838024021DB0508044805495B
:102AA00000680968044AC1F34231515CC84070476C
:102AB000940200200838024021DB0508154810B5B3
:102AC000006810F00C02144813D01449042A0FD0E7
:102AD000082A0ED10F4C241F2268236802F03F02FF
:102AE0005B0207D52068C0F38810A0FB010106E057
:102AF000084610BD2168C1F38811A1FB0001002325
:102B0000FDF7C8FB2168C1F30141491C4900B0FB36
:102B1000F1F010BD083802400024F40040787D0137
:102B20002DE9F84F04006ED02078DFF84C93C007F1
:102B3000A9F104054AD009F104000168C1F381013B
:102B4000012908D00068C0F3810002280AD1D9F811
:102B50000000400206D52868800337D56068002849
:102B6000E1D033E06068B0F5803F10D0B0F5A02F21
:102B7000286810D020F480302860286820F4802055
:102B800028606068A8B1FFF7B9FA06460DE028682A
:102B900040F48030F4E740F480202860F7E700BF7D
:102BA000FFF7ACFA801B642873D828688003F7D538
:102BB0000CE0FFF7A3FA064605E000BFFFF79EFA18
:102BC000801B6428F0D828688003F7D42078DFF8C9
:102BD000AC8280074FF0000A3ED5A748001D01686F
:102BE00011F00C0F08D00068C0F3810002280BD14F
:102BF000D9F80000400207D42868800716D5E0689D
:102C0000012800D112E033E1E068B8B10120C8F832
:102C10000000FFF773FA064605E000BFFFF76EFA03
:102C2000801B0228C0D828688007F7D5286821694A
:102C300020F0F80040EAC10028600DE0C8F800A0CC
:102C4000FFF75CFA064604E0FFF758FA801B0228FB
:102C50001FD828688007F7D42078000722D5864F30
:102C600087486169703771B101210160FFF746FA49
:102C7000064604E0FFF742FA801B022809D83868AC
:102C80008007F7D50EE0C0F800A0FFF737FA064638
:102C900005E082E0FFF732FA801B02287DD8386811
:102CA0008007F7D42078400768D5DFF8CCB100273B
:102CB0000BF13C0BDBF80000C0000BD4DBF800107C
:102CC00041F08051CBF80010DBF80000012700F044
:102CD000805000906B4E3068C00510D4306840F4CE
:102CE00080703060FFF70AFA009005E0FFF706FAFF
:102CF0000099401A022850D83068C005F6D55E4EBB
:102D0000A0686C3601280FD00528306810D020F05C
:102D100001003060306820F004003060A068B8B175
:102D2000FFF7ECF900900FE0306840F00100F4E7A5
:102D300040F004003060F7E7FFF7E0F90099411A2E
:102D400041F28830814266D830688007F4D50EE0C1
:102D5000FFF7D4F9009007E0FFF7D0F90099411A86
:102D600041F28830814256D830688007F4D42FB1C0
:102D7000DBF8001021F08051CBF80010A069C8B337
:102D80003D49091D0968C1F3810102294AD0022881
:102D9000504607D0C8F8600000E03CE0FFF7AEF90D
:102DA00004463BE04746C8F86000FFF7A7F906462F
:102DB00005E000BFFFF7A2F9801B02282BD8286886
:102DC0008001F7D4D4E907010843A16A2E4A4908D3
:102DD00002EB0141626A41EA8211084394F82C1027
:102DE00040EA0161C9F8001001203866FFF786F952
:102DF000044606E03EE000BFFFF780F9001B022812
:102E000009D828688001F7D534E000BFFFF776F9CC
:102E1000001B022802D90320BDE8F88F2868800132
:102E2000F4D427E00128F7D0D9F80000E26900F4D3
:102E3000800191421CD1226A00F03F01914217D1DA
:102E400047F6C071626A0140B1EB821F10D1A26ADD
:102E50004FF0FF3300F4403103EB5202B1EB024F6D
:102E600006D194F82C1000F07060B0EB016F01D027
:102E70000120D1E70020CFE704380240000047429C
:102E8000800E4742007000400000FFFF10B5006850
:102E90000B4641680D480140080CD870C1F304246A
:102EA0005C7001F03F049C70C1F34231197052B95B
:102EB00002F0E0FAD870587802F0DCFA587098788E
:102EC00002F0D8FA9870002010BD00003FFFFF000C
:102ED00010B50B460168896A596001680969C1F338
:102EE0000E019960006801680D480140C1F305407A
:102EF0001870C1F306245C7001F07F049C70890D8A
:102F0000D97052B902F0B6FA1870587802F0B2FAD5
:102F10005870987802F0AEFA9870002010BD00004A
:102F20007F7F7F0010B5040002D0607F10B106E003
:102F3000012010BD00202077204600F041F802203B
:102F400060772068C168C943C90632D5CA21416289
:102F5000216853204862204602F096FA20BB206880
:102F60008168164A11408160216888686268104350
:102F7000D4E904231A43104388602168E06808619B
:102F800020680169228941EA02410161204602F07C
:102F90009FFA48B921680A6C22F480220A642168E9
:102FA0000A6CA3691A430A642268FF21516208B1BE
:102FB00010BD00200121617710BD0000BFFF8FFF11
:102FC00010B586B0044618216846FDF7DEF90949B8
:102FD000206888420CD102200090000204906846CC
:102FE000FFF7E8FB08B1FDF76BFF0349012008601C
:102FF00006B010BD002800403C0E474270B50446A4
:103000000B482168C860FFF779F805464FF47A76D7
:1030100007E000BFFFF772F8401BB04201D9032060
:1030200070BD2068C0688006F4D5002070BD000027
:103030005F3F0100704770B5040009D0606A002549
:1030400040B125616561A56294F8510040B10CE082
:10305000012070BD6068B0F5827FF4D0E561F2E7D1
:1030600084F85050204600F045F8022084F85100C2
:103070002068016821F040010160A088218900F4E6
:10308000827001F404410843A18901F400610843FE
:10309000217C01F002010843217D01F00101084378
:1030A000218B01F400710843217F01F038010843AE
:1030B00094F8201001F080010843218D01F40051A3
:1030C000084321680860A069042101EA104094F8CF
:1030D000241001F010010843216848602068C1698C
:1030E00021F40061C1616565012084F85100002070
:1030F00070BD000070B586B0064614216846FDF725
:1031000044F920493068884239D11F4800250168B8
:1031100041F480410160006800F4804005901A4845
:103120001038016841F0020101600068694600F052
:10313000020005904FF4204000900220CDE90105E7
:1031400003200390052004901048FEF7D5FE114C93
:103150000F48C4E900054020C4E9020500012061D0
:10316000400060618000C4E9060525622046656272
:10317000FEF70EFE08B1FDF7A3FEB464A66306B029
:1031800070BD00000038004040380240000402409A
:1031900070600240580500202DE9F84F9846164609
:1031A0008A460446FEF7AAFF814694F8510001289A
:1031B0001ED1BAF1000F73D0002E71D094F85000D8
:1031C000012815D0012784F85070032084F851009D
:1031D00000256565C4F830A0A686E686A563A587A8
:1031E000E58765642564A068B0F5004F03D00CE066
:1031F0000220BDE8F88F2068016821F040010160DD
:103200002068016841F48041016020680168490636
:1032100003D4016841F040010160E068B0F5006F3F
:10322000606803D048B3012E27D047E008B1012ED3
:103230001FD1206B21680088C86006E02068816883
:10324000890709D5216B0988C160206B801C206328
:10325000E08E401EE0860CE0FEF750FFA0EB090177
:10326000414503D3B8F1FF3F03D035E0B8F1000F7B
:1032700032D0E08E0028E1D123E0206B2168007875
:10328000087306E02068816889070AD5216B0978F0
:103290000173206B401C2063E08E401EE0860DE031
:1032A0002BE0FEF72BFFA0EB0901414503D3B8F15A
:1032B000FF3F03D010E0B8F1000F0DD0E08E0028E2
:1032C000E0D14A464146204602F060F908B120208C
:1032D0006065A06830B109E084F8517084F85050FE
:1032E000032086E72068C1688068009084F85170E8
:1032F00004F8505F60680028F3D0012079E70000EF
:1033000070B5044690F8510001281CD1C9B1C2B172
:1033100094F85000012816D0012084F850000320B2
:1033200084F85100002565652163A286E286A563C5
:1033300065642564A587E587A068B0F5004F04D0D3
:103340000DE0012070BD022070BD2068016821F0F1
:10335000400101602068016841F480410160A16C76
:1033600017480864A16C1748C863A16C1648C86464
:10337000A06C0565E38E2268216B0C32A06CFEF711
:1033800071FD30B1606D40F01000606584F8505000
:10339000D7E720680168490603D4016841F040017D
:1033A000016084F850502068416841F0200141607C
:1033B0002068416841F002014160002070BD0000BA
:1033C0001D55000827550008FB540008704770473A
:1033D0007047704710B590F83C20012A22D0012296
:1033E00080F83C20CA688C6822F4407222434C6802
:1033F00022F4806222430C6822F4006222430C69AA
:1034000022F4805222434C6922F400522243C969BB
:10341000002322F480420A4301684A6480F83C3069
:10342000002010BD022010BD70B590F83C20012A8C
:103430002CD0012480F83C40022280F83D20036813
:103440005A689D6822F070060A6832435A60104B31
:1034500002689A420ED0B2F1804F0BD00D4B9A42C7
:1034600008D00D4B9A4205D00C4B9A4202D00C4B1F
:103470009A4204D1496825F080031943916080F88D
:103480003D40002180F83C10084670BD022070BD10
:10349000000001400004004000080040000C004013
:1034A0000040014010B5040003D094F83D0010B175
:1034B00007E0012010BD002084F83C00204600F009
:1034C0001FF8022084F83D00211D206802F0DCF97D
:1034D000012084F8460084F83E0084F83F0084F818
:1034E000400084F8410084F8420084F8430084F8E6
:1034F000440084F8450084F83D00002010BD000021
:1035000008B50068B0F1804F08D10548016841F066
:1035100001010160006800F00100009008BD00009A
:103520004038024090F83D10012901D00120704739
:10353000022180F83D1000680E4988420ED0B0F19B
:10354000804F0BD00C49884208D00C49884205D0E6
:103550000B49884202D00B49884204D1816801F0AE
:103560000701062903D0016841F001010160002034
:1035700070470000000001400004004000080040C7
:10358000000C00400040014090F83D10012901D09E
:1035900001207047022180F83D100168CA6842F09E
:1035A0000102CA6000680E4988420ED0B0F1804F17
:1035B0000BD00C49884208D00B49884205D00B49F2
:1035C000884202D00A49884204D1816801F007018B
:1035D000062903D0016841F0010101600020704715
:1035E000000001400004004000080040000C0040C2
:1035F0000040014070472DE9F04104460068C6686C
:1036000005694FF00007A90713D5B10711D5F91EB9
:10361000016101202077206880698007204602D060
:10362000FFF7E8FF04E000F0C1F8204600F07EF963
:103630002777680716D5700714D521686FF0040046
:103640000861022020772068806910F4407F2046BE
:1036500002D0FFF7CFFF04E000F0A8F8204600F00A
:1036600065F92777280715D5300713D521686FF03E
:1036700008000861042020772068C0698007204680
:1036800002D0FFF7B7FF04E000F090F8204600F00A
:103690004DF92777E80616D5F00614D521686FF0A6
:1036A00010000861082020772068C06910F4407F6E
:1036B000204602D0FFF79EFF04E000F077F8204696
:1036C00000F034F92777E80708D0F00706D0216822
:1036D0006FF001000861204600F0BAF9280608D50D
:1036E000300606D521686FF0800008612046FFF79C
:1036F0006FFE680608D5700606D521686FF0400099
:103700000861204600F0D9F9A8060AD5B00608D508
:1037100021686FF0200008612046BDE8F041FFF706
:1037200058BEBDE8F081000010B586B004461421F3
:103730006846FCF72AFE2368174C0021174802222E
:10374000A34211D1036843F001030360006800F055
:103750000100059050020090CDE901210120CDE942
:10376000031069460E4812E00E4CA34211D10368C3
:1037700043F002030360006800F00200059060154A
:103780000090CDE90121CDE9031269460648FEF714
:10379000B3FB06B010BD000000000140303802400D
:1037A000000002400008004000040240704770B56D
:1037B000044690F83C0000260D4601280FD0012059
:1037C00084F83C006AB1042A1DD0082A2FD00C2AA4
:1037D0003FD00126002084F83C00304670BD022016
:1037E00070BD206802F0BAF82068816941F00801D4
:1037F00081612068816921F004018161206881690B
:103800002A69114311E0206802F0D0F8206881692C
:1038100041F4006181612068816921F480618161E6
:10382000206881692A6941EA02218161D2E7206822
:1038300002F0E8F82068C16941F00801C161206820
:10384000C16921F00401C1612068C1692A6911437D
:1038500011E0206802F002F92068C16941F40061BA
:10386000C1612068C16921F48061C1612068C169BA
:103870002A6941EA0221C161ACE710B5040003D016
:1038800094F83D0010B107E0012010BD002084F83D
:103890003C00204600F01EF8022084F83D00211D67
:1038A000206801F0F1FF012084F8460084F83E0012
:1038B00084F83F0084F8400084F8410084F8420016
:1038C00084F8430084F8440084F8450084F83D00FF
:1038D000002010BD08B500681149884212D1114876
:1038E000016841F0010101600068002200F0010060
:1038F00000900F211A20FEF72BFFBDE808401A2088
:10390000FEF718BF0849884209D10648001F016820
:1039100041F004010160006800F00400009008BD5F
:103920000000014044380240000800407047000099
:1039300010B50446022249B104290ED0082913D03B
:1039400094F84100012816D0012010BD94F83E00E3
:103950000128F9D184F83E200FE094F83F000128B7
:10396000F2D184F83F2008E094F840000128EBD120
:1039700084F8402001E084F841200122206801F011
:10398000D5FF12492068884203D1426C42F40042BC
:103990004264206888420ED0B0F1804F0BD00C49B1
:1039A000884208D00B49884205D00B49884202D092
:1039B0000A49884204D1816801F00701062903D031
:1039C000016841F001010160002010BD00000140CC
:1039D0000004004000080040000C0040004001408E
:1039E00030B504460D460068002201F09FFF174BDA
:1039F00041F2111120688A10984209D1036A0B42E2
:103A000006D1036A134203D1436C23F40043436499
:103A10002068036A0B4206D1016A114203D1016892
:103A200021F00101016001203DB1042D08D0082DD5
:103A300009D084F84100002030BD84F83E00FAE748
:103A400084F83F00F7E784F84000F4E70000014005
:103A500000680349884201D1FEF7E8BD70470000C5
:103A60000048014070B5044690F83C00012812D08F
:103A7000012584F83C50022084F83D00204602F0E5
:103A80000FF801004FF0000007D084F83D5084F893
:103A90003C00012070BD022070BD2168CA6822F080
:103AA0004002CA602168CA6822F48042CA6084F871
:103AB0003D5084F83C00002070BD7047704710B541
:103AC00004460068406994F84110C0F3C0102129F1
:103AD00011D180B12068143050E8001F21F080011E
:103AE00040E80012002AF5D1A06B08B1FEF724F8D7
:103AF000204602F021F92068406994F84210C0F392
:103B00008010222911D180B12068143050E8001FA4
:103B100021F0400140E80012002AF5D1E06B08B125
:103B2000FEF70AF8204602F0E0F8002010BD7047CA
:103B3000F8B5016804460868CA684B6910F00F0FB1
:103B40004FF0000559D003F0010602F49077374397
:103B500065D0C10705D0D10503D5616C41F00101E5
:103B60006164410705D5D90703D0616C41F00201BA
:103B70006164810705D5D90703D0616C41F0040168
:103B80006164010707D502F02001314303D0616C65
:103B900041F008016164616C00293AD0800604D5C7
:103BA000900602D5204602F0D5F820684069616C85
:103BB000C0F38010090700D460B3204602F095F8E6
:103BC00020684069400621D52068143050E8001F65
:103BD00021F0400140E80012002AF5D1E06BA8B1C5
:103BE0006E490165E06BFDF7F0FF002811D0E06B36
:103BF000016D01B0BDE8F040084783060FD593067C
:103C00000DD52046BDE8F84002F0A4B82046FFF7E5
:103C10008EFFF8BD2046FFF78AFF6564F8BD266B6E
:103C20002023012E7DD1C6067BD5D60679D508681E
:103C30004868009048694FF00206400641D5E16BA4
:103C4000086840680004000CE8D0A28D8242E5D9E3
:103C5000E085C869B0F5807F2DD020680C3050E831
:103C6000001F21F4807140E80012002AF5D120687D
:103C7000143050E8001F21F0010140E80012002A32
:103C8000F5D12068143050E8001F21F0400140E8D1
:103C90000012002AF5D184F84230256320680C30E8
:103CA00050E8001F21F0100140E80012002AF5D171
:103CB000E06BFDF741FF6663A08DE18D401A81B294
:103CC0002AE0A08DE18D401A81B2E08D0028A5D0B8
:103CD0000029A3D022680C3252E8000F20F4907023
:103CE00042E80007002FF5D12068143050E8002F7B
:103CF00022F0010240E80027002FF5D184F842307D
:103D0000256320680C3050E8002F22F0100240E8B4
:103D10000023002BF5D166632046FFF7CFFEF8BDE8
:103D2000FFE705062BD5150629D594F84100212873
:103D3000F5D1A068B0F5805F01D12069B0B1206AEB
:103D4000411C2162216800784860E08C401E00041C
:103D5000000CE084E3D12068C16821F08001C160DB
:103D60002068C16841F04001C160D8E7206A00883E
:103D7000C0F308004860206A801C2062E5E7400626
:103D8000CDD55006CBD5CA68204622F04002CA6085
:103D900084F8413000F044F9C1E70000A15B00085D
:103DA00070B5040004D094F84100002510B106E07D
:103DB000012070BD84F84050204600F023F82420F4
:103DC00084F841002068C16821F40051C160204698
:103DD00002F022F82068016921F490410161206815
:103DE000416921F02A0141612068C16841F4005114
:103DF000C1606564202084F8410084F84200656356
:103E0000002070BD2DE9F04186B0064614216846B9
:103E1000FCF7BBFA2F493068884258D12E4800245D
:103E2000016841F020010160006800F02000059069
:103E300029481438016841F00101016000686946B1
:103E400000F0010005904FF4C05000900220CDE931
:103E5000010403200390082004902048FEF74CF84A
:103E6000204D1F484FF4806887052860C5E901741C
:103E7000C5E903486C61AC61EC612C6228466C6258
:103E8000FDF786FF08B1FDF71BF8F563AE63154D2E
:103E9000134860357830E5E802074020A5E81101B5
:103EA000104845F814496030AC61EC612C626C62DA
:103EB000FDF76EFF08B1FDF703F8B5630022052199
:103EC0004720AE63FEF744FC4720FEF733FC06B004
:103ED000BDE8F08100140140443802400000024077
:103EE00028640240F406002090F84230202B01D0D4
:103EF0000220704721B11AB10023036302F012B807
:103F000001207047704770472DE9F843044690F848
:103F10004100984616460D46202802D00220BDE8F2
:103F2000F88385B17EB100206064212084F84100CF
:103F3000FEF7E4F8A6848146E684A0682027B0F561
:103F4000805F02D003E00120E9E7206910B12E462E
:103F500000250EE000260CE08021204602F02AF821
:103F6000A8B9C6B116F8010B21684860E08C401E64
:103F7000E084E08C4B464FF00002CDF80080002832
:103F8000EAD14FF04001204602F014F840B184F825
:103F900041700320C3E735F8020BC0F30800E3E7E4
:103FA00084F841700020BAE770B5044690F84100EB
:103FB000202801D0022070BD49B342B32162A284FF
:103FC000E28400206064212384F84130A56B114B0A
:103FD000EB63A56B104B2B64A56B104BEB64A36BD1
:103FE0001865256813462A1DA06BFDF73BFF216865
:103FF0006FF0400008602068143050E8001F41F066
:10400000800140E80012002AF5D1002070BD012097
:1040100070BD00009F5C0008E15C0008B15B000817
:1040200070477047FEE700002DED028B304F314E98
:10403000314D9FED328A00BF29F0A4FB192230498F
:104040002B48FFF751FF3868C16841F01001C1608B
:104050000D212CA001F09CFD202021F0CBF8306038
:10406000202021F0C7F80024C5F80000B0EE480A6F
:10407000306821F006F9B0EE480A286821F001F90D
:10408000641C202CF2DB234C55202070AA20607089
:104090000320A070FDF718FA032008F053FE052254
:1040A000211D1D48FDF7B6FC1C48FFF73BFA08210F
:1040B0001B48FFF73DFC00F073FAFCF76CFE08B9F3
:1040C000FCF79EFE00224FF480611648FEF711F8BF
:1040D00008F0B0FF01F0ECFA15F06EFC1CF020F8CF
:1040E00028F05CFA2AF014F9002029F07DFAA3E701
:1040F000AC060020800200208402002000000000A6
:1041000090060020706F7765722D7069636F0D0ADD
:1041100000000000D4030020E4030020000600207B
:10412000B80500200004024001684A69D2435205E4
:104130000FD46FF480624A61002140F8301F2022C2
:1041400042738173026942F004020261017301202B
:1041500070470020704700002DE9F84F04460068C2
:1041600089460B9D01689846174641F480610160BD
:104170002068016841F48071016000954FF0011BD7
:104180000022594620460A9B00F0E4F84FF4007ADA
:1041900040B120680068C00501D5C4F840A00320E4
:1041A000BDE8F88F216809F0FE0008612B46284918
:1041B00020460A9A00F016F9F0BB20684169806930
:1041C00000902A4620460A9900F0A2F940B1206CDE
:1041D00004283AD12068016841F40071016034E09C
:1041E000FEB2B8F1010F09D02168380A08612A46E9
:1041F00020460A9900F08CF90028E8D12068066171
:104200002A4620460A9900F083F90028DFD1206869
:10421000016841F4807101600095002259462046F2
:104220000A9B00F097F80028B3D1216809F0FF003D
:1042300040F00100086100E007E02B4604492046F9
:104240000A9A00F0CFF80028AAD00120A8E70000C1
:10425000020001002DE9F843044600680D46DDE93F
:10426000089701689846164641F4807101604B46F4
:1042700000224FF001112046009700F06BF848B182
:1042800020680068C00502D54FF400702064032048
:10429000BDE8F883216805F0FE0008613B464A4608
:1042A0001549204600F09EF888B920684169806968
:1042B00000903A464946204600F02AF948B1206C61
:1042C000042804D12068016841F4007101600120D4
:1042D000DEE7F5B2B8F1010F09D02168300A0861B4
:1042E0003A464946204600F013F90028E7D12068F5
:1042F00005610020CCE700000200010070B5164601
:104300000D4604461EE02046FFF70EFF08B10120CF
:1043100070BD681C16D0FDF7F1FE801BA84200D8C6
:1043200085B920684069C04340070BD5002044F898
:10433000300F20216173A073216941F020012161B8
:104340002073E4E720684069C0434007DBD40020C5
:1043500070BD00002DE9F047984617460D4604460B
:10436000C1F30746DDF820902AE000BFB8F1FF3F17
:1043700026D0FDF7C3FEA0EB0901414502D8B8F1F4
:10438000000F1DD12068012E16D0806925EA00009B
:104390000004000C12D00020B84211D1002044F8D3
:1043A000300F20216173A073216941F02001216148
:1043B00020730120BDE8F0874069E7E70120EBE7C3
:1043C0002068012E0AD0806925EA00000004000C54
:1043D00006D00020B842C9D00020EBE74069F3E7DF
:1043E0000120F7E72DE9F047984616460D460446AA
:1043F0004FF000094FF0200AC1F3074723E020687F
:104400004069C043400515D42068016841F400713B
:10441000016021686FF480604861C4F8309084F8CE
:104420003DA084F83E90216C41F00401216484F8A1
:104430003C9021E0701C06D0FDF760FEA0EB080068
:10444000B04203D816B1012F1FD021E02068012F00
:1044500015D0806925EA00000004000C18D000BFC8
:1044600044F8309F84F80DA084F80E90216941F043
:104470002001216184F80C900120BDE8F08740699B
:1044800025EA00000004000CEAD12068406901E040
:104490002068806925EA00000004000CAFD1ECE739
:1044A0002DE9F041002590460E460446202728E0DD
:1044B0004069C043C0060CD454F8301B6FF01000A4
:1044C000486144F810596777A577206A20622577FC
:1044D00014E0FDF713FEA0EB0800B04200D886B947
:1044E00020684069C04340060BD544F8305F6773CD
:1044F000A573206940F02000206125730120BDE8EC
:10450000F08120684169C9434906D1D40020F6E70B
:1045100070B516460D4604461EE02046FFF704FE21
:1045200008B1012070BD681C16D0FDF7E7FD801BA7
:10453000A84200D885B920684069C04300060BD561
:10454000002044F8300F20216173A073216941F0ED
:10455000200121612073E4E720684069C043000620
:10456000DBD4002070BD000008B50C4C684600F09C
:1045700087F878B101230022694620681FF07CFF8C
:1045800001F0F4F830B103F073F932201FF0D4FEDB
:1045900003F068F90A201FF0CFFEE7E720000020B3
:1045A00030B587B08C212248FBF7EFFE204C002568
:1045B0000C3C1421C4F898506846C4F89C50FBF792
:1045C000E4FE1C48016841F0010101600068694691
:1045D00000F0010005901F20CDE900050120164DD7
:1045E00002902846FDF788FC002301222946184640
:1045F00000F024F8002302222946012000F01EF8D2
:10460000002308222946022000F018F80023042283
:104610002946032000F012F8002310222946042026
:1046200000F00CF80E2020701220A06007B030BD02
:10463000EC010020303802400000024070B505282F
:104640000BD251B10D4CC0EBC00004EB800444F818
:104650000C1FA2801BB1012002E0002070BD0020D1
:10466000A0710120E0710025257265721FF071FEB6
:10467000E060257465610120A56170BDE001002046
:104680002DE9F05F04007DD01FF063FE4FF00008BD
:10469000DFF84891054646464FF0010BC6EBC601D0
:1046A00009EB8107F87C0C37B8B1B98897F806A0F8
:1046B0003868FDF711FDBAF1000F02D0012802D0D1
:1046C00000E0B8B30020397A814201D03872FD6031
:1046D00018B10BFA06F040EA0808761CF6B2052E6F
:1046E000DCD3002049460646C9F89880C0EBC002DA
:1046F00001EB8202D37C0C326BB3D3684F88EB1A88
:10470000BB4228D3137A577A9F4224D05372002B8E
:10471000D1F89C700BFA00F30FD01F43C1F89C70C6
:104720005561956116740A78D20714D0207084F808
:1047300001B049E0FFE70120C5E79F43C1F89C7045
:104740000B78DF0702D0207002203CE09B0701D5E8
:10475000137CDBB11674401CC0B20528C6D3002000
:10476000C0EBC00201EB8202D37C0C327BB3537AE4
:104770006BB38E680BFA00F35F461E4228D0536974
:10478000EB1A00E028E0167C2EB111E02070032027
:104790006070167418E08E889E4219D817740B78D2
:1047A00013F00C0F04D020700420607095610BE0B2
:1047B0000B781B070CD59369CE88EB1AB34207D34D
:1047C00095612070052060700120BDE8F09FFFE733
:1047D000401CC0B20528C3D30020F6E7E00100204A
:1047E0002DE9F04104461D4616460F462A2000F0EA
:1047F000E3F9204600F0D0F9304600F0CDF92B2047
:1048000000F0DAF9384600F0C7F9284600F0C4F99C
:10481000BDE8F0412C2000F0CFB900000249002093
:104820000968C86370470000B80500202DE9F04111
:10483000141A5D1A641C6D1C6C43154D069E2F786E
:10484000144D3B4439442D789BB22A44284492B2FB
:1048500089B280B2FFF7C4FF0F4D4FF40060E860EB
:104860002868016841F400610160A2B2314628461F
:10487000FEF746FD0948006841680029FCD1002088
:10488000E8602868016821F400610160BDE8F081FA
:10489000DE010020DD010020000500205805002079
:1048A0002DE9F047804612480C461F46017816460F
:1048B0005818401E83B20F48214489B20078DDF8B1
:1048C00020900244521E404492B280B2FFF788FF0B
:1048D0000AE0454604E0484600F05EF96D1CADB2C2
:1048E000B542F8D3641CA4B2BC42F2D3BDE8F08751
:1048F000DE010020DD010020F0B587B014216846FC
:10490000FBF743FD1848016841F0020101600168AE
:1049100001F002010591016841F0020101600068A7
:104920004FF4805600F00200059001240F4FCDE9AE
:1049300000640325694603953846FDF7DDFA012238
:1049400031463846FDF7D5FB2E02CDE90064084C10
:10495000694603952046FDF7CFFA012231462046ED
:10496000FDF7C7FB07B0F0BD30380240000402403D
:104970000000024070B5FFF7BFFF00224FF48071C6
:104980006748FDF7B6FB674D4FF48054002221467F
:104990002846FDF7AEFB6420FDF79CFA0122214674
:1049A0002846FDF7A6FB6420FDF794FA112000F0DD
:1049B00003F97820FDF78EFA362000F0FDF85A480A
:1049C000007800F0B3F83A2000F0F6F8052000F087
:1049D00009F9B22000F0F0F80C2000F003F90C20E7
:1049E00000F000F9002000F0FDF8332000F0FAF8A4
:1049F000332000F0F7F8B72000F0DEF8352000F0A3
:104A0000F1F8BB2000F0D8F8192000F0EBF8C02036
:104A100000F0D2F82C2000F0E5F8C22000F0CCF82D
:104A2000012000F0DFF8C32000F0C6F8122000F0EB
:104A3000D9F8C42000F0C0F8202000F0D3F8C62038
:104A400000F0BAF80F2000F0CDF8D02000F0B4F854
:104A5000A42000F0C7F8A12000F0C4F8E02000F086
:104A6000ABF8D02000F0BEF8042000F0BBF80D2019
:104A700000F0B8F8112000F0B5F8132000F0B2F8FB
:104A80002B2000F0AFF83F2000F0ACF8542000F0ED
:104A9000A9F84C2000F0A6F8182000F0A3F80D208B
:104AA00000F0A0F80B2000F09DF81F2000F09AF80D
:104AB000232000F097F8E12000F07EF8D02000F0ED
:104AC00091F8042000F08EF80C2000F08BF81120F3
:104AD00000F088F8132000F085F82C2000F082F810
:104AE0003F2000F07FF8442000F07CF8512000F0D7
:104AF00079F82F2000F076F81F2000F073F81F20BF
:104B000000F070F8202000F06DF8232000F06AF823
:104B1000212000F051F8BDE87040292000F04CB889
:104B20000000024000040240DC01002010B50446F1
:104B3000362000F041F80F4900223CB15A2C0DD02C
:104B40005023B42C06D0B4F5877F0BD04A701046A2
:104B50008A700AE04A708B70C02006E04A708A7042
:104B6000702002E04B708A70A020BDE8104000F079
:104B700039B80000DC010020411F5F2909D84FF43B
:104B8000967110FB01F06421B0FBF1F00149096856
:104B9000C8637047B805002008B5010A8DF80010F9
:104BA0008DF801000123022269460248FEF7F4FA5B
:104BB00008BD00000005002070B5094D06464FF401
:104BC0000074002221462846FDF793FA304600F093
:104BD00009F821462846BDE870400122FDF789BA50
:104BE0000000024001B501231A4669460148FEF75C
:104BF000D3FA08BD0005002008B5084C01230022A7
:104C0000694660691FF0DAFB10B9684616F0CAF908
:104C10001EF04EFC01201FF08FFBEFE70C00002080
:104C20007FB500212F480091019102912C4A0391F8
:104C3000026001254FF480320561C0E9012101764F
:104C400080F820101203C26205244FF0C062C461D4
:104C50008262C16080F830504561FCF754FE08B1B3
:104C6000FCF72EF9CDE90045022569461D4802955D
:104C7000FCF794FD08B1FCF723F90620CDE9000507
:104C800069461848FCF78AFD08B1FCF719F90720B6
:104C900000900320019069461248FCF77FFD08B19F
:104CA000FCF70EF9082000900420019069460D4899
:104CB000FCF774FD08B1FCF703F90920CDE9000405
:104CC00069460848FCF76AFD08B1FCF7F9F80548A1
:104CD00048300068016841F0100101607FBD0000AC
:104CE00000200140E4030020194808B5016841F4A0
:104CF00000110160016801F400110091016841F4A4
:104D0000800101600068002200F48000009005210D
:104D10000F20FDF71DFD0F20FDF70CFD00220521E2
:104D20003820FDF715FD3820FDF704FD0022052190
:104D30003920FDF70DFD3920FDF7FCFC002205218F
:104D40004520FDF705FDBDE808404520FDF7F2BC14
:104D50003038024010B501F089F9044A00210448B6
:104D60001FF0BEFB0349086010BD00009CE502086F
:104D700025570008000000202DE9F04186B01421DD
:104D80006846FBF702FB23480024016841F0040158
:104D90000160016801F004010591016841F0010121
:104DA0000160016801F001010591016841F0020113
:104DB00001600068184F00F002004FF400550590A4
:104DC000002229463846FDF794F9DFF85080EE10AE
:104DD000002231464046FDF78CF900950125CDE9CA
:104DE0000154694638460394FDF786F80096CDE9EC
:104DF0000154694640460394FDF77EF81020CDE942
:104E00000004694640460294FDF776F806B0BDE816
:104E1000F0810000303802400008024000040240E7
:104E20000D4810B50B4901600C49416000214FF459
:104E300080428160C0E9031241618161C161016208
:104E4000FDF762F9002803D0BDE81040FCF738B840
:104E500010BD0000005400408C040020A08601001A
:104E60000B4810B50949016000217F22C0E90112F9
:104E7000FF22C0E9032141618161FEF753F8002858
:104E800003D0BDE81040FCF71BB810BD002800405F
:104E9000E0040020104810B50E4901604FF4827103
:104EA0004160002102228160C0E9031201224261B7
:104EB0005202C0E906210162416281620A21C16297
:104EC000FEF7B9F8002803D0BDE81040FBF7F8BFA3
:104ED00010BD0000003800400005002010B592B061
:104EE00000240F941C2108A81094FBF74EFA2021EF
:104EF0006846FBF74AFA20481E4901606321C0E971
:104F000001144FF49671C0E9031444618461FEF703
:104F1000B4FC08B1FBF7D4FF0F940FA91648109406
:104F2000FEF782FA08B1FBF7CBFF6020CDE9080459
:104F30000A940B940C940D94082208A90E480E9420
:104F4000FEF735FC08B1FBF7BBFF00944FF40050AF
:104F5000CDE90440029401940394694606480794FD
:104F6000FEF738FA08B1FBF7ABFF0348FEF7DCFBAE
:104F700012B010BD00000140B805002010B588B087
:104F800014216846FBF701FA0024154805944FF0F8
:104F90008041069401600921C0E9011440F2E73123
:104FA000C0E9031480218161FEF77CFA08B1FBF7A8
:104FB00087FF009469460A480194FEF753FD08B143
:104FC000FBF77EFF2020CDE9050405A90448FEF784
:104FD0002BFA002801D0FBF773FF08B010BD0000CA
:104FE0000006002010B58AB0002407941C216846F2
:104FF0000894FBF7CAF91748154901606321C0E915
:1050000001144FF4FA71C0E903148461FEF735FC12
:1050100008B1FBF755FF079407A90E480894FEF75F
:1050200003FA08B1FBF74CFF60200090FA20CDE9AD
:1050300001040C22694607480494FEF7B8FB08B146
:10504000FBF73EFF0348FEF76FFB0AB010BD000000
:1050500000080040480600200C4810B50A490160CD
:105060000B494160002181600C22C160C0E904123B
:105070008161C161FEF794FE002803D0BDE81040B5
:10508000FBF71EBF10BD000000140140AC0600205D
:1050900060E31600FEE70000134C00264FF4FA759B
:1050A0002078012805D1267010A11348FBF77FF95D
:1050B00018B128461FF040F9F2E710A001F01CF8E3
:1050C0000120FBF7DFFE6420FCF704FFBFF34F8FE6
:1050D0000E4801680E4A01F4E06111430160BFF31C
:1050E0004F8F00BFFDE7000008000020757064616D
:1050F00074650D0A00000000900600207374617250
:1051000074207570646174650D0A00000CED00E098
:105110000400FA0508B50A4800231A4669460068E3
:105120001FF04CF920B99DF8000018B1012803D0F8
:10513000002008BD012008BD4FF0FF3008BD000071
:1051400028000020FEE700002DED028B002384B034
:105150001A46012155481FF011FA554D554FDFF8F9
:1051600058914FF480680026686000231A4601A910
:1051700038681FF023F9002876D1287800289DF898
:10518000040004D0012827D002282CD06EE000288B
:1051900028D1012241464846FCF7ABFF474800F0C2
:1051A0001FF90021454800F053F900231422FA2189
:1051B000424800F031F922F03FFD68681FF0D5F950
:1051C00010B168681FF02FFA4FF47A7168681FF009
:1051D00011FA0120287049E0002241464846FCF7B8
:1051E00088FF2E705DE0DDED020AF5EEC00AF1EEFB
:1051F00010FA3BDD9DED030AB5EEC00AF1EE10FAA0
:1052000034DD10EE900A2E4988422FDC10EE100A91
:105210002C4988422ADCF3EE040A20EE200A10EE24
:10522000100AFBF780FA9FED288B53EC182BFBF745
:10523000CCF8FBF75FFA9DED020ADFED250AC4B258
:1052400020EE200A10EE100AFBF76DFA53EC182B33
:10525000FBF7BBF8FBF74EFA81B200232246174852
:1052600000F0DAF822F0E8FC2878D0B107F022FF4D
:1052700020B910214846FCF72FFF90B98DF8006047
:10528000002403E0641CE4B2032C05D269461148F3
:10529000FBF718FE0028F5D19DF8000008B108F0D2
:1052A000ABFF01201FF048F85FE700001173000812
:1052B0002C0000202400002000040240B808002038
:1052C0000000A0410000A0407B14AE47E17A843F7B
:1052D000000048426408002010B50C460022072157
:1052E00007F050FF208010BD21F0F1B8D8B390F83E
:1052F00030308B4238D9B2B300EB81004FF000015F
:105300004069830F137006D0012B08D0022B11D0F7
:10531000032B19D11AE05180C0F389230FE0C0F3A9
:1053200089235380C0F309539380D180C0F30900CF
:10533000108109E0C0F389235380C0F3095393809F
:10534000C0F30900D080118101207047C0F34743AA
:105350005B009380C0F307235B0000F07F00538065
:1053600000EB8000EEE7FFE700207047F8B5054648
:105370001E4617460C4668461FF095F9EC80E00B78
:1053800008D09DF80000102800D9102000EB400044
:10539000114913E09DF8030000289DF8000007D094
:1053A000102800D910200C4900EB4000CC3905E052
:1053B000172800D91720094900EB400001EB8000B5
:1053C0002860D0F804C0BCF1000F04D033463A4640
:1053D00021462846E047F8BDFCD8050810D7050847
:1053E00010B504463421FAF7D0FF0148206010BD03
:1053F00010D70508024901600021017270470000C2
:1054000010D7050830B1036823B19B6813B109B107
:1054100002B11847002070472DE9F0410446408949
:105420000E461F461546B04202D1207BA8420DD041
:10543000204607F01BF97F1E50EA070106D066815F
:10544000257384F831000120BDE8F0810020FBE7DE
:1054500010B54174002141810446017390F8300079
:10546000002806D00A46204607F000F984F83100EB
:10547000012010BD010901EB810100F00F0000EBDC
:105480004100C0B2704700002DE9F04104460068B9
:105490000025C168490618D4C16841F08001C16087
:1054A000FCF72CFE06464FF47A78042707E000BF8D
:1054B000FCF724FE801B404501D967770125206851
:1054C000C068400601D4002DF2D02846BDE8F08126
:1054D00070B5044600680025C16821F08001C160F4
:1054E00020688068800606D42046FDF787FD10B14D
:1054F000042060770125284670BD10B5806B0168D7
:105500004A6822F003024A60416D41F01001416592
:10551000012180F85110FDF78DFD10BD10B5806B95
:10552000FDF755FF10BD38B50546846BFCF7E6FD69
:10553000024628680068C00523D42068416821F02D
:10554000200141602068416821F00201416064212E
:10555000204600F01BF818B1606D40F02000606537
:10556000A068002118B92068C26880680090E186B0
:10557000012084F85100606D18B12046FDF75AFDF6
:1055800038BD2046FDF722FF38BD0000F8B51546AE
:105590000E460B46009204460122022100F02CF830
:1055A000A0B9134813490068B0FBF1F04FF47A71C9
:1055B000484300906068B0F5827F0DD133460022E9
:1055C00080212046009500F017F870B1606D40F022
:1055D000200060650320F8BD009830B1401E0090A7
:1055E00020688068C0430006F6D50020F8BD0000A2
:1055F0009402002000366E012DE9F8431E469146C4
:1056000088460446089DFCF779FD401B351AFCF7D7
:1056100075FD074625480068C0F3CB30684338E085
:10562000701C37D0FCF76AFDC01BA84203D215B12D
:10563000009860B32CE02068416821F0E0014160EF
:105640006068B0F5827F0BD1A068B0F5004F02D042
:10565000B0F5806F04D12068016821F0400101603D
:10566000A06AB0F5005F09D12068016821F40051FB
:1056700001602068016841F400510160012084F854
:105680005100002084F850000320BDE8F883002575
:10569000401E00902068816838EA010004D0002193
:1056A0004945BDD10020F0E70121F9E7940200202F
:1056B00000B587B014216846FAF767FE002002465D
:1056C000059069461548FDF703FC002205A913481B
:1056D000FDF7DCFB9DF8170040F26D1110FB01F0A7
:1056E0009DF81510C1EB411108449DF816100844AF
:1056F0009DF8001000EB400001EBC0004FF4616129
:1057000048439DF80110C1EB011100EB81009DF8A9
:10571000021008440249086007B000BDE004002000
:1057200004000020064D4FF400544FF4FA76214651
:105730002846FCF7D6FC30461EF0FEFDF7E70000D9
:105740000008024010B54FF0E020006928F0E0FCAE
:10575000012803D0BDE8104028F0A0B910BD00001A
:1057600001480078704700008C0200200148407812
:10577000704700008C0200200148808870470000BC
:105780008C020020642803D802490870FFF7F4B99E
:10579000704700008C020020024900B101204870CF
:1057A000704700008C02002030B15A2804D0B42881
:1057B00002D0B0F5877F03D102498880FFF7B6B9E0
:1057C000704700008C02002030B593B0302168464D
:1057D000FAF7DBFD14210CA8FAF7D7FD1D480024C9
:1057E000016841F080510160006800F08050119024
:1057F0001948016841F4404101600068102100F43B
:10580000404011900A2000900120CDE903010225BB
:10581000CDE905050820CDE907406420CDE909055B
:1058200004200B906846FDF77BF908B172B6FEE7DD
:105830000F20CDE90C054FF48050CDE90E40032137
:105840000CA81094FDF760F8002801D072B6FEE7AE
:1058500013B030BD4038024000700040024801687B
:1058600041F470010160704788ED00E010B5044814
:10587000FDF7C1FEBDE810400248FDF7BCBE0000C8
:10588000B8050020B4070020F0B50268204B214C79
:105890009F03214D214E984207D0B84205D0A04227
:1058A00003D0A84201D0B04204D122F0700C4A6863
:1058B00042EA0C02984210D0B8420ED0A0420CD05E
:1058C000A8420AD0B04208D0154CA04205D0154CD1
:1058D000A04202D0144CA04203D122F44074CA6802
:1058E00022434C6922F08002224302608A68C2622D
:1058F0000A688262984201D109690163012141610C
:105900000169C90703D0016921F001010161F0BDFE
:10591000000001400004004000080040000C00406E
:1059200000400140004401400048014010B501F032
:105930001F030121046A99408C430462016A9A4062
:105940001143016210BD10B5846842EA032224F4B9
:105950007F440A432243826010BD000030B5036AD1
:10596000026A22F0010202624268846924F073052F
:105970000C682C4323F002058B682B430A4DA84288
:105980000BD123F00805CB6822F440722B434D69FC
:1059900023F0040315438A692A43426084614968FD
:1059A0004163036230BD00000000014030B5026A6F
:1059B000036A23F010030362436884690D6824F4CA
:1059C000E64444EA05248D6822F0200242EA0512EA
:1059D0000B4DA8420ED1CD6822F0800242EA05129A
:1059E0004D6923F4406343EA85038D6922F0400248
:1059F00043EA85034360846149688163026230BD84
:105A00000000014030B5036A026A22F4807202622B
:105A10004268C46923F4007324F073050C682C43B6
:105A20008D6843EA05230C4DA8420ED1CD6823F4BE
:105A3000006343EA05234D6922F4405242EA05120D
:105A40008D6923F4806342EA05124260C4614968AB
:105A5000C163036230BD00000000014030B5046A3C
:105A6000026A22F4805202624268C3690D6823F41C
:105A7000E64343EA05238D6824F4005444EA0534E0
:105A8000064DA84204D14D6922F4804242EA8512B3
:105A90004260C36149680164046230BD0000014096
:105AA00070B5036800249A6822F070054A682A439A
:105AB00022F007050A682A439A604A6812F00F0F1D
:105AC00031D11211082A2ED2DFE802F02E2E2E2E0E
:105AD0000B2127040B69D1E902210068FFF733FF8E
:105AE00022E00A68052A10D00268136A156A25F0B8
:105AF0000105156202689569096925F0F00545EA16
:105B000001119161006803620EE0012070BD0A6915
:105B10008968006800F00AF806E00A698968006888
:105B200000F015F800E00124204670BD10B5036AAE
:105B3000046A24F001040462846924F0F00444EA55
:105B4000021423F00A020A438461026210BD10B5F8
:105B5000036A046A24F010040462846923F0A00339
:105B600024F4704444EA023243EA01118261016282
:105B700010BD01201DF0D6BB10B51FF0B1FA0028F2
:105B800005D0D0E90021BDE810400846104710BDFF
:105B90000A46014601230148FEF7B6B9AC060020CB
:105BA00010B5806B0021C185C184FDF7C0FF10BD19
:105BB00070B5846B2068406994F84110C0F3C01040
:105BC0000025212904D118B1E584204600F0B4F85D
:105BD0002068406994F84210C0F38010222904D153
:105BE00018B1E585204600F080F8606C40F01000A8
:105BF00060642046FDF79BFF70BD10B50146806BC9
:105C0000096809684FF00002C9052ED4C2850168F1
:105C10000C3151E8003F23F4807341E80034002C3C
:105C2000F5D10168143151E8003F23F0010341E848
:105C30000034002CF5D10168143151E8003F23F005
:105C4000400341E80034002CF5D1202180F84210B7
:105C5000016B012909D101680C3151E8003F23F0A3
:105C6000100341E80034002CF5D14263016B012997
:105C700002D0FEF747F910BD818DFDF71FFF10BD63
:105C800010B5806B01214163016B012902D0FEF741
:105C90003AF910BD818D4908FDF710FF10BD10B510
:105CA0000146806B09680968C90516D40021C184C2
:105CB0000168143151E8002F22F0800241E80023EE
:105CC000002BF5D101680C3151E8002F42F0400261
:105CD00041E80023002BF5D110BDFEF7A1F910BD5E
:105CE00010B5806BFEF79DF910BD01680C3151E8CD
:105CF000002F22F4907241E80023002BF5D10168B7
:105D0000143151E8002F22F0010241E80023002B5A
:105D1000F5D1016B012909D101680C3151E8002F3F
:105D200022F0100241E80023002BF5D1202180F859
:105D3000421000210163704701680C3151E8002FC7
:105D400022F0C00241E80023002BF5D1202180F889
:105D50004110704708B590F84210222901D0022066
:105D600008BD82684FF480539A4201D1016921B184
:105D7000816A9A421BD04AB10AE00268816A52687D
:105D8000C2F308020A80816A891C08E0026972B1C4
:105D90000268526802F07F020A70816A491C8162BF
:105DA000C18D491E0904090CC18503D01BE002689E
:105DB0005268F1E70168CA6822F02002CA600168EF
:105DC000CA6822F48072CA6001684A6922F001023E
:105DD0004A61202180F8421000214163026B012AB0
:105DE00003D0FEF78FF8002008BD016301680C3175
:105DF00051E8002F22F0100241E80023002BF5D1DA
:105E000001680A68D20602D50A6849680091818D46
:105E1000FDF754FEE7E7000070B50446006801692D
:105E2000E26821F44051114301612169A068E269EF
:105E300008436169114308432168CA6849F20C6349
:105E40009A430243CA6020684169A26921F4407103
:105E50001143416131492068884202D0304988426B
:105E600002D1FCF71BFE01E0FCF708FEE26900230B
:105E7000192164253226B2F5004F626828D0A0FBB4
:105E80000101930F9200FAF705FA0146B0FBF5F015
:105E90006FF01802504301EB800006EB0010B0FBDE
:105EA000F5F000F0F002B1FBF5F002EB0012B1FBEF
:105EB000F5F06FF01803584301EB800006EB00107B
:105EC000B0FBF5F000F00F0021681044886070BD51
:105ED000A0FB010192185B41FAF7DCF90146B0FB27
:105EE000F5F00201B1FBF5F06FF01803584301EB38
:105EF000800006EBC000B0FBF5F000F0F80002EB0C
:105F00004002B1FBF5F0584301EB800006EBC00006
:105F1000B0FBF5F000F00700D6E7000000100140EC
:105F20000014014038B58162044682850020134682
:105F30006064222284F84220E56B1B4AEA63E56B29
:105F40001A4A2A64E56B1A4AEA64E26B10650A464B
:105F50002168E06B091DFBF785FF20680168406838
:105F60000090206948B120680C3050E8001F41F4CF
:105F7000807140E80012002AF5D12068143050E802
:105F8000001F41F0010140E80012002AF5D120680D
:105F9000143050E8001F41F0400140E80012002A90
:105FA000F5D1002038BD0000FB5B0008815C0008D3
:105FB000B15B00082DE9F843984617460D460446A4
:105FC000089E24E0701C22D0FCF798F8A0EB080093
:105FD000B0421AD8CEB12068C168490717D5802DC4
:105FE00015D0402D13D00168C94309070FD40168AB
:105FF0000025406800902046FFF777FE0820606487
:1060000084F840500120BDE8F8830320FBE72068B6
:10601000006835EA000004D00020B842D2D0002049
:10602000F1E70120F9E700000C4810B500680168AD
:10603000C943C9060DD40A4A012111706FF010013D
:1060400001600648FDF73BFD192206490348FDF7AC
:106050004BFFBDE810400148FDF76ABDAC060020CB
:106060000800002090060020FEE7000010B5002286
:10607000022104201EF0D4F9184C00220C2160618A
:1060800004201EF0CDF9A0610022012104201EF0A1
:10609000C7F9E061124A002112481EF021FA104AA5
:1060A00020606C32002110481EF01AFA0C4AE060A1
:1060B000483200210D481EF013FA094AA06024322C
:1060C00000210B481EF00CFA054A60609032002156
:1060D00008481EF005FA206110BD00000C000020E9
:1060E000C0E5020829400008495100086945000838
:1060F00099500008F94B00080FB4054B10B503A9DF
:10610000044A029800F030FC10BC5DF814FB00005B
:1061100061CF0008C40300200FB47CB50C0009ADAA
:1061200001D0611E00E00021CDE90001064B6A4666
:106130002946089800F018FC002C02D0009A002193
:1061400011707CBC5DF814FB857100080FB4084B1E
:1061500010B504A902AA039800F006FC044602A99F
:10616000002001F01AF8204610BC5DF814FB000076
:106170009B7100080907090E002804DB00F1E020EC
:1061800080F80014704700F00F0000F1E02080F864
:10619000141D704710EE100AC0F3C7517F3917293C
:1061A000A8BF7047DFED140A002970EE200A0DDA4F
:1061B000F5EEC00AF1EE10FA1ADD0028A8BF0020A3
:1061C00016DAB0F1004F18BF0C4811E00C4ACA4073
:1061D000104208BF7047F5EEC00AF1EE10FA07DD75
:1061E000002804DA4FF4000323FA01F10844904335
:1061F00000EE100A70470000CAF24971000080BF2B
:10620000FFFF7F0010EE100A10B5A0F500014FF05F
:10621000000CB1F1FE4F6CD200F500216FF07E0250
:1062200002EBE153C1F302524FF07E5101EB0251F8
:1062300000EE901AA0EBC3500CEB030100EE100A25
:1062400051EA020036D030EE601A30EE200AC1EE7C
:10625000000A20EEA00A60EE801A9FED3D2A9FED15
:106260003D1A3D48DFED3F2A00EE021A784400EB6C
:1062700082009FED3A2A21EE810A01EE101AD0ED3C
:10628000001A3748B8EEC11A784400EB820041EE9C
:10629000021A01EE101A90ED002AB8EEC11A01EEB2
:1062A000222A9FED311A32EE000A00EE810A31EE09
:1062B000800A10BDF7EE000A9FED2D1A70EE600AFD
:1062C0009FED2A0A00EE801A9FED2A0A60EEA01ABE
:1062D00000EE810A9FED281A00EE801A21EE810A55
:1062E0009FED261A00EE810AB5EE0B1A00EE810A28
:1062F00010BD4FF07F41B1EB400F03D2BDE810401D
:1063000000F098B8B0F1FF4F08BF10BDB5EEC00A5D
:10631000F1EE10FA06D2012000F0A8F8BDE8104016
:1063200000F08CB8B5EEC00AF1EE10FA07D10220E9
:1063300000F09CF800F074F8B1EE400A10BDDFEDFB
:10634000100A6FF0160C20EE200A10EE100A63E718
:10635000DE02323E3B3D943EBC88050000209A3E62
:10636000C0880500FC849A36D95B5E3F924FA93DF8
:106370007279DEBD2D3E143ED85B5EBE157B4B3C74
:106380000000004B10B52DED028BB0EE408A18EEE8
:10639000100AFAF775FA01EE100A18EE100AB7EEB5
:1063A000000A78EE410A10F0004F4FF07F4010EEE7
:1063B000901A12D0B1F13F4F24BF10EE901AB0EBFB
:1063C000410F12D210EE901AB1F17C5F1CDD10EE7D
:1063D000901AB0EB410F17D314E0B1F13F4F07D93A
:1063E00010EE901AB0EB410F02D331EE401A0BE0E1
:1063F00010EE901AB1F17C5F06DB10EE901AB0EB54
:10640000410F01D331EE001A18EE100ABDEC028BD9
:1064100011EE101A61F31E0000EE100A10BD00000C
:10642000DFED030AB7EE001A81EE200A7047000084
:106430000000000030EE000A70470000DFED020AA5
:1064400080EEA00A704700000000000002E008C8CB
:10645000121F08C1002AFAD170477047002001E0DE
:1064600001C1121F002AFBD17047000001490860DA
:1064700070470000D003002070B5044600256FF07F
:106480002F0608E02068411C2160007805EB85019B
:1064900006EB410145182068007800F043F9002818
:1064A000F0D1284670BD70B514460D461BB9114693
:1064B0000DF03CFD034603FB05F0142C0ED0E11F4C
:1064C00003290AD8072C0DD0082C0DD0092C0DD08B
:1064D0000A2C0DD0002100EB810070BD590801FB92
:1064E000050070BD0221F6E70421F4E71021F2E770
:1064F0004FF48071EFE710B504461CF0D7FF08B1E8
:1065000015F0BEFF2046BDE810401CF079BF10B565
:106510002DED028B26F01CF8B0EE408A26F030F804
:10652000F0EE480ABDEC028BBDE8104021F098BBAC
:106530007CB526F00DF810EE104A26F021F810EE8A
:10654000100AFAF7F0F841EC100B10A153EC102BE5
:106550006846FFF7FBFD0F4D6946E86814F08AFABC
:106560002046FAF7E0F89FED0C1B53EC112BFAF7DD
:1065700045F841EC100B05A153EC102B6846FFF7D2
:10658000E5FD6946A86914F075FA7CBD252E3266D2
:1065900000000000280100200000000080842E413F
:1065A0002DE9FF5F82B00021DDE90430020DDDF846
:1065B00040B0034318D044F61050A2F2FF324243D9
:1065C0001514119801281FD0A5EB0B00401C5FEAA1
:1065D000000A4FF000064E4FDFF83891B0465046A3
:1065E00015D5CAF1000413E0119801244AA301282B
:1065F00001D16FEA0B010298119AC0E90031C0E99C
:10660000024206B0BDE8F09FCBF10000DFE7044690
:106610000021404A491842EB0450CDE9001012E035
:10662000E00707D032463B4640464946F9F774FF3B
:106630008046894632463B4610461946F9F76CFFBC
:1066400006460F466410002CEAD1DDE90401DDE9BD
:106650000023BAF1000F06DAF9F75EFF42464B4617
:10666000F9F75AFF05E0F9F7C9FF42464B46F9F73B
:10667000C5FF04460E460022284BFAF795F903D8C9
:106680004FF0FF30014607E00022254B20463146FF
:10669000F9F79BFEFAF76FF9102409E0002C0ADBEA
:1066A0000A220023F9F7F6FD039B30321A55641EC7
:1066B00050EA0102F2D1641C039AC4F1110314449C
:1066C000119A012A03D0012208430DD10AE00843A0
:1066D00004D000204FF0110B119072E7A3EB0B05D3
:1066E0006D1E0DE05B4504DD4FF0000205F1010574
:1066F00004E003DA4FF00002A5F10105002AECD016
:1067000002981199C0E90231C0E9004579E700001B
:10671000000014400000F03F300000000000F04393
:106720000000E03F3038092801D8012070470020E0
:1067300070472DE9FC5F9B460CAB8A468146DDE93C
:10674000116093E81210DDE90F575FEA80784FF08F
:1067500030031AD45EB15FEAC07808D000F00C08AC
:1067600058EA0C0803D0761E01E00B55641CBC42AD
:1067700004D2202CF9D301E00B55641C5FEAC078E9
:1067800003D0B44201D2202CF6D35FEAC06825D5ED
:106790005FEA40580AD44CB1BC4201D0B44205D1A2
:1067A000641E03D0102D03D1641E04E0102D02D00E
:1067B000022D0AD00EE0850603D4202C1ED27825A7
:1067C00006E0202C1AD2582502E0202C16D2622591
:1067D0000D55641C202C11D20B55641C202C0DD29D
:1067E000BCF1000F01D02D2306E0430701D52B2378
:1067F00002E0030702D520230B55641CCDE900BA43
:10680000C846154681468B46AA46800714D12746BE
:1068100007E02A46DDE900316D1C2020C446E04730
:106820007F1CB742F5D307E02A466D1C641EDDE9E4
:1068300000311BF80400C047002CF5D15FEA8970D5
:1068400006D409E02A46DDE900316D1C2020C0474E
:10685000A5EB0A00B042F5D32846BDE8FC9F2DE920
:10686000F04F8FB099468B46DDE91818DDE91C63BF
:10687000DDE91A4792468646002209B923F0100343
:10688000580507AD00D5C9B1B1FBF4F004FB1010F9
:10689000C0B20A2801D2303009E05FEA836C02D529
:1068A0004FF0410C01E04FF0610C60440A38B1FB3D
:1068B000F4F1A854521C09B1202AE5D3CDF8088080
:1068C000CDE90563CDE90052CDE903474B46524679
:1068D00059467046FFF72DFF0FB0BDE8F08F2DE948
:1068E000FF4F8FB01CACDDE9239594E8030820AC82
:1068F00094E8C004002450EA010201D125F01005FB
:106900006A050DF11C0802D550EA010217D0324683
:106910003B46F9F7BFFCD2B20A2A01D2303206E078
:10692000AB0601D5412300E061231A440A3A08F876
:106930000420641C50EA010201D0202CE7D3CDE9E9
:106940000084CDF808B0CDE90595CDE9036A0FAF15
:1069500097E80F00FFF7EDFE13B0BDE8F08F9A4205
:1069600000D28854704770472DE9FF4F95B09A4682
:10697000884606460025EEE1252877D100242746E3
:10698000F94A0121039400E0044316F8013F203B3B
:1069900001FA03F01042F7D130782A2811D06FF0B5
:1069A0002F033078A0F13002092A16D8039A44F058
:1069B000020402EB820203EB42021044761C0390B5
:1069C000EFE758F8042B0392002A03DA504244F40C
:1069D0000054039044F00204761C30782E2816D11F
:1069E00016F8010F44F004042A280DD06FF02F028E
:1069F0003078A0F13003092B09D807EB870302EBAD
:106A00004303C718761CF3E758F8047B761C3078EC
:106A10006C280FD006DC4C2817D068280DD06A28C7
:106A200014D104E0742810D07A280FD10DE044F47A
:106A300000140AE044F4801401E044F44014727835
:106A4000824202D104F58014761C761C30786628C8
:106A50000BD013DC582877D009DC002875D04528E6
:106A6000F6D04628F4D047281AD193E118E06328DD
:106A700035D0642879D0652812D18BE1702873D085
:106A800008DC6728F1D069286FD06E280DD06F28F8
:106A900006D1ACE073282CD0752874D0782853D058
:106AA0005246179990476D1C54E1C4F302500228D6
:106AB00009D003280DD0D8F8001004280DD00D609F
:106AC00008F1040846E1D8F80010EA17C1E90052BD
:106AD000F6E7D8F800100D80F2E70D70F0E718F82F
:106AE000041B8DF8001000208DF80100EB460120FA
:106AF00003E058F804BB4FF0FF3061074FF000018E
:106B000002D40DE009F101018946B9420FDA81454D
:106B1000F8DB1BF809100029F4D108E009F10101A4
:106B200089468142FADB1BF809100029F6D1039847
:106B30005346A0EB090721463846179A00F080FA21
:106B4000284400EB090507E044E008E10DE01BF8EC
:106B5000010B524617999047B9F10109F7D25346F4
:106B600021463846179AF2E039E00A21C4F302526E
:106B70004FF0000B0091022A06D058F8040BC11701
:106B8000032A09D00AE023E008F1070020F00702F9
:106B9000F2E80201904605E000B2C117042A01D1D3
:106BA00040B2C117002906DA0A460021404261EBD3
:106BB00002012D2202E0220504D52B228DF80420AB
:106BC000012203E0E20701D02022F7E7914657E0D7
:106BD0000A2100E010214FF0000B00910BE0102182
:106BE0004FF0000B44F004040827009103E0082054
:106BF0004FF0000B0090C4F30252022A05D058F85F
:106C0000040B0021032A08D008E008F1070020F057
:106C10000702F2E80201904603E080B2042A00D1A4
:106C2000C0B24FF0000922072AD53278702A07D067
:106C3000DDF800C08CF0100C5CEA0B0C05D00EE007
:106C400040228DF80420012208E050EA010306D01A
:106C500030238DF804308DF8052002229146009BE8
:106C600083F0080353EA0B030AD150EA010201D171
:106C7000620705D530228DF804204FF001097F1EF0
:106C80003278582A04D039A20C920CAA02920BE056
:106C90003BA2F9E75B46009AF9F7FCFA0C9B9B5C78
:106CA000029A521E0292137050EA0102F2D1029827
:106CB00004A9081A00F1200B600702D524F48034DF
:106CC00000E001275F4502DDA7EB0B0000E000209C
:106CD00000EB0B01009003984944401A0390E00335
:106CE00006D453462146179A039800F0A9F90544A3
:106CF000002706E001A85246C05D179990476D1C19
:106D00007F1C4F45F6DBE0030CD553462146179A0E
:106D1000039800F095F9054404E030205246179995
:106D200090476D1C0099481E00900029F5DC08E092
:106D30000298029952460078491C0291179990478F
:106D40006D1CBBF10001ABF1010BF1DC5BE100F06C
:106D500065F90544761C307800287FF40DAE19B033
:106D60002846BDE8F08F0000092801003031323399
:106D70003435363738396162636465660000000077
:106D80003031323334353637383941424344454661
:106D900000000000600700D4062708F1070020F07B
:106DA0000700F0E80223804603F0004C5FEA0C0085
:106DB00001D097A009E0200501D596A005E0E007E5
:106DC00001D095A001E0AFF24C001390307823F091
:106DD000004365280CD006DC452809D046281DD084
:106DE00047287FD13BE0662818D067287AD136E063
:106DF0000021112F01DB112000E0781CCDE90001FA
:106E000004A90CA8FFF7CCFBDDE90D010C9A4FF0AB
:106E1000000B07F10109109200914EE04FF0004085
:106E20000097CDE9011004A90CA8FFF7B9FBDDE933
:106E30000D020C9B0F994FF0000B9146109300929E
:106E400011B9791C00EB0109B7EB090003D4C0F1BB
:106E5000FF3B07F10109A9EB0700019042E0012F78
:106E600000DA01270021112F01DD112000E0384652
:106E7000CDE9000104A90CA8FFF792FBDDE90D01A3
:106E80000C9A00914FF0000BB946109221070FD4D5
:106E9000009A4A4503DA914601E0A9F10109B9F1E6
:106EA000010F05DD109AA9F10101515C3029F4D0E0
:106EB000B84202DA10F1040F03DA0121CDE9011022
:106EC00010E0002803DC8344A9EB000102E0411C30
:106ED000494500DD8946A0EB0B00401C01904FF0B6
:106EE00000400290200705D40198484502DB4FF08E
:106EF000FF30019000208DF84B0002980DF14B07F8
:106F0000B0F1004F25D002200C902B200D9002985C
:106F100000280CDA404202902D200D9007E00A2153
:106F20000298F9F72FFC3031029007F8011D0C99F7
:106F3000481E0C900029F2DC02980028EFD1791E3F
:106F40000D980870307800F0200040F0450007F8F8
:106F5000020D11A8C01BC01D02901398007800B14B
:106F6000012000EB0901019801EBE0710298014456
:106F70000398401A401E0390E00306D4534621466E
:106F8000179A039800F05CF805441398007818B13C
:106F90005246179990476D1CE00323D5534621466E
:106FA000179A039800F04CF805441BE0BBF1000F62
:106FB00007DB0098584504DD1098179910F80B006E
:106FC00001E0179930205246904701980BF1010BD0
:106FD000401E05F10105019004D12E20524617995B
:106FE00090476D1CB9F10001A9F10109DEDC05E053
:106FF00017F8010B5246179990476D1C0299481ECD
:1070000002900029F4DC53462146179A03989EE625
:107010002D0000002B000000200000002DE9F041B1
:10702000044600251E461746880404D405E0394668
:107030002020B0476D1C641EF9D52846BDE8F081BC
:107040002DE9F041044600251E469046C80301D5AF
:10705000302700E02027880404D505E04146384663
:10706000B0476D1C641EF9D52846BDE8F0810000CC
:107070007CB5114C206AF9F756FB41EC100B0FA1BF
:1070800053EC102B6846FFF761F8A4F180056946C0
:10709000E86D13F0EFFC606AF9F745FB41EC100B6B
:1070A00008A153EC102B6846FFF750F86946686F4B
:1070B00013F0E0FC7CBD0000A8010020252E326604
:1070C00020560000252E32662041000010B525F024
:1070D0003CFA144C01460022E0681AF046F825F00C
:1070E00047FA0028A0694FF0010102D014F0A3FD77
:1070F00001E017F0CEFF25F039FA60B15A280CD024
:10710000B4280CD0B0F5877F0BD107A1606BBDE828
:10711000104013F0AFBC06A1F8E707A1F6E708A1FD
:10712000F4E710BDCC0000203C20323730203E0078
:107130003C20203020203E003C203930203E000002
:107140003C20313830203E0010B5FDF7E3FF012828
:1071500009D0401C0FD107F05BF920F099FFBDE882
:10716000104025F041BD07F053F9BDE81040002163
:1071700001A013F0DDBE10BD505053205061676573
:10718000000000004A68002A06D00A68531C0B6001
:1071900010704868401E486070470A68531C0B60B6
:1071A0001070704770B51D4C06461B4DE0690022FB
:1071B000114655F8200018F06FFBA4F1800186B14C
:1071C000E069401CE0614978012902D0022904D01D
:1071D00018E0072816DD002013E00D2812DD082036
:1071E0000FE04878012802D0022806D00AE0E069C2
:1071F00008B9072005E0401E03E0E0690828FAD13D
:107200000D20E061E0690022032155F82000BDE86F
:10721000704018F041BB00002C080020A80100209D
:10722000F0B52B4F89B0384697F801E00024406A4A
:10723000DFF8A4C02749CDE9044CCDE90614274E58
:107240006FF077034FF4FA7207F18005BEF1010F7A
:107250001DD07821CDE9001402940021039413F08D
:1072600013FE01207870E8690022114656F82000CC
:1072700018F012FBEC6100220321306818F00CFBBF
:10728000E86809B016A1BDE8F04013F0F3BBCDE902
:107290000034029478230021039413F0F5FD0220BA
:1072A0007870E8690022114656F8200018F0F4FAC8
:1072B0000820E86100220321306A18F0EDFA0EA1DF
:1072C000E86813F0D7FB09B0BDE8F040FFF7D0BE87
:1072D0002801002085AE0108B7FC00082C0800201A
:1072E0007072657373206865726520746F205661D3
:1072F000726961626C650000707265737320686505
:10730000726520746F204669786564205365740047
:10731000F8B5174C6078401C607007F07DFF154E83
:10732000002560B18DF800500123002269463068C5
:107330001DF0A2F8657060681DF075F9F8BD607801
:107340000A28FBD301208DF800000346002269467D
:1073500030681DF091F8657060681DF064F90022D6
:107360004FF480610448FAF7C4FE2570F8BD0000B0
:107370002C00002028000020000402402DE9F047E6
:1073800088B00024264E4FF0140ACDE90664254F3C
:107390004FF41675CDF800A005974FF6FF78CDE9AC
:1073A0000145DFF88490CDE9034832232A4621467F
:1073B000D9F8140013F068FDCDE90664CDF800A0FB
:1073C0000597CDE90145CDE9034832232A46C82176
:1073D000D9F8180013F058FDCDE90664CDF800A0E7
:1073E0000597CDE90145CDE9034832232A46D90066
:1073F000D9F81C0013F048FDCDE90664CDF800A0D3
:107400000597CDE90145CDE9034832232A462946AF
:10741000D9F8200013F038FD08B0BDE8F08700006F
:1074200081AE0108B7FC00087000002070B50D4661
:10743000040011D08DB100F067F800280BD061680E
:1074400000690AF0EFFD0646E16B28468847E168CF
:107450000844E060304670BDFEE7FEE72DE9FF41DD
:1074600014460E4605460A461F4621466846DDF884
:10747000288009F006FB00281AD00198616822686C
:10748000411A009808FB0151821A55183168384496
:10749000441A684609F0E3FA002107E0625C6B5C7D
:1074A0001A44FF2A00D9FF226254491C8142F5D3B5
:1074B000BDE8FF8110B502004FF000000CD04B1E5C
:1074C000194200D0FEE70A44521E9A43B2F5803FAB
:1074D00002D20C2A01D9104610BD0C2010BD084460
:1074E0004A1E401E9043114200D0FEE7704710B57F
:1074F000402013F0B1FF040005D04022002114F019
:10750000DCF8204610BDFEE72DE9FC410D460400E5
:107510002AD055B304F12400804618F09CFE009058
:1075200008B30769616838460AF07CFD06462946BB
:107530003846626814F006F804F1300013F0B1FE2A
:10754000019098B10422694613F0FCFF204600998F
:1075500006F010FA042201A913F0F4FF2146304688
:1075600062680AF06FFD07E0FEE7FEE7404600991B
:1075700018F03BFE002000900098BDE8FC81000060
:107580002DE9F0410F460121002504462E46C16336
:1075900009E01A491AF044F808B16D1C02E0E06BEA
:1075A000401CE063761C57F8260010B101780029D2
:1075B000EFD1A06BA8421FD0206B002610B111F0B4
:1075C00071F82663606B10B111F06CF866632801E6
:1075D00013F042FF206338B1680013F03DFF606391
:1075E00018B1216B11B102E0FEE7FEE700256A0049
:1075F000002114F062F8A563BDE8F081701B01085A
:1076000010B5044690F85400E26BC107616C04D1D8
:1076100021B14B1C18D0491E6164A9B90AB1C10738
:1076200012D02146144813F0E1FE00F027F821693A
:1076300009B120468847616909B12046884720463C
:10764000BDE8104011F02EB8216C49426163002A58
:1076500010D0C10702D1A16B49426163411C61F3A3
:10766000000084F85400E16A606A6162E062206BA5
:107670002263E06310BD00004053002010B50A4CA7
:10768000012084F8A40004F1AC0013F0E5FD00280B
:10769000D4F8A80003D0BDE810401BF0A3BFBDE89C
:1076A00010401BF08DBF0000945200202DE9F041E6
:1076B0003D4D95F8A50038B15FF0000085F8A500B4
:1076C0003948AC30074664E00120F7E7206D1BF035
:1076D00013FE616B084460631BF014FE20650020FC
:1076E00085F8A40094F8540095F8A510C0F3400262
:1076F0008A4254D061F3410084F8540041071ED4FB
:10770000616B002941DB000709D4A16939B120462A
:107710008847616A01446162E16A0844E062204688
:107720001EF070FEE16809B12046884794F85400C5
:1077300040F0040084F8540020461EF083FD606B86
:10774000002822DB216B884200DD6163216A20462C
:107750008847A16A0646B1420DD0A662626812B19E
:1077600031462068904795F8A40088B9A2682AB1EC
:1077700031462046904795F8A40048B9D4E90C0159
:1077800081420CDB2046FFF73BFF95F8A40030B1A7
:10779000384613F061FD040098D1BDE8F081214620
:1077A000384613F06BFDF6E79452002070B504469E
:1077B00040680D4608B1FFF7F9FF2268002A04D09F
:1077C00029462046BDE87040104770BD70B50D6871
:1077D00006460C46286838B1296AC90204D52060DB
:1077E00021463046FFF7F2FF214630462560BDE8CE
:1077F0007040FFF7DBBF08F001BF08F045BF000095
:1078000010B5416C96B0044601B3684608F004FA1E
:107810002146684608F0B4FA0F49684608F096FA1F
:107820006846616C08F08AFA01220021684608F077
:10783000A1FA0A49684608F08BFA0949684608F037
:1078400076FA684608F0BEFA16B010BD16B0BDE86C
:1078500010401DF057BC00008951020809FD0008C6
:107860008B5102080C210148FCF7BAB848060020E9
:107870000C210148FCF75CB84806002010B504460E
:10788000406882080AD0496821F00301091D0844B4
:107890006060204600F042F8204610BDFEE74068D8
:1078A000103120F00300884201D3012070470020EE
:1078B00070472DE9FC47054648680C4620F0030058
:1078C00001AA69461CF008FBDDE9007005EBC71151
:1078D00001EB80098046D9F83C0060B164B1C4E98D
:1078E000020504F10806C46030460421FFF7F7FDE5
:1078F000864202D0FEE7FEE7FEE7C9F83C400120E1
:10790000296900FA07F21143296105EB870100FAA2
:1079100008F04A6902434A61BDE8FC8710B5044695
:1079200000F087F8046010BD2DE9FC4706464FF0D3
:1079300000000D0000900746019042D00C46E94639
:107940000DF10408802907D3084623F053F8411F9E
:1079500001208840401E04444246494620461CF00F
:10796000BBFA009C0A2C2CDA06EB8400019A4069D1
:107970004FF0FF3101FA02F210400CD1641C306963
:10798000A14008401DD023F02DF80446009006EBDE
:107990008000406978B123F025F8034606EBC41156
:1079A000019001EB8000C76B5FB1786820F00300A5
:1079B000A84201D2FEE7FEE739463046009A1EF0A3
:1079C0007DFC3846BDE8FC8710B50446FFF7A6FFEE
:1079D000416841F002014160606840F00100606070
:1079E00010BD10B5044600F024F8416821F00201F2
:1079F0004160606820F00100606010BD70B506460F
:107A00000D46084600F015F8040010D02079C00794
:107A10000BD0686880080BD02146304600F03CF857
:107A200021462846FFF72AFF0546284670BDFEE797
:107A3000FEE7426800F1080122F00300001F08443D
:107A4000910800D1FEE7704770B506460C004FF074
:107A500000001ED0F2B120791546C0071BD0114698
:107A60002046FFF71CFF78B12946204600F025F894
:107A700005462046FFF752FF6868294640F002009D
:107A800068603046FFF715FF2046FFF7AAFF04F1B4
:107A9000080070BDFEE7FEE77CB5054648680C4669
:107AA00020F0030001AA69461CF016FADDE9002364
:107AB000214628461EF002FC7CBD2DE9F0410D4612
:107AC000044600F10801281F0E18606806F1080737
:107AD00020F00300401BA0F1040838460421FFF702
:107AE000FEFC874200D0FEE7606820F0030108EB4F
:107AF0000500001D814200D0FEE7307900F0030050
:107B000040EA0800706020F003000C2800D2FEE775
:107B1000207900F00300284360603046FFF754FFEF
:107B20003046BDE8F08138B5044611F0ADFE05469B
:107B300011F0E5FE0028204605D0616C216416F0A6
:107B400048FC012038BD10F003F9002820461ED063
:107B50000FF0AEFFD4E9100181420CD06064206CBC
:107B600000906A462021204617F0F3FC0128E9D155
:107B7000204616F02EFC284611F0D0FE0428E0D155
:107B8000204615F078F8002111F013F9D9E710F02C
:107B90003DF9D6E7002802D0C01C20F00300704752
:107BA00010F080BDC01C13F057BC2DE9F041044615
:107BB000006815461346476A0E4600222046B8471D
:107BC00001280FD10020BDE8F0812946204600F0B1
:107BD00013F80028F7D020682B460022476A314668
:107BE0002046B8470228F0D020682A46314603696B
:107BF0002046BDE8F041184770B5044600680E46BF
:107C0000026A20469047050010D020683246294677
:107C100043692046984728460AF0FFF9A269314691
:107C2000904728460AF0F0F9012070BD002070BD91
:107C30002DE9F04F0C4685B00546002114F03FFFBA
:107C400058B32146284600F08DFA2146284600F018
:107C500069F80021284615F02BFE834600212846AE
:107C600015F074FE04900021284615F0F8FC012858
:107C70001BD000270021284615F0DCFF804600219C
:107C8000284615F070FD6FF040490646C8450ED1F4
:107C9000688D00050BD401200AE005B02046BDE840
:107CA000F04F2022002113F008BD0127E2E7002059
:107CB0008046284614F0A1FF8246284600218222F1
:107CC00015F06EFEC2B22369A1682068CDE90031CB
:107CD000CDE902075B464146504606F0A1F9A06196
:107CE0004E4504D1688D400501D4012600E00026F0
:107CF000284614F071FF074628460021832215F01C
:107D00004FFEC2B2606900256368E1688DE82B0010
:107D100031463846049B06F083F9E06105B0BDE8C2
:107D2000F08F00002DE9F34F81B00C46019805F06B
:107D300003FC06004FF000081ED1019814F0F0FF7C
:107D400005F0FAFB070074D0019805F0F9FB8146B5
:107D5000019805F0F9FB80468500281D13F07CFB97
:107D600006462A4607EB890113F0ECFB6FF06041F1
:107D700046F828104FF00108019814F03EFF8346A2
:107D8000304600F01DFF2061800013F065FB20608D
:107D90002069800013F060FB0025DFF82CA1A060B3
:107DA00038E056F82510DFF82491514531D10027ED
:107DB0001FE03946019814F082FE4549009016F004
:107DC00010F8A8B9009805F0BFFB012810D1009861
:107DD00005F0B6FBA8420BD1009815F0B5FF494657
:107DE000484501DA084602E0009815F0ADFF8146EB
:107DF0007F1C019814F0A2FEB842DAD8B9F1000F46
:107E000003DBA16841F8259003E0A168002041F858
:107E100025006D1C2069A842C3D8DFF8AC9000256E
:107E200009F10109C9F1000352462F4628469A4636
:107E300014E046E056F82010494503DB6B1803EBCD
:107E40000A050AE0914204D1A16851F820100F44BC
:107E500003E0A3680F4443F82010401C21698142CD
:107E6000E8D80021019815F023FD2169C1F1010234
:107E700000FB02B0C01B00D50020002114E000BFB1
:107E800056F821204A450EDB02EB0A0300FB03F201
:107E900005EBD57702EB670292FBF5F2A768ED1AC6
:107EA000801A47F82120491C22698A4201D9002DF5
:107EB000E6D1B8F1000F04D03046BDE8FE4F10F017
:107EC000F1BBBDE8FE8F00009AFFFF1F010000E03C
:107ED000010006002DE9FC5F054615F071F88346A8
:107EE000A86808B10021C1610021284615F015FEDF
:107EF00001900021284615F083FD8246284615F0A2
:107F00006FFB014601982E4C014401EB0A072846FD
:107F100014F014FE8046002639E0A868DFF8A0902F
:107F20002849006850F82600009015F05AFF68BBF9
:107F3000009816F0AFFAE0BB0021009815F074FB32
:107F4000B8B3012836D0022834D0032832D000211B
:107F5000009815F07EFE60B90098143008F070FDAE
:107F6000019900EB01090021009815F035FC484407
:107F700081460021009815F014FC4844A04205DB1E
:107F80000021009815F00DFC00EB0904761C464515
:107F9000C3D3A86810B1CBF10001C1616FF060409C
:107FA000C44203D004EB0A00B84200DA3846BDE808
:107FB000FC9FFFE70098A969006A401A401CD7E7B8
:107FC000010000E0010004002DE9FE4F054614F019
:107FD000F1FF0290A86808B10021816100212846C4
:107FE00015F06CFD00900021284615F038FD834601
:107FF000284615F003FB00EB0B010098DFF85C91BD
:1080000001EB00084C46284614F098FD0746002175
:10801000284615F018FB01284FF0000645D082E0F5
:10802000A868CA464E49006850F82600019015F02D
:10803000D8FEC8BB019816F02DFA20B10198E96965
:108040004069081A14E00021019815F0EDFA58B1C2
:10805000032809D0062807D0082805D00021019858
:1080600015F0F4FD30B112E00199E8694969401A50
:10807000401C0BE00198143008F0F1FC009900EB73
:10808000010A0021019815F095FB50448246002119
:10809000019815F08FFB5044A04205DB00210198A8
:1080A00015F088FB00EB0A04761CBE42B8D34C45A1
:1080B0003FD05C443DE0A868CA462949006850F8B2
:1080C0002600019015F08DFE60BB019816F0E2F9D4
:1080D000E0BB0021019815F0A7FAB8B3012836D00B
:1080E000042834D0072832D00021019815F0AEFDC5
:1080F00058B90198143008F0B2FC00EB0B0A0021CB
:10810000019815F060FB504482460021019815F05B
:108110005AFB5044A04205DB0021019815F053FBA7
:1081200000EB0A04761CBE42C5D34C4501D0009832
:108130000444A86810B10299494281614C45404607
:1081400002D0444500DD2046BDE8FE8FFFE70198E0
:108150006969C069401A401CD6E70000010000E0D0
:10816000010004002DE9F34F81B00C46019805F0A1
:108170009AFD06004FF000081ED1019814F0D0FDC2
:1081800005F091FD070072D0019805F004FE8146CC
:10819000019805F004FE80468500281D13F05CF967
:1081A00006462A4607EB890113F0CCF96FF06041CF
:1081B00046F828104FF00108304600F001FD6061DC
:1081C000800013F049F960606069800013F044F9A1
:1081D0000025DFF838A1E0603AE056F82500DFF826
:1081E0003091504533D10027DFF828B11FE03946E0
:1081F000019814F064FC5946009015F0F2FDA8B9FE
:10820000009805F0CCFD012810D1009805F0C3FDC1
:10821000A8420BD1009814F033FD4946484501DAD5
:10822000084602E0009814F02BFD81467F1C01985F
:1082300014F084FCB842DAD8B9F1000F03DBE1682E
:1082400041F8259003E0E168002041F825006D1C0D
:108250006069A842C1D8DFF8B490002509F101098E
:10826000C9F1000352462F4628469A4614E04AE0D8
:1082700056F82010494503DB6B1803EB0A050AE0AA
:10828000914204D1E16851F820100F4403E0E36803
:108290000F4443F82010401C61698142E8D8002156
:1082A000019815F053FB8346019814F095FC0146A4
:1082B0006069C0F101020BFB0210C01B00D5002059
:1082C000002113E056F821204A450EDB02EB0A0399
:1082D00000FB03F205EBD57702EB670292FBF5F2A8
:1082E000E768ED1A801A47F82120491C62698A4222
:1082F00001D9002DE6D1B8F1000F04D03046BDE819
:10830000FE4F10F0CFB9BDE8FE8F00009AFFFF1FAF
:10831000010000E00100060070B5044600216E2255
:1083200015F03EFBD8B9204600216C2215F038FB31
:108330004FF48075A84212D1204600216D2215F01D
:108340002FFBA8420BD120460021712215F028FBFB
:1083500028B920460021722215F022FB08B1022024
:1083600070BD20460021602215F01AFBC0B2FF2824
:108370000DD120460021732215F012FB38B920469A
:108380000021672215F00CFB10F0FF00E8D001205F
:1083900070BD2DE9F041044606A81D46174690E839
:1083A0004C0002290FD003290BD1294638461AF078
:1083B00039F90546304608F052FB401B2168084455
:1083C0002060BDE8F081294638461AF02BF90546B1
:1083D000304608F044FB00EBD071491005EBD57036
:1083E000A1EB6000EAE700002DE9FF4F95B0C878E7
:1083F000269CC0070D46002801D0FE4800E0FE483C
:10840000099001D0FD4800E0FD480F9001D1FB48E4
:1084100000E0FB48109001D0FA4800E0FA480390D1
:1084200001D0FA4800E0FA48069001D1F54800E092
:10843000F548059001D1F54800E0F5484FF01409E2
:10844000049069E0D4E901124FF0000BA1EB0203A4
:10845000584659464FF00C0E0FE000BF01EB4102A9
:10846000266909EBC20C16F80CC05FEACC7C08D078
:108470000EEBC202B2589B1A491C8F42EED8002163
:1084800044E04FF0100C0CEBC202B2581044F3E77A
:1084900001EB4106276909EBC60A17F80A20D20743
:1084A00033D1E8B34FF0100C93FBF0F20CEBC60C99
:1084B000CDF848C057F80C804FF0080C08FB02F8C4
:1084C00004220CEBC60C02EBC60257F80CC0BA58DB
:1084D000CDF820C0C44500DDC446624503DC089ADF
:1084E000424500DD4246424504D04FF0010C47F8BA
:1084F0000AC0E346D4F810C00EEBC6064CF80620BE
:108500002769129EBE59801B9B1A491C62698A42C8
:10851000BED8BBF1000F02D06769002F92D100E0F6
:1085200028E00021159815F0A0F8012823D000219B
:10853000002088460D900E900EA90DA8CDE90001EF
:108540002878E368626824991CF0BAF8E87810EAA1
:10855000080F05D0159814F050FB0D9908440D90A4
:108560001799159814F0ABFA0646DFF8A8926FF049
:10857000704B3AE1FEE70121DAE7A749304615F0F2
:1085800030FC00287AD10021304615F0E3F8E8B33A
:108590000027384661690FE0226900EB400352F87A
:1085A0003320B24207D100EB40020C20216900EBDE
:1085B000C2000F5802E0401C8142EDD8E878C007A5
:1085C000708D04D020F4806040F4006003E020F45B
:1085D000006040F48060708506F114000F998246B7
:1085E0008847B84224D0304615F0F3FE70691190E8
:1085F000B0691290F0691390306A1490099A394664
:108600005046904711AA2E21304600E00CE016F0AB
:10861000A0FF304614F084FB3246272116F099FF64
:10862000304615F0D6FE03E0708D20F44060708572
:108630006878012823D0022804D0059A002130460A
:10864000904727E0109906F1140088472168059AA1
:10865000491C21F00101081A00EBD0704FEA600AB2
:108660000021304690470746049A00213046904743
:10867000381A00EBD0710AEB61000BE0ADE0109905
:1086800006F1140088472168049A0F1A0021304629
:108690009047381A0790E87810EA080F06D00F992B
:1086A00006F1140088470D99081A0D9030460021F4
:1086B0006A2215F075F90746304600216B2215F045
:1086C0006FF98246304615F03FFB0C90304614F0AF
:1086D000D7FA0146C7F3417001280DD127F0C040F9
:1086E000484509DCB0F1805F01DBABEB00000C9A80
:1086F0005043642290FBF2F7CAF3417001280CD179
:108700002AF0C040484508DCB0F1805F01DBABEBEC
:1087100000004843642190FBF1FA71692298401AE5
:108720000744B1692398411A01EB0A000190E878E7
:10873000C00706D0039A0021304690470D9908449F
:1087400000E0079800EB070AE878C00701D0079817
:1087500005E0039A0021304690470D99084401999D
:1087600047185AEA070019D0304615F032FE7169F1
:1087700001EB0A007061F16901EB0A00F061B06978
:108780003844B061306A38443062304615F021FE1A
:1087900000233A465146304615F0C4FEE87810EA08
:1087A000080F14D10F9906F1140088472599039AF0
:1087B00008440E9947180021304690470744069A0E
:1087C0000021304690470D993844084404E00E9942
:1087D000259808440D99081A0D90E87817AAC0F357
:1087E0008001159805F03EF90646002E19D0DDE906
:1087F000170113E03B0D0108310D01085F0A010864
:10880000410A0108C1D70108E5D70108D3D70108FB
:10881000AFD70108FEFFFF1F0100060088427FF46A
:10882000ACAE19B0BDE8F08F2DE9F04F91B00E005D
:1088300005463AD0AE61286808B10FF033FF06EB69
:108840004601062000EB410012F006FE286018B336
:10885000022101EB46010144E960042101EB86019C
:108860000144C5E9010101210024012E15D0300188
:10887000103012F015FEA346B100CDE9051B82466B
:10888000C1F1010700EBC600891000F108095C4640
:10889000CDF834B0099196E0FEE7B4220270E868A2
:1088A0000480E8684180A868048011B0BDE8F08FBA
:1088B0004FF00008002F05DC0699032000EB410073
:1088C000074408E0DDE905010A1A052101EB420130
:1088D000401E0F4405900698401C069005A800F025
:1088E000DAF870B1059809AB82100DA943F8282079
:1088F00000F0030041F8280008F10108B8F1040F66
:10890000D8DBB8F1040F64D10C99099888420AD1D8
:108910004AF8240049F824B0DDE90D010144DDE9FD
:108920000F02104418E00A99884218D04AF824002F
:1089300049F824B069680D98085569680001085520
:108940000998641C401E4AF8240049F824B0DDE967
:108950000E0101441098001D084469682CE00B9931
:108960004AF82400884249F824B0DDE90D010844A2
:1089700011D0696808556968000108550998641C98
:10898000401E4AF8240049F824B0DDE90F010844EC
:108990000830696810E00F990844696808556968EB
:1089A000000108550998641C401E4AF8240049F843
:1089B00024B0109869680C300BF1010B08556968F8
:1089C00000010855641C05A800F065F800287FF434
:1089D0006FAF0AEB840140F2D320464351F8041CE8
:1089E000B012814205D109EB840151F8041C814287
:1089F00019D0A6EB8021B1F5007F03DC494341F398
:108A0000CF3106E0C1F58061494341F3CF31C1F177
:108A10000F014AF8240049F8240068680155686885
:108A200009010155641CA01E0DE000BF59F820206B
:108A30004AF824205AF8202049F8242069680A5C62
:108A40000A55401E641C0028F0DAEB680021084635
:108A500019801AE0EA6822F81100AB683AF8202081
:108A600023F811200AE0AB685AF8202033F811608F
:108A7000964200DA324623F81120401C59F8202093
:108A80008A4201D1A042EEDB491CA042E2DB504603
:108A90000FF008FE09E703C8814201DC012070479E
:108AA00000207047012070477CB504460FF06CFB36
:108AB000064620460FF064FB0546304614F030F9B8
:108AC0000446302D23D00B2D4DD110F0DDFE10B11A
:108AD000007A012847D06946304614F083F994F8AB
:108AE000300010F00C0F30461BD014F086F805460D
:108AF0000021204614F0CBFD0128009805EBD5712C
:108B00000CD000EB610000BF90FBF5F512E0E16ACC
:108B100002B00022BDE8704019F006BBC0EB610056
:108B2000F2E714F059F8019900EBD07201EB620101
:108B300091FBF0F5002D00DA0025E06A0026A8423E
:108B400000D0012610F0A0FE08B1012200E00022B2
:108B50002946204619F0E8FA002E04D000222021F0
:108B6000204616F0F6FC7CBD30B5002822DA8B1AC0
:108B7000002B00DC531A64225343C0F30901B3FBFA
:108B8000F1F1C0F30953C0F38922C0F3095000EB9F
:108B9000800003EB83034000B1EB430F01D20C468E
:108BA00000E0044602EB8205B4EB450F03D202EB72
:108BB0008200400030BDB1EB430FFBD2084630BD10
:108BC000014600206FF0604200E0401C51F8203068
:108BD0009342FAD170471FB5044690F8640000F044
:108BE0000100884225D094F8640011B140F00100E2
:108BF00001E020F0010084F8640004F150016846AF
:108C000007F0AAFEE06A00994269114400910199B7
:108C1000806908440190E06A029940690844029022
:108C2000E06A03998069084403906946204615F07C
:108C3000EBFB1FBD08B50846114609F086FF009002
:108C4000BDF800009DF8021040EA014008BD000098
:108C50002DE9FC5F088C0C46C0F307208F6C09F0EF
:108C600095FF8146208D636A81B2CA00B2FBF9F09C
:108C7000072202EBC002D6081A0C01FB02FA02FB23
:108C800000F599B20E23364800960AF049FF060017
:108C900007D0206AD6F81080000C000704D5386A87
:108CA00018E00020BDE8FC9F207C012801D080B1A5
:108CB00015E001A80090534642460C21386804F0A4
:108CC000A0F910B90199514509D030460AF069FF61
:108CD000E7E7E06852460169404612F033FC208C19
:108CE000C0F307200E2837D008EB0A00A0F1010BD3
:108CF00008EB0500A0F1010A012000FA09F0401E6E
:108D0000002100F0FF0E0B4624E000BF9BF800009E
:108D10004A46C84010EA0E000FD080460AE000BF65
:108D2000C2F1080C00FA0CFC4CEA080C4A440CF0A6
:108D3000FF08D2B2082AF3D340468AF8000001EBBC
:108D40000900C1B2082902D30021ABF1010BAAF13D
:108D5000010A5B1CAB42D9D3FE610120E662A1E7A8
:108D60008C5300202DE9FC478F6C086A0E46D7F81B
:108D700000A0C0F307254FF48079072D0DD0082DF2
:108D80000DD0092D0DD00A2D0DD000218900884667
:108D9000C0F3C04048B1386A28E00221F6E7042158
:108DA000F4E71021F2E74946F0E7307C012801D0D2
:108DB000D8B115E0084612F04FFB040009D001A815
:108DC0000090434622460C21504604F01AF920B97F
:108DD00000E0FEE70199414505D020460FF062FC16
:108DE0000020BDE8FC877C6001E0F0680469346322
:108DF000072D09D0082D09D0092D09D00A2D09D039
:108E0000002070630120ECE70220FAE70420F8E775
:108E10001020F6E74846F4E72DE9F0430024DDE9A9
:108E20000759D617072808D0082810D0092819D0C4
:108E30000A2821D00020BDE8F08302EB567405EB30
:108E4000E40502F007020120C2F1070416E002EB7C
:108E50009674022005EBA40502F003020624A4EB9D
:108E600042040BE002EBD274042005EB640502F02F
:108E70000102A0EB820401E0082015440122824097
:108E8000521E1FFA82FC0026C0F1080211E02F7862
:108E900009EB8608E74007EA0C0701EB8707241A6D
:108EA0003F6864B2C8F80070002C01DA14466D1CEB
:108EB000761C9E42EBDB0120BDE710B10268D2694F
:108EC0001047FEE770B505460FF05AF904462846EC
:108ED0000FF0B0F9352C07D1D0F8F802002803D0F4
:108EE000BDE870401AF07EBB70BD00002DE9F8436C
:108EF00017460D4680460AF0BBF80E4E04467078C1
:108F0000844205D05A2014FB00F0FBF70FFE74706A
:108F1000307850B10097A88983B2288982B2A88896
:108F200081B2288880B2FBF781FC4046BDE8F84357
:108F30000AF044B8C00300202DE9F0410446C0699E
:108F40000E4610B10020BDE8F0810122002130461C
:108F50000BF026F905004FF0FF3716D030460BF026
:108F600089FD90B10220A86405F13800E561C4E9EB
:108F70000160204603F03BFCE16903208864002087
:108F8000E0610BF0ADF80120DDE73846DBE7414357
:108F900002EBA121414303EBA12141438812704719
:108FA0007CB5044618F0D2F894F8A01004F12C0512
:108FB00041F0010184F8A010F8B101281DD0022869
:108FC0001DD110F061FC694610F07CFC032269465B
:108FD000204616F0BFFE0021204614F04CFB01286D
:108FE0000ED00026204606F023F9014694F84C00E6
:108FF0000E40B04206D0012205E0C4F89C507CBD72
:109000000126EFE7002204F1380089B3009902B38A
:10901000D4F884209142F0DBE26F91423ADC626F37
:10902000E16F009B891A01EBD17102EB6102D11A49
:10903000002900DC991AD4F88460D4F88C20921BA3
:1090400002EBD27206EB6206F21A002A4ADC9A1B85
:1090500048E0D4F88C209142CFDC626F914219DB5A
:10906000DDE700BF44F89C5F207920F0020006E0B5
:1090700007E000BF44F89C0F207940F00200207107
:109080007CBD01994AB1D4F890209142B5DCA26F21
:1090900091420ADAC4F89C007CBDD4F88820914241
:1090A000ABDBD4F880209142F4DCD4F88020A16FAF
:1090B000521A02EBD27201EB62020199511A002995
:1090C00001DC0199891AD4F89030D4F888209B1AD1
:1090D00003EBD37302EB6303019A9A1A002A01DCB3
:1090E000019AD21A8A42C5DABCE72DE9FF4FB7B020
:1090F000154637981F460C468268DDF81081469E5B
:109100001DA807F0BEFC00287DD01DA807F0A7FC15
:109110001C9005A82C22002112F0CFFA1C9812F006
:109120009BF903900B900020219022902390012323
:109130004246294624A80EF037F824A82190002F93
:1091400007DD00233A4621462DA80EF02DF82DA864
:10915000229010A805900D90BDF81401ADF82900DB
:109160009DF816018DF82B008DF828602068C11934
:109170002868814200DD08461890A068A968C01BD5
:10918000884200DB08461A906068C119686881420D
:1091900000DD08461990E068C11BE868814200DAEA
:1091A00008461B9018A807F05AFC61686A6891424B
:1091B00001DC012100E000218946E168EA68914272
:1091C00001DB012100E000218A4621682A689142E2
:1091D00001DC012600E00026A168AA68914201DBBB
:1091E000012200E00022904606EA080101EA090196
:1091F0004FF0010B11EA0A0F03D0322801DA4FF0C9
:10920000000B012000E030E18DF8300019EA0B0F6F
:109210000CD0189810901A98129060681190686895
:1092200005A9401E139037980CF015FC1AEA0B0F95
:109230000CD0189810901A981290E86805A9401C54
:109240001190E068139037980CF005FC2968A86825
:10925000814205DB96B1B8F1000F02D0206812E020
:1092600066B120681090286805A9401E12901998D0
:1092700011901B98139037980CF0EDFBB8F1000F8C
:109280000CD0A868401C1090A068129019981190FA
:109290001B98139005A937980CF0DDFB1D98BBF1C6
:1092A000000F109006D018981F9A411E8A423EDA8D
:1092B00010463DE01F98129068686168401AB842F5
:1092C00000DA3846814600252EE060684619E068DD
:1092D000A0EB05081E98B04202DD2099414522DB33
:1092E000FF211C9A039812F0E8F91C98009033466D
:1092F00021A8109A03990DF03DFE8DF830001E98BC
:10930000B04205DC119605A9139637980CF0A3FB23
:109310002099414507DBCDF8448005A9CDF84C8064
:1093200037980CF098FB6D1C4D45CEDB92E0401E4B
:10933000129010A807F093FB051E39DD56EA0900CC
:1093400019D01E9C14E011942A46FF21139403980F
:1093500012F0B3F90095234621A8109A03990DF055
:1093600009FE8DF8300005A937980CF074FB641CD9
:109370001998A042E7DC56EA0A0619D01B9C13E0B4
:1093800011942A46FF211394039812F096F9009540
:10939000234621A8109A03990DF0ECFD8DF83000BA
:1093A00005A937980CF057FB2098641CA042E7DA17
:1093B00012991D98491C884201DD014601E012996D
:1093C000491C10911A99491C884201DC1A98401CCA
:1093D00010901F98129010A807F041FB051E39DD70
:1093E00058EA090019D01E9C14E011942A46FF2166
:1093F0001394039812F061F90095234621A8109A5E
:1094000003990DF0B7FD8DF8300005A937980CF0E1
:1094100022FB641C1998A042E7DC58EA0A0019D024
:109420001B9C13E011942A46FF211394039812F019
:1094300044F90095234621A8109A03990DF09AFD4E
:109440008DF8300005A937980CF005FB2098641CB6
:10945000A042E7DA24A80DF0CBFD002F02DD2DA8F5
:109460000DF0C6FD03980FF01DF93BB0BDE8F08F7D
:109470002DE9FF4794B015460C46824604A82C22DD
:109480000021209E12F019F9CDF810D0BDF85C0033
:10949000ADF825009DF85E008DF827008DF824605A
:1094A00060686968884201DC012700E00027E06805
:1094B000E968884201DB012600E00026206829686F
:1094C000884201DC012100E000218946A168AA68E8
:1094D000914201DB012100E000210090A068029090
:1094E0006068019068688846401E03901FB104A917
:1094F00050460CF0B0FAE868401C0190E068039018
:109500001EB104A950460CF0A6FA20680090286805
:10951000401E02900FB1686800E0606801900EB1D3
:10952000E86800E0E0680390B9F1000F03D004A9F7
:1095300050460CF090FAA868401C0090A068029079
:10954000B8F1000F03D004A950460CF084FA18B00B
:10955000BDE8F0872DE9F04F8B46A2F57F41A1B021
:1095600091460646FF3942D0F46A208D80469842E3
:1095700004D02385608D40F0080060854FF4802A78
:109580005146204614F00EFB07465146204614F083
:109590002DFB054638460FF07AF80746304604F0B2
:1095A00050F980697A1909FB0200014605EBD57074
:1095B000A1EB60001D9038446D1E28441F90F06A96
:1095C00041691C91C0691E9068460CF005F86A4616
:1095D0005146204614F06FFD1CAA694658460BF010
:1095E000E5FDA4F82880608D20F00800608521B09A
:1095F000BDE8F08F2DE9F04F0E46A2F57F41A5B0F2
:1096000090460546FF395CD0EC6A278D9F4204D016
:109610002385608D40F00800608503A80AF09CFF58
:109620004FF4802903AA4946204614F086FC494697
:10963000204614F0DBFA1190284604F002F90500E8
:109640003FD00B980FF023F8119AA969131808FB63
:10965000031119911146199A01EBD171A2EB610125
:10966000119A19911144401E08441B90606918908A
:10967000E0691A9018AA06F118011FA807F001FA6C
:10968000D0B118360DF17C0C96E80F008046894663
:1096900092469B469CE80F0086E80F002846183E3D
:1096A00010F022FE0A9005F1140203A930460AF0D8
:1096B00022FF183686E8000F2785608D20F008000D
:1096C000608525B0BDE8F08F7FB50446D0F8A8527C
:1096D00004E000BF0AF00CFD0AF04EFCA86B002865
:1096E000F8D1204609F000FD18B12648006924F0A1
:1096F00038F901202063A16BC90702D0A16B89074B
:1097000000D400206063606B08B1012600E00026F1
:10971000A06A20B3286821696A460569D4F8000365
:10972000084400906169D4F8040308440190216959
:10973000D4F80803084402906169D4F80C03084483
:1097400003903A21204609F071FDA36A2A46694632
:10975000204698476A463B21204609F067FD20468F
:1097600009F0C2FC00280BD094F83900012801D17F
:10977000002E05D0616AE069814200D1206A6062F2
:109780007FBD00009452002038B540680C46010CA3
:10979000491E83B200220091114620465B1E07F04D
:1097A000C2FA38BD2DE9F047B8B005460EF0ECFC22
:1097B000044628460EF01FFD8246E06A10F094FD34
:1097C000054694F86400C00771D004A80BF004FFAC
:1097D0004FF4C02904AA4946204614F06CFC04F159
:1097E0005001684607F0B8F8E06A009942691144F0
:1097F0000091019980696A4608440190E06A0299E3
:10980000406908440290E06A039980690844039023
:1098100004A950460BF0CAFC4946204613F097FFB6
:1098200006464946204614F070F8871949462046F6
:1098300014F0B3F84FF000081E490644CDF8D48068
:10984000CDF8D880206E0968284488470246206EEB
:10985000411935A811F076FE00985822384400903E
:109860000198414630440190E06A14F099F80546A9
:1098700020A80AF071FE20AA4946204614F05DFB9C
:109880009DF83000022805D829462B9809F06EF97A
:1098900000280CD135A827909DF8CC006A4640F0EE
:1098A00040008DF8CC0020A950460AF024FE38B0C4
:1098B000BDE8F08710E005082DE9F04FEDB0054652
:1098C00038300E465E9011F059FD00287ED105F12A
:1098D000140206F1180168A807F0D3F8002875D023
:1098E000183668AC96E80F0083462091CDE96423D2
:1098F00094E80F0086E80F003DA8183E0BF05DF9D4
:109900004FF4C0243DAA2146284614F070FB21A83C
:109910000BF062FE21AA2146284614F0CCFB21461A
:10992000284614F08DF900EBD070471021462846E8
:1099300014F086F900EBD0704FEA600A5E9811F0DF
:10994000A4FC90E040223DA94EA811F0FBFD70223E
:1099500021A9684611F0F6FDA089ADF86401A07B4D
:109960008DF86601A089ADF82100A07B8DF8230059
:10997000A08AC00502D5D4E900010BE0A2686FF00F
:10998000004082426BD066AB2846216908F0CCFDCE
:10999000DDE966016A6902EB0008A86900EB0109CC
:1099A00027B1BAF1000F01D0012000E0002066903D
:1099B000A8EB07005F9008EB07006190A9EB0A0095
:1099C000609009EB0A006290207D00E056E081077C
:1099D0001CD0C00701D0686900E04046CDE95509B8
:1099E000207D800701D5E86900E04046CDE95709B0
:1099F0000020519003904EA930460BF0A2F86698D3
:109A000020B15FAA694630460BF0D0FB207D10F0F4
:109A10000C0F1ED0CDF85481207D400701D5A869D8
:109A200000E04846CDE95608207D000701D5286AA8
:109A300000E0484658900120519003904EA93046CE
:109A40000BF07FF8669820B15FAA694630460BF0AC
:109A5000ADFB3F98401C3F902398401C239021462B
:109A60005E9811F00FFC04007FF46CAFDDE9642315
:109A70002099C6F818B01C3686E80E006DB0BDE817
:109A8000F08F2DE9F04F884601F11802A5B0044689
:109A900000F114011AA806F0F4FF002872D008F1B2
:109AA000180114AD91E80D00D8F82410179185E83D
:109AB0000D001AAE08F1180096E82E0080E80E009E
:109AC00000212046C8F8245013F035FE0546002139
:109AD000204613F008FF28441E900021204613F072
:109AE0004AFF0544204613F088F81390204613F0EF
:109AF00073F8129002A80BF060F802AA0021204629
:109B000014F075FA20460021322213F049FF00F0CC
:109B1000FF090021204613F00EFE82462046002158
:109B2000342213F03DFFC6B2204613F07BF9239098
:109B3000204613F039FAA16EB9B3A1692944A1EB0B
:109B4000000B60690990E0690B90B4F8680000258B
:109B500007B2B9F1020F26D9BAF1000F23DDB00721
:109B600005D50021204613F006FF00B90125F007B6
:109B700019D020460021112213F012FF98B97F1E40
:109B80003FB210E055E0A16E1298491E6843B0FB49
:109B9000F1F058440A900C9002A9049540460AF04E
:109BA000D0FF6D1C2DB2BD42EDDBE06EC0B361692C
:109BB0001E98002701442398B9F1020FA1EB000B76
:109BC000A0690A90206A0C90B4F86C0005B225D9FF
:109BD000BAF1000F22DD700705D50021204613F0F1
:109BE00082FE00B90127300718D520460021132234
:109BF00013F0D6FE90B96D1E2DB20FE01398E16EF2
:109C00007843491EB0FBF1F0584409900B9002A92B
:109C1000049740460AF095FF7F1C3FB2AF42EDDB50
:109C200014AD08F1180195E81D0081E80D00C8F891
:109C3000244025B0BDE8F08F2DE9F047A0B00646DE
:109C40000EF09EFA054630460EF09EFA0446172D99
:109C50002DD01A2D28D1206C002825D0E06B0028AB
:109C600022D0A06C00281FD0E06C00281CD0304609
:109C70000EF0C1FAA16D054601F0030001287BD06A
:109C8000890779D002280FD168460AF065FC6A4638
:109C90000021204614F051F9E06A079004F1140203
:109CA000694628460AF027FC20B0BDE8F087304618
:109CB0000EF0B2FA054600780228F5D0A06D4FF0FC
:109CC0000106C143890755D000F00301022951D094
:109CD000C0F3840008F07DFFF0BB20460021442241
:109CE00013F05EFEC0B2FF2844D1606CA0BBA06C34
:109CF0003102884207D1E06C884204D1002204F18D
:109D00001401686830E007A920460FF0B1FB204637
:109D100012F0B6FF0746204614F016F80146B4F8D4
:109D20004820B4F84C0092B2009207AB80B2CDE963
:109D3000010300233A4603A80FF05DF80399606918
:109D4000084403900499A069084404900599606947
:109D500008440590069901E00CE00DE0A06900229E
:109D60000844069003A9686806F0ABFE10B1206BAA
:109D7000002899D02E7097E701A80AF0CDFA01AA21
:109D80000021204614F07FF8D5E90880D5E9066760
:109D9000814611A920460FF06BFBA06C0D90E06C82
:109DA0000E90606C0C9094F85800C109BDF85000FA
:109DB00061F30C30ADF85000B4F85800010B9DF879
:109DC000510061F303008DF85100206B1B90E06A95
:109DD0000890A269206C1044401E00906169E06BFD
:109DE0000B1816A882465B1E06F09DFF2046002138
:109DF0000C2213F0D5FD1A90B4F85800C0F30322DA
:109E00000A2A10D2A06B0090514604F11400636B33
:109E100006F080FC0DF1580C9CE80F000DF1700C61
:109E20008CE80F0007E00C2A0ED016AC94E80F0067
:109E30001CAC84E80F001CAA01A928460AF018FAF5
:109E4000183585E8C0032FE705F1180104F1140265
:109E5000084606F016FED4E90D12504606F056FFED
:109E6000E8691799411A206C091A491C91FBF0F214
:109E70004243A8691699411AE06B091A491C91FBE3
:109E8000F0F14143504606F041FF18350DF1700CDA
:109E900095E80F008CE80F00BDF85000183D40F425
:109EA0000050ADF85000C6E72DE9F04FADF5117D3B
:109EB00005460EF069F9044628460EF09CF98F908D
:109EC00001A9204612F0AAFE00216822204613F0C4
:109ED00067FD054600216922204613F061FD024618
:109EE000294601A806F0C0FD01A806F0B8FD0990BA
:109EF00001A806F0A5FD0790D4E90C10401A5FEA0E
:109F0000000801D14FF0010894F870000027C0F359
:109F1000C200012805D0022806D007990998884276
:109F200001DB012700E00027204607F0BFF8129070
:109F30000021204613F0D1FC5D900021204613F053
:109F4000EDFC5C900021204613F00FFD5B9000219A
:109F5000204613F095FC059004F13C0001A9009007
:109F600006F0DFFCE16B5D986FF001050144E163F1
:109F7000616C5C98091A6164216C5B9801442164EE
:109F8000A16C0598091AA164009877B106F058FDF4
:109F9000042818DA0798A16900EBD07005EB60007F
:109FA00008442064001DA0640DE006F058FD04285C
:109FB00009DA0998616900EBD07005EB600008448C
:109FC000E063001D6064009806F049FD05460098B6
:109FD00006F036FD2FB1A94604F14405C548009EA0
:109FE00005E08146C44804F1400604F148050D909F
:109FF000E26E501C14D0616E206BA36E091A181A01
:10A0000001FB09F100FB09F091FBF8F190FBF8F07E
:10A01000401A5043C21700EB126001EB202006E00B
:10A02000A16B206B081A00FB09F090FBF8F0E26DC1
:10A030008346501C14D0616D206BA36D091A181A49
:10A0400001FB09F100FB09F091FBF8F190FBF8F03E
:10A05000401A5043C21700EB126001EB202006E0CB
:10A06000D4E90B10081A00FB09F090FBF8F08246C7
:10A0700020460021272213F093FCC0B20FB1012823
:10A0800000D0002094F84C10814208D030462E4673
:10A0900001210546CAF1000ACBF1000B00E00021C6
:10A0A00047B1326802EB0A002860326802EB0B000D
:10A0B000306008E02A68A2EB0A00401C30602A6881
:10A0C000A2EB0B002860129840B3206B404200FBCB
:10A0D00009F090FBF8F097B129B133682A46181AB5
:10A0E0003146401C03E033683246294618442B6849
:10A0F00011E00B6010601FE0136008601CE021B1EC
:10A100002B682A463146184404E02B683246181A58
:10A110002946401C33688342EEDDEAE70D9900983A
:10A120008847012808DC00221F21204615F011FA7B
:10A130000DF5117DBDE8F08F7AA8009906F0F1FBCE
:10A1400022A80BF049FA22AA4FF40031204613F05E
:10A15000B2FF204600210C2213F022FC054607998D
:10A160000998884200DB0846B5EB600F00DD45101A
:10A17000DDF8A480009806F072FC0446009806F012
:10A180005FFC8442009802DA06F069FC01E006F008
:10A1900057FCB8EB600F01DD4FEA60089DF8B7008F
:10A1A000002400F0070017B1022802D002E00128C5
:10A1B00000D101242E9800B101245D9801264FF0B2
:10A1C0000009002810DB5C9800280DDB5B98002854
:10A1D0000ADB0598002807DBA84505DA2A4601A90D
:10A1E0007AA806F06EFC98B34E4694B3702222A96A
:10A1F0005EA8F6F7B1F88DF8C0918DF8B3918DF89F
:10A20000D0918DF898917AAA5EA98F980AF0CEFF26
:10A210008DF8F490702222A93EA8F6F79DF88DF8EB
:10A2200050910DF5F47A8DF840918DF864919AE88B
:10A230000F000DF5FE7A8AE80F00ECB197B1019995
:10A240005D9808447F9003995C98081A819011E00A
:10A2500000E04CE054F0010049D08DF8D0908DF82A
:10A26000E090D5E702995B9808448090DDE90410FE
:10A27000081A8290CDF814917FAA10218F980AF0C5
:10A280002FFC07467FAA3EA90AF090FF83A80AF098
:10A2900089FF4EB101AE96E80F008AAE86E82F0026
:10A2A00083A938460AF046FF4CB17AAC94E80F0017
:10A2B0008AAC84E80F0183A938460AF03BFF07A85F
:10A2C0000AF02AF87FAA07A90E978F980AF08CFB4C
:10A2D000702222A93EA8F6F73FF88DF818918DF864
:10A2E00033917AAA3EA98F980AF060FF20E77AAAF4
:10A2F00022A9F8E75F0A0108410A01082DE9F043A5
:10A30000BDB005460DF040FF044628460DF073FF32
:10A3100081460021204613F0AEF901280BD000251C
:10A32000204604F085FF064694F84C103540A942BB
:10A3300003D0012502E00125F2E70025204616F0B2
:10A3400010FF074620467EB112F09AFC804637B1D6
:10A35000E06A002803DA1DB104E038900EE00DB188
:10A36000E06BFAE7606CF8E713F0EEFC80460FB3A1
:10A37000E06A00281EDAF5B11FE0399068460BF05C
:10A380002BF96A464FF44031204613F094FE3346D1
:10A39000424638A920461AF0CCF904F1840038A9C5
:10A3A000074606F0D0FA204616F0D0FE022806D066
:10A3B0003A462AE00DB1A06CDFE7206CDDE77022A1
:10A3C00069461CA811F0BEF83A46694648460AF0AC
:10A3D000EDFE2EB115B1606C389004E0E06BFBE748
:10A3E000D5B1206C39903346424638A920461AF040
:10A3F000A0F904F1740038A9044606F0A4FA70220A
:10A400001CA9684611F09EF82246694648460AF0A3
:10A41000CDFE3DB0BDE8F083A06CE3E72DE9F04F41
:10A42000ADB004460DF0B0FE054612F079FC0646CC
:10A430000EA80AF091F80EAA0021304613F07DFD17
:10A4400020460DF0D8FE00F1180104460FC98B46D6
:10A45000CDE90723824604F1180106F1140223A86E
:10A460002B9106F00EFB002860D023AF97E80F0079
:10A4700004F1180787E80F0027A9304603F093FC82
:10A4800068690190A8690290E8690390289801AA78
:10A49000049010462B9906F0F4FAC8B1D4E908816B
:10A4A000F4E906670DF1040C89469CE80F0084E886
:10A4B0000F002846183C0FF017FF159005F1140205
:10A4C0000EA920460AF017F804F1180080E8C0032E
:10A4D000686901902A980290E8690390286A01AAA5
:10A4E000049010462B9906F0CCFAC8B1D4E9088143
:10A4F000F4E906670DF1040C89469CE80F0084E836
:10A500000F002846183C0FF0EFFE159005F11402DD
:10A510000EA9204609F0EFFF04F1180080E8C003FF
:10A52000DDE90723C4E90823C4E906AB2DB0BDE883
:10A53000F08F00002DE9F0438BB00646DDE912985C
:10A540001D4617460C46484618F0EBF8002872D115
:10A5500000234A4601A928460DF0C9FFBDF80C00AA
:10A56000002868D0BDF80A10002964D0BDF90E306B
:10A570003A681A441144491E07920991D5E9031219
:10A58000891A7A681144BDF91020091A891A0844F9
:10A59000401E0A900891002207A8B16806F0E8FA68
:10A5A00030B1B1680022E06806F0E2FA002842D13A
:10A5B0000198002580B39DF812000021401E082854
:10A5C00021D20095BDF80C30BDF80A20A06909F031
:10A5D00088FC010017D1A06908B109F0E2FABDF8C2
:10A5E0000C20BDF80A1001FB02F0402800D25200F6
:10A5F0000E231248009509F093FA01000DD0BDF822
:10A600000C00C880A16101A80DF06CFF206008B1AA
:10A610009DF81200207102E000E0FEE7257107A816
:10A62000A06001A8002320611A4621463046C04799
:10A6300001A80EF02EF80BB0BDE8F0837453002093
:10A64000F0B58FB01D4616460C0007464CD0207959
:10A65000092849D2DFE800F0051919481948484887
:10A660001900684609F0E1F8E07D8DF82800A08A1D
:10A67000ADF82000A07D8DF82200012009906946E8
:10A680003846E2680BF0DBFB2EE0A3680DF12C0CE2
:10A690000FCB8CE80F000BA806F0E1F90E2109F0B2
:10A6A00045FC0B99401E08440D9068462C22002161
:10A6B00011F003F8A08AADF81500A07D8DF8170001
:10A6C000E07D8DF814002068016906910BA90891BE
:10A6D0000089694680B20990A068009002208DF838
:10A6E0001C0038460BF0B7F9002E09D0002D07D01A
:10A6F0000FB02A4631463846BDE8F0400CF01CB990
:10A700000FB0F0BD2DE9F34F086B0C46401E43100F
:10A7100000F00100C518C969606A8FB0814201DA92
:10A720000A4600E00246009200DD0846A0F1010062
:10A730000290206A6946A0EB05000190206A184447
:10A7400003900F988268084606F09BF9002838D0DD
:10A75000A06B18B1606B08B1012600E000262C2127
:10A7600004A810F0EAFFCDF810D0A08DADF82500B8
:10A7700094F82E008DF8270094F83C006D468DF873
:10A780002400D6B1684606F06AF90646039F019890
:10A790000390D4E90D100844009991FBF0F200FBFE
:10A7A000121A304610F058FE4FF0020B0C958DF83F
:10A7B0002CB081460A90019D35E004A90F980BF05A
:10A7C0004AF911B0BDE8F08F3246FF21484610F03B
:10A7D00074FF002150460B465A4617E0D4F834C0A7
:10A7E000844506DBACEB000C0FFA8CFC6144604442
:10A7F00008E0D4F83880C444844501DA002001E040
:10A8000009F80130401C8DF82C20491CB142E5DBD1
:10A8100004A90F980BF01FF90198401C01900398B0
:10A82000401C6D1C0390BD42CEDD48460DF03AFF42
:10A83000C7E700002DE9F34F8A46096ADAF82800D5
:10A84000D9B00AF11C040AF12406814205DA214636
:10A85000684615F02BFC314604E03146684615F099
:10A8600025FC2146DDE90057684615F01FFCDDE9AF
:10A870000046A4EB0508A6EB0709B8F1000001DCCF
:10A88000C8F10000B9F1000101DCC9F10001884202
:10A8900001DD012000E000200190DAF8301058B10D
:10A8A000B9F1000001DCC9F100004201B8F100007B
:10A8B0000DDCC8F100000AE0B8F1000001DCC8F1CD
:10A8C00000004201B9F1000001DCC9F1000092FB77
:10A8D000F0F0924A105C48433F30C0114FEA600BE1
:10A8E00000F0010202EB0B010691A54201DA2946B4
:10A8F00000E02146A1EB00010A9101DD294600E0BC
:10A90000214601440C91B74201DA394600E0314654
:10A91000A1EB00010B9101DD394600E0314608440E
:10A920000D9059980AA98268084606F0AAF80028EE
:10A930007DD014210EA8F5F728FD1EA80E902CA896
:10A940000F9001990020002972D0B8F1000F13DD9B
:10A95000A6EB0B01CDE900102346A7EB0B0229461D
:10A960001EA80CF08DFB069801213044CDE90001B2
:10A97000069823463A1812E0069923463144CDE959
:10A980000010069829463A181EA80CF079FB012100
:10A99000A6EB0B002346A7EB0B02CDE900012946ED
:10A9A0002CA80CF06DFB9AF83D004FF0020BC0068E
:10A9B0001AD4032107EB0800CDE90001A5EB090338
:10A9C0003A4629463AA80CF05BFB06EB0801CDE9B4
:10A9D000001BA4EB09033246214648A80CF050FBAB
:10A9E0003AA8109048A811900AA806F038F8044632
:10A9F00015F008FD08F000FB05460AA806F025F84A
:10AA0000A84203D20AA806F020F80546A846284620
:10AA100010F022FD81460D9F0B980D9000254246B7
:10AA2000FF21484610F049FE2C2113A801E071E0F7
:10AA300014E010F082FE0AA91391BAF82C20ADF8A8
:10AA400061209AF82E008DF863009AF83C008DF88A
:10AA50006000CDF864901B910B9E3AE0CDE9006058
:10AA600006983A46231829181EA80CF009FB012065
:10AA7000CDE90060A4EB0B033A46A5EB0B018FE791
:10AA8000009409EB05010A9A33460EA808910CF0D0
:10AA900071FA8DF8680018B92146089810F04DFE3B
:10AAA00025442919414503D20D98401C0D900FE013
:10AAB0008DF868B013A959980AF0CDFF0D980025BC
:10AAC000401C0B900D904246FF21484610F0F5FDCA
:10AAD000761CBE42D4DD0D990B98884207D0481EE3
:10AAE0000D908DF868B013A959980AF0B4FF484644
:10AAF0000DF0D8FD1EA80CF07BFA2CA80CF078FA0B
:10AB00009AF83D00C00605D43AA80CF071FA48A89E
:10AB10000CF06EFA5BB0BDE8F08F000094E0050821
:10AB20002DE9F04F8346086B0C46401E411000F0A3
:10AB300001004218E06991B0821A08440092029024
:10AB4000216AA06A814200DA08460190216AA06A5F
:10AB5000814200DD0846401E039069460846DBF846
:10AB6000082005F08EFF00283BD0A06B18B1606B69
:10AB700008B1012600E000262C2104A810F0DDFD1C
:10AB8000CDF810D0A08DADF8250094F82E008DF8EA
:10AB9000270094F83C006D468DF82400EEB168461D
:10ABA00005F05DFF0F90039F019803900F9810F040
:10ABB00053FC80460A9002200C958DF82C00D4E9B5
:10ABC0000D10084401994FF0000991FBF0F200FBD1
:10ABD00012150E464FF0010A25E004A958460AF066
:10ABE0003AFF11B0BDE8F08FFF2140460F9A10F0F8
:10ABF00064FD606BA84202DA8DF82C9001E08DF8BC
:10AC00002CA0D4E90D100844A84200DC002504A9BA
:10AC100058466D1C0AF01FFF0198401C01900398D4
:10AC2000401C761C0390BE42DEDD40460DF03AFD2E
:10AC3000D7E72DE9FF4705460DF0A6FAC46A284676
:10AC40000DF0D9FAE26A054600F11801684614329F
:10AC500005F017FF002834D0D5E90881F5E906672B
:10AC600089469DE80F0085E80F0094F84C00183DD8
:10AC7000800628D5A26C206C824208D12123294667
:10AC80002046FEF767FC20462123A26C13E0202318
:10AC900029462046FEF75EFC204620232946A26C6A
:10ACA000FEF7A8FC204601232946226CFEF752FC41
:10ACB000226C204601232946FEF79CFC183585E8C6
:10ACC000C003BDE8FF87204620232946A26CFEF77B
:10ACD00041FC20462023A26CEDE700002DE9F04F57
:10ACE000F7B005460DF050FA0446806B00287DD081
:10ACF00028460DF080FA7290608D40F00801618561
:10AD000020466CA911F08AFF0025278D2585608DCE
:10AD10002E4640F0080161853BA80AF05DFC57A86B
:10AD200009F01AFC4FF4A0293BAA4946204613F02B
:10AD3000C2F957AA4946204613F0FFF8608D00215A
:10AD400020F0080060852046278512F011FE7590DE
:10AD50000021204612F097FD74900021204612F049
:10AD6000BFFD73900021204612F0DBFD82460DE10D
:10AD7000761CE06A90A150F8260016F051FC0028DD
:10AD8000F6D0606B30F81500C1067CD44FF0000897
:10AD9000C10501D54FF00108400602D548F08000FA
:10ADA00012E0206CA84210D1B80601D548F0200866
:10ADB000B80701D548F00208780701D548F0040823
:10ADC000380702D548F008008046206B00EB0511DB
:10ADD00003A805F0AFFD03996C98049A0144039110
:10ADE0006D99114404910599084400E0D6E005905E
:10ADF0006D990698B8F1000F084406907ED0A4F82B
:10AE00002880608D40F0080161850AA80AF0E4FB03
:10AE100026A809F0A1FB0AAA4946204613F04BF9DF
:10AE200026AA4946204613F088F82785608D20F031
:10AE3000080161859DF871000C95C10636D520F09A
:10AE40001F000F308DF8710063697399039A1944DC
:10AE50008A4203D120F004008DF87100E26905995F
:10AE6000A2EB0A00814205D19DF8710020F0080094
:10AE70008DF87100A269759804991044814207D138
:10AE80009DF8710000E07FE020F002008DF8710075
:10AE9000226A74980699101A814207D19DF87100B0
:10AEA0004108490061F304008DF8710003A805F022
:10AEB000C7FD07905FEA886008D5606B30F8150021
:10AEC000400503D504990798081A049003AA0AA913
:10AED00072980AF06BF92E987190359870903499A9
:10AEE0000191E06A50F826B06CA805F0B8FD9DF815
:10AEF000E3200199CDE90010029200E051E0DDE984
:10AF00007032594608A817F031FB03A805F0A7FDD9
:10AF10000899401A039900EBD07001EB6000039090
:10AF200003A805F08DFD0999401A049900EBD07033
:10AF300001EB600004900899039808440590099972
:10AF40000498084406905FEA88600FD5606B30F87B
:10AF5000150040050AD50798049900EBD070A1EBC5
:10AF6000600104910699A1EB600006909DF8E40051
:10AF7000CDF8B4B040F040008DF8E40003AA26A953
:10AF80002895729809F0B7FA6D1C761CA06BA84240
:10AF90003FF6EFAE608D20F00800608577B0BDE829
:10AFA000F08F70223BA90AA810F0CCFA542257A9BE
:10AFB00026A810F0C7FA3DE70A0000002DE9F04F7F
:10AFC000F9B005460DF0E0F8044628460DF013F9F7
:10AFD00071900021204612F0B1FB0546002112229B
:10AFE000204612F0DDFC28447790002113222046F1
:10AFF00012F0D6FC00EB050B03A809F0ADFA03AA8A
:10B000004FF40031204612F098FF206B40B181468A
:10B0100094F84C00002700F00F00012807D007E04B
:10B0200080222DA920460CF063FE2DA8EFE7012712
:10B0300020460021272212F0B3FCC0B2012800D123
:10B040000127606B4FF0000800285CD00EF00CFC6C
:10B050008246022818D04DA9606B0EF03BF80128FB
:10B0600022D04FF0FF363546A069691E7390084420
:10B0700075906069711E72900844CDF800807490DC
:10B08000B7B10722779B16E011989DF857206FF013
:10B0900060418DE80700129B0B9A50A8616B17F076
:10B0A00065FADDE95065DFE74E9886B2050CDBE70F
:10B0B000CBF10003082272A904F1140005F02AFB69
:10B0C000BAF1020F49D04DA809F026F94FF4003A21
:10B0D0004DAA5146204612F0D6FE05EBD57042101F
:10B0E00006EBD67041105DA814F0E5FF20466E22F5
:10B0F000514612F055FC5890606B549072AA4DA9BD
:10B10000719809F0B5F818A809F026FA18AA0021D4
:10B11000204612F012FF26989DF8AB206FF0604198
:10B120008DE8070049466FA8279B209A17F01EFA62
:10B1300060696F996B900844401E6D90A06970998A
:10B140006C900844401E6E90606B70B1CDF800802A
:10B1500087B1CBF1000308220EE0606B0A9072AA5F
:10B1600003A9719809F0C7F9CDE700230922CDF8AA
:10B17000008001E0779B07226BA904F1140005F021
:10B18000C9FACDF87C90206B28B99DF8AC0040F04E
:10B1900040008DF8AC006BAA18A9719809F0ABF9C2
:10B1A00079B0BDE8F08F2DE9F04FABB005460CF05B
:10B1B000EBFF044628460DF01EF805461FA9204661
:10B1C00011F0E8FC204602F046FB064603A809F011
:10B1D000C3F9E06A0A90606D1390A06D149094F822
:10B1E0005C0000F00700032808D01FA805F028FC29
:10B1F000B0F5806F02DB04F1380017908DF85760CE
:10B2000003AA0021204612F098FE9DF856004FF048
:10B21000010808B98DF85680606C0C90A06C0D90F8
:10B220000C994FF6FF70814226D00D99814223D0B0
:10B230004FF48029274658224946204612F0B0FB99
:10B2400002464946384614F0BEFB0090BDF80000A7
:10B25000ADF83B009DF802008DF83D0020461C2211
:10B26000494612F09DFB0090BDF80000ADF83E008D
:10B270009DF802008DF8400094F85C006FF0604B80
:10B2800000F00700022801D0032817D19DF85600CE
:10B29000022801D0032811D11199CDE9001B029693
:10B2A000129B0B9A27A8E16A17F060F91FA805F016
:10B2B000D6FB2799884201DA8DF8568005F11802ED
:10B2C0001FA919A805F0DDFB00287ED094F85C00CA
:10B2D000400709D1204611F067FE424200211FA815
:10B2E00005F014FD206A229094F85C0000F007003D
:10B2F00002281BD0032819D01FAA03A9284609F049
:10B30000FAF8D5E907800DF1640C81469CE80F003E
:10B3100005F1180CD5F824A0AF698CE80F0094F85B
:10B320005C0000F00700032818D051E0D5E907823F
:10B330000DF1640C91469CE80F0005F1180CD5F84E
:10B3400024A0AF698CE80F001FAA03A9284609F0C2
:10B35000D2F805F1180080E88007D2E71199CDE90D
:10B36000001B0296129B0B9A29A8E16A17F0FEF8BF
:10B370001FA805F074FB2999884212DA2022114691
:10B380000B980DF052F9616D299A00EB40001144C1
:10B3900008441390A06D14901FAA03A9284609F031
:10B3A000AAF81FA805F04CFB2A99884210DA606DB4
:10B3B00013900B980DF06BF9A16D2A9A1144084473
:10B3C00014901FAA03A9284600E004E009F093F8AE
:10B3D000183585E880072BB0BDE8F08F2DE9F043E4
:10B3E000A7B007460CF0CCFE054638460CF0CCFE64
:10B3F00004464FF480261A2D7DD01D2D7CD1384671
:10B400000CF0F9FE054603A809F0A6F803AA314698
:10B41000204612F092FD22A9204602F0C4FC22AA86
:10B4200005F1180118A805F02CFB002864D020466F
:10B4300002F00EFA8146204612F086FC0646484687
:10B440000EF052FF01461198CDE90006012202924A
:10B4500020A8129B0B9A17F089F8204611F010FCD7
:10B4600007460021204612F0A3FBC268D9F8181045
:10B4700002EBD27201EB6201A269064607EBD778B4
:10B4800002EB68000F1A484611F0FAFBF168401A07
:10B49000002802DDB90391FBF0F70B98A26902EBDB
:10B4A0006801C068219A121A7A4301EBA23100EBBD
:10B4B000D070A1EB60080021204612F042F9074647
:10B4C00020460021122212F06BFA06462046002187
:10B4D000132212F065FA6169F2191144CDE91C18C2
:10B4E000E169081AC01B21991E9008EB01001F900A
:10B4F0009DF8570001E020E01CE040F00100183505
:10B500008DF8570095E8D1000DF1600C80469CE85D
:10B510000F0085E80F004846183D0EF0E5FE0A9042
:10B520001CAA03A9284608F0E6FFC5F818801C35B8
:10B5300085E8D00027B0BDE8F08338460CF05BFE0C
:10B5400005461CA9204602F02EFC68460AF044F885
:10B550006A463146204612F0AEFD1CAA69462846CE
:10B5600009F024FEE6E72DE9F043C7B005460CF0EC
:10B570000BFE044628460CF03EFE814642A92046BA
:10B5800011F008FB05A80AF027F805AA4FF40031CE
:10B59000204612F090FD42AA05A9484609F006FE91
:10B5A000204611F06DFB054604F1140005F057FA32
:10B5B000461BE06A411C05D07043C11700EB1160C7
:10B5C000071208E0204612F027F810F0010F01D012
:10B5D000374600E0002720460021272212F0E0F93C
:10B5E000C0B2012800D1F71B60690090A0690190EA
:10B5F000E0690290206A03900098002D3844009082
:10B6000001DD6D1E00E0002528444FF44037029014
:10B610003946204612F073F906463946204612F0A4
:10B620008CF905463946204612F0B1F98046394674
:10B63000204612F034F901460098019A801B0090D0
:10B64000029828440290A2EB080001900398084455
:10B65000039023A809F0C0FF23AA3946204612F020
:10B660002AFD6A4623A9484609F0A0FD47B0BDE877
:10B67000F0832DE9F04FADF5137D05460CF084FD08
:10B68000044628460CF0B7FD814600F1180204F18B
:10B69000140105A805F0F5F900287ED009F118007D
:10B6A00005AE90E80E00D9F82400CDE90A12CDE9E4
:10B6B0000C3096E82E0009F1180080E80E002046B4
:10B6C00000213022C9F8245012F06AF98B90002131
:10B6D000204612F05FF990900021204612F0E2F827
:10B6E00091900021204612F00DF98F900021204604
:10B6F00012F026F98E90208D002514902585608DFE
:10B7000040F0080161852FA809F066FF4FF4A026DC
:10B710002FAA3146204612F0CEFC6BA808F01CFF81
:10B720006BAA3146204612F008FC14982085608DE3
:10B73000002620F008012046618511F041FC0146F9
:10B74000A26990981044411A8B980E950844401EA7
:10B75000CDE91050204611F02DFC8D90002120469F
:10B7600011F08FFF012800D000208246002092E1D6
:10B77000A16B51F8280011998C90491C401E084477
:10B78000119008980F9181427DDCBAF1000F0BD027
:10B79000E1698E98091A8D9800E08AE1091A8B9860
:10B7A000081A401E0E9008E061698F9801448D9838
:10B7B000091A8B980844401E1090002565E1606BC3
:10B7C0004FF0000B50F8260008B190F800B0BAF125
:10B7D000000F0AD00E98401E1090E06B109950F8A0
:10B7E0002500081A401C0E9009E01098401C0E908D
:10B7F000E06B0E9950F825000844401E1090002779
:10B8000018E0616BF01951F82000C0B10078C00752
:10B8100015D0E9190422E06B02EB8101BAF1000FA7
:10B82000405803D00E99081A0E9002E0109908446F
:10B8300010907F1CE06A7919401E8142E1D3119972
:10B84000069881427CDB0E982B900F982C901098D4
:10B85000CDE92D019DF8050141070BD562698F9B4C
:10B860002B991A44914205DD409A02EBD272A1EB6A
:10B8700062012B9181070DD5A36990992C9A1944E7
:10B880008A4207DD00E00BE1409901EBD171A2EBA8
:10B8900061012C91010710D5E3698E992D9A591AEF
:10B8A000491E8A4209DA409901F0010201EBD17187
:10B8B00002EB61012D9A11442D91C00710D0226A2C
:10B8C00091982E99101A401E814209DA409800F092
:10B8D000010100EBD07001EB60002E9908442E901E
:10B8E000626C0020424554D1216CA94251D1218D76
:10B8F0004A0602D48A0600D520208A0701D540F0E6
:10B9000002004A0701D540F00400090701D540F0C4
:10B910000800F0B32085608D40F0080161854BA8D8
:10B9200009F05AFE16A808F017FE4BAA4FF4A02102
:10B93000204612F0C0FB16AA4FF4A021204600E0DA
:10B9400092E012F0FAFA14982085608D20F0080138
:10B950006185CDE94D85CDE918852BAA4BA94846CF
:10B9600009F024FC606B50F8260000287CD04FF4CE
:10B97000A021204611F0C6FF02904FF4A0212046DE
:10B9800011F0DEFF85904FF4A021204612F002F85E
:10B9900000E033E084904FF4A021204611F082FFB4
:10B9A0000146002000900E9A029810446790109A69
:10B9B0008598101A69900F9A84981044689011988D
:10B9C000401A6A90CBF340005FEA000B01D00120DF
:10B9D000009067A805F043F8009A2499CDE900107B
:10B9E0000292606B259B739A50F8261087A8083145
:10B9F00016F0BCFDBBF1000F0BD01CE070222FA98C
:10BA00004BA80FF09FFD54226BA916A80FF09AFDCA
:10BA10009FE78C980F9A00EBD070889902EB600238
:10BA200001EBD1714010A2EB610200EB61000F99B4
:10BA3000689208446A900EAA05A980A805F021F82A
:10BA400090B10DF5007B09F118009BE80E1080E81D
:10BA50000E00C9F824C0606B67AA16A950F826002A
:10BA600008301D90484600E00BE008F044FD0DF161
:10BA7000140B09F118009BE80E1080E80E00C9F8BD
:10BA800024C03E443D44761C6D1CE06AA8423FF64B
:10BA900096AE08F10100216B804641453FF668AE45
:10BAA0000AAD09F1180495E80F0084E80700C9F809
:10BAB00024300DF5137DBDE8F08F2DE9F0479AB0E5
:10BAC00005460CF061FB044628460CF094FB8246C8
:10BAD000E06A0EF009FC007800284FD1206B0028A6
:10BAE0004CD00078002849D004A808F035FD04AAFD
:10BAF0004FF40021204612F020FA94F8700000075D
:10BB000005D59DF85B0040F001008DF85B00002139
:10BB1000204611F0FAFE81460021204611F013FF65
:10BB200080460021204611F038FF074600212046BC
:10BB300011F0BBFE06460021204611F008FE054626
:10BB400004F11401684604F007FF009809EB0501B1
:10BB500008440090029808EB0501401A02900198F1
:10BB600079190844019003987119401A0390206BC9
:10BB70000B906A4604A9504608F0BDFC1AB0BDE817
:10BB8000F08730B5A5B00C46054620AA1CA911F0D7
:10BB90001DFA1CA804F059FF20B920A804F055FF95
:10BBA00000281CD0694628461BF0BAFF012816D190
:10BBB0001CA804F04AFF30B1002002901CAA69467C
:10BBC000204609F0F3FA20A804F03FFF002806D031
:10BBD0000120029020AA6946204609F0E7FA25B024
:10BBE00030BD2DE9F04F884601F11802B9B0044686
:10BBF00000F1140120A804F044FF00286FD008F1E0
:10BC0000180020AE90E80E00D8F824002991019089
:10BC1000CDE92B2396E82E0008F1180080E80E00ED
:10BC200000212046C8F8245011F05DFE0646002190
:10BC3000204611F0A0FE8146204610F0DEFF28903D
:10BC4000204610F0C9FF259004F12C002A900FF037
:10BC500007FB05460021204611F033FE226F28998C
:10BC6000C2F1010303FB0010B0FBF2FA4FF4A02174
:10BC7000204611F026FE8346C5F1010202FB0BA00F
:10BC8000B0FBF5F7012F00DA01270021204611F063
:10BC900052FD0546204611F0C5F8301A284434906C
:10BCA000204611F081F9A9EB00002844339002A846
:10BCB00009F092FC02AA4FF4A021204612F0FBF9F1
:10BCC0009DF83700099920F007008DF83700FF2014
:10BCD0008DF82800206A00260844319069E075E05C
:10BCE0002899401EA1EB0A017143B1FBF0F1349891
:10BCF0000844616900EB01090020CDE904062A9897
:10BD00000FF0AAFA52E0287CC0074BD194F87400D7
:10BD1000000701D4E96800E000217A1E4A4430920D
:10BD2000CDF8B89007EB0B02484602EB0009209BC8
:10BD3000309A9A4233DB229A904239DC2889ADF856
:10BD40002900A87A8DF82B008819216FDDF894C09E
:10BD5000B0FBF1F201FB1201686850F82120287C49
:10BD6000C0F3001304EB8303586CDB6C121A02FB64
:10BD70000CF2181A92FBF0F0ACEB00023398A369B6
:10BD8000104418442F90686850F821006FF000416B
:10BD9000884204D02EAA02A9404609F007FA049866
:10BDA000401C049029462A980FF068FA0500AAD191
:10BDB000761C206FB04293D8DDE92B2308F11800E0
:10BDC0002999019C80E80E00C8F8244039B0BDE8EC
:10BDD000F08F2DE9F04F01F11802884600F11401AF
:10BDE000CDB0044691460F4644A804F04AFE002810
:10BDF0007DD008F1180144AE91E80D00D8F8241068
:10BE00000990CDE938219A4696E82E0008F11800ED
:10BE100080E80E00C8F82450206F022867D3002164
:10BE2000204611F088FC05460021204611F05BFDFC
:10BE300046190021204611F09EFD0544204610F0D1
:10BE4000DCFE0890204610F0C7FE0690204610F059
:10BE5000E9FF61693144081A3D90204611F0A4F8C9
:10BE6000A1694A462944081A4290394649A804F073
:10BE700008FE00283BD028A808F09FFE28AA4FF40F
:10BE8000A021204612F0B3F80CA809F0A5FB4FF44E
:10BE900000350CAA2946204612F00DF92946204605
:10BEA00011F0CEFE00EBD07046102946204611F06E
:10BEB00060FC00EBD0704110894634984E4500DAA2
:10BEC000314600EBD070B1EB600F05DD9DF8DD0071
:10BED00040F010008DF8DD003498012805D19DF860
:10BEE000DD0040F010008DF8DD00216F00E033E14F
:10BEF0000898814201DB012000E00020439004F11A
:10BF00002C0005460B900FF0ABF9401E2A900E90C6
:10BF100028460FF0BAF913E1287CC00706D02A980A
:10BF2000401E2A900E98401E0E9005E12889ADF81B
:10BF3000CC00A87A8DF8CE002889ADF85100A87AF7
:10BF40008DF8530000202B900F9094F87400000798
:10BF500001D4E86800E000203A903D982F9031909D
:10BF60003A9848906968834651F82000297CC1F3CB
:10BF7000001104EB81020699536CC01A4843D16C3E
:10BF8000C91A90FBF1F00699091A42980027084453
:10BF9000329003900590A5E031982F903298309020
:10BFA000711C2F9A0AEB010082427EDC0898216FF7
:10BFB0007843491EB0FBF1F13D98069B084431904F
:10BFC0003A98226F3844B0FBF2F102FB110B69681A
:10BFD00051F82B00297CC1F3001104EB8102516C54
:10BFE000D26C401A5843511A90FBF1F0191A42983A
:10BFF0000844329009983199801B401E81426EDBC3
:10C00000002F6CD04398A0B36968489851F820205D
:10C010006FF00040824262D051F82B1081425ED016
:10C0200032990598814200DB0846059003988142C9
:10C0300000DC0846039031992F9888424FD03298FF
:10C040003B90481E31902F90039830900598329085
:10C0500032993098884201D1481C329028A9404634
:10C0600008F06FFD3198401C31903B98039005908B
:10C0700035E0FFE72F983099801B3E902F98304491
:10C080004090A1EB09003F9001EB090041906868E6
:10C09000489950F821206FF000418A420CD050F8A6
:10C0A0002B106FF00040814200E01FE004D028A96F
:10C0B00040462B9708F045FD8EB1B9F1000F0ED028
:10C0C0006968489851F820106FF00040814206D00E
:10C0D000781E0F903EAA0CA9404609F067F87F1C15
:10C0E000CDF820B1206FB8423FF656AF4398E8B97B
:10C0F000206FB8421AD169686FF0004051F82B10D8
:10C10000814213D031983299801B3E9031987F1E26
:10C1100030444090A1EB09003F9001EB09000F97DC
:10C1200041903EAA0CA9404609F040F80E98401EE6
:10C130000E902A98401E2A9029460B980FF0A2F8DC
:10C1400005007FF4E9AEDDE9383008F11801099AFD
:10C1500081E80C04C8F824004DB0BDE8F08F000061
:10C160002DE9F04F8A4601F11802C9B0054600F1E9
:10C1700014013CA804F085FC00287DD00AF11801C8
:10C1800033AC91E80D00DAF82410369184E80D0004
:10C190003CAE0AF1180096E81E0080E80E0000216F
:10C1A0002846CAF8244011F0C6FA04460021284661
:10C1B00011F099FB06460021284611F0DCFB0746EA
:10C1C000284610F01AFD4190284610F005FD4090D9
:10C1D000284610F027FE0146686932191044401ABB
:10C1E0004290284610F0E0FE0146AA693819104432
:10C1F000401A43901FA808F0E0FC1FAA4FF4A021AA
:10C20000284611F0F4FE03A809F0E6F94FF40034D3
:10C2100003AA2146284611F04EFF2146284611F078
:10C220000FFD00EBD0704FEA60092146284611F05F
:10C23000A0FA00EBD070401080462B994A46C145C9
:10C2400000DA104601EBD171B0EB610F05DD9DF80E
:10C25000B90040F010008DF8B9002B98012805D1E5
:10C260009DF8B90040F010008DF8B90005F12C00E0
:10C2700037900FF00AF8E8E0EAE0207CC0077DD1B3
:10C280002089ADF8A800A07A8DF8AA002089ADF821
:10C290002D00A07A8DF82F0095F87400000701D4C6
:10C2A000E66800E000264298269044962890606850
:10C2B000B34650F826000A2826D0419800902068FE
:10C2C000002350F82670207CC0F3C00005EB8000EE
:10C2D000C26D416D38460FF0F7F8429900230844CB
:10C2E000289040980090217C6068C1F3001105EB14
:10C2F000810150F82600CA6C496C0FF0E5F84099AE
:10C30000081A4399084401E05448289000262990CF
:10C3100082E028982690299827902A6F0BEB060038
:10C32000B0FBF2F102FB110760686FF0004150F8BA
:10C33000270088427ED040990091217C0023C1F3E0
:10C34000001105EB8101CA6C496C0FF0BDF84099F2
:10C350000023091A43980844299041980090217CB1
:10C360002068C1F3C00105EB810150F82700CA6DB8
:10C37000496D0FF0A9F84299084400E061E0289067
:10C380005EB32699A1EB0900459001EB09002799BE
:10C390004790A1EB0800469001EB080048906168C7
:10C3A000449851F820206FF00040824214D051F898
:10C3B0002710814210D01FA95046229608F0C1FBD9
:10C3C000B9F1000F08D0B8F1000F05D045AA03A9B4
:10C3D0005046069608F0EAFE4497286FB0421AD1FC
:10C3E000606850F827106FF00040814213D0289801
:10C3F00045AAA0EB09004590289803A94844479016
:10C400002998A0EB08004690299806964044489049
:10C41000504608F0CBFE761C286FB0423FF679AF4D
:10C42000219833AF401C21900598401C059097E857
:10C430004D0000E00FE00AF1180181E80D00CAF894
:10C440002460214637980EF01DFF04007FF415AFDD
:10C4500049B0BDE8F08F4497DDE70000010000E03F
:10C460002DE9F84304460BF08FFE804620460BF082
:10C47000D3FE0646C06C4068B0F5A02F62D13046AE
:10C480000BF008FB054630460BF0FDFA044655EA72
:10C49000040057D0F06C00278668072E05DB402289
:10C4A0003146404605F0E8FB28B10DB185F8207013
:10C4B0000CB184F828704FF400423146404605F034
:10C4C000DBFB20B354B1404616F0FAFE0090BDF8F5
:10C4D000000020849DF8020084F8220075B16620D7
:10C4E00085F82000404616F0EBFE0090BDF80000F5
:10C4F000A5F821009DF8020085F82300404605F0CC
:10C50000B9FBB04203D115B1B22085F820004FF439
:10C5100080423146404605F0AFFB002812D0002C87
:10C5200010D0FF2084F828004046203416F0C8FEC2
:10C530000090BDF8000020809DF80200A0706068A7
:10C54000401C6060BDE8F8832DE9F0410F4604000F
:10C5500005D004F1300080460EF07EFE11E0FEE7CB
:10C56000286861680669304605F05CFD05F05EFDEF
:10C5700018B9A269394630469047294640460EF020
:10C580007DFE0500ECD104F1240013F00BFE4046C3
:10C590000EF042FE0020E060BDE8F0812DE9F041A0
:10C5A000174604002DD069B304F12400804613F02F
:10C5B00027FE050027D02E69A269394630469047EC
:10C5C000E16B30468847E168091AE16030466168EE
:10C5D00005F028FD07462869E16A0844294650F815
:10C5E000046C404613F08AFE384605F00DFD3146D6
:10C5F00004F130000EF0FAFE3046BDE8F0410CF0D8
:10C6000051B8FEE7FEE7BDE8F0810879052801D0C2
:10C6100006281ED1C86C826B2ABBC26B1ABBC26AC9
:10C620003AB9036B4FF48072934202D1436B934249
:10C6300001D0012300E00023826E02B101221A42E0
:10C6400011D1008CC0F307201AB10E280BD014288A
:10C6500009D091F85100642805D3642081F8510075
:10C66000012081F850000020704700002DE9FE43B2
:10C670000746407C002690468946082802D30020C1
:10C68000BDE8FE832149002401EB800534E000BFB2
:10C690009DF80000032805D0A878D8B1BDF80400A3
:10C6A000800818E04FF6FF71BDF8022001EA49004A
:10C6B00002EB820208EB880182421BD8BDF80420FD
:10C6C00002EB8202824215D3BDF80600884211D3E4
:10C6D0002046D5E70120C1B2E87818B1BDF80600C0
:10C6E000800800E00120C0B211FB00F029888142DF
:10C6F00000D32646641CE4B26A4621463846F8F761
:10C70000F5FD0028C4D13046BAE70000C8D90508B5
:10C7100010B50446007E400721D42089282820D067
:10C7200029281ED04FF48041206811F053FB0028C7
:10C7300016D0208913381F2813D2DFE800F010121A
:10C7400012121010101010101010101212101212DD
:10C7500012101010101212121210101210000020DD
:10C7600010BD012010BD70B504460DF08DF840B12C
:10C77000207E810701D5012070BDC00701D00020B7
:10C7800070BD2068856805B108350122214628461C
:10C790000BF090FD0128F3D1217E8907F0D42146CA
:10C7A000002010F076F90128EAD1217E8907E7D42C
:10C7B0000022214628460BF07DFD0546012814D1B4
:10C7C000207E800711D4206810F0AAFA06000CD051
:10C7D0002046FFF79DFF40B120462660FFF7C3FFCC
:10C7E0000546012801D1207E8107284670BDC26917
:10C7F00011790B292DD2DFE801F02C060A0E121652
:10C80000241E1A212800D16C08320AF095B8D16C88
:10C81000083209F014BBD16C083209F081BBD16C2D
:10C8200008320AF08FBAD16C08320AF06BBAD16CB8
:10C83000083208F021BFD16C0AF0A3BAD16C0AF01B
:10C8400053BFD16C08320AF087BAD16C08320AF0B3
:10C8500049BD70472DE9FF4F89B00E46DDE916B49A
:10C8600017460021099811F0E8F9054600210998BA
:10C8700010F07CFF0146F07882070BD5C3076FF0FC
:10C88000404202D0954202D006E0914206D120F00B
:10C890000200F070C00701D0714800E07148814685
:10C8A000F078C00712D06F484FF0000AC4F804A017
:10C8B000C4F808A0C4F814A0C4F800A0C4F80CA0E0
:10C8C000C4F810A080463946009798E06448EBE72A
:10C8D0000098B84206D04FF40011284611F07AFAB9
:10C8E00000287DD16049284611F07BFA00287BD1D1
:10C8F0000021284610F02EFF0690A8B36069401C66
:10C900006061A26802EB0B01A160217EC9075AD0C9
:10C9100000EB4000C100206913F036FD079078B1AC
:10C92000606900EB4001079800EBC1004FF0000187
:10C9300040F8185CF078C007284602D0042201E0D5
:10C94000FEE7062211F02CF8616901EB410207991C
:10C9500001EBC20141F8140CF0784FF00001C00760
:10C96000284602D0052201E01EE0072211F018F847
:10C970006169079A01EB410102EBC10141F8100C1A
:10C980006169079A01EB410102EBC101069841F888
:10C99000080C616901EB4102079901EBC20141F802
:10C9A00004AC079820610EE0284649468847F17894
:10C9B000890704D5A1680A180C998A4225DCA26867
:10C9C00058441044A06028464146884701462068E4
:10C9D000814202DD2846414688472060E06801E048
:10C9E00013E001E0401CE060F078400702D54FF012
:10C9F000FF3000E0012000994118009105D409980A
:10CA000010F05DF8051E7FF463AFA068002802DD1A
:10CA1000A0EB0B00A060606908B10C9800E0A06872
:10CA20006060CDB10098B84216D109996A4689680C
:10CA3000096851F82050F078C0F38001099801F09E
:10CA400011F84DB12846414688472060284649469E
:10CA5000884760600120E06000980DB0BDE8F08F6D
:10CA60004FDD010887CC0108010006002DE9F04FD9
:10CA700093B0044600217D2210F092FF9DF817101C
:10CA8000421C62F30001820862F34101C00860F3B6
:10CA900082018DF81710204600217E2210F080FFC1
:10CAA0008DF81400204600217F2210F079FF8DF8C8
:10CAB000150020460021802210F072FF8DF816002C
:10CAC0000021204610F0D1FD012800D00020804632
:10CAD0009DF817004FF00001C00720460CD010F061
:10CAE00038FF81469DF817004FF00001C00720462F
:10CAF00005D010F0E0FE04E010F0DDFEF1E710F0EC
:10CB000028FF07909DF81700C007204602D010F0BC
:10CB100074F801E010F060F8002106900F462046FE
:10CB2000102210F03DFF05463946204610F0FDFD6D
:10CB300006463946204610F0E3FD800700D535440F
:10CB4000A0690544204610F03BFA281A00210890FD
:10CB50000E462046122210F023FF0546314620469D
:10CB600010F0E3FD07463146204610F0C9FD4007AE
:10CB700000D53D4460690544204610F01BFA281A90
:10CB800011909DF817009DF81660C00701D008AD00
:10CB900000E011AD0021204611F04FF81290002165
:10CBA000204610F0E3FD83469DF81700C10708D02A
:10CBB0006FF04042934502D1618D490509D5C10707
:10CBC00008D112996FF04042914203D1618D09055D
:10CBD00000D40026B8F1000F08D0C00706D116B166
:10CBE000012E02D002E0012600E000260027BA460E
:10CBF000109776B39DF81700400703D5A068028D03
:10CC0000521E13E0002211E000200F9009A907989E
:10CC1000CDE9000105A92046069BFFF71BFE099AF6
:10CC200007EB090157180AF1010A0246A068008DB6
:10CC3000904201DD002AE7DABAF1000F01D0A7EB3C
:10CC400009079DF81700C007204603D00FF0C4FF66
:10CC500002E00AE00FF0D1FF10A9CDE90051014632
:10CC600053463A46304617F02BFD9DF81700410712
:10CC700003D5A1680E8D761E00E00026B8F1000FE6
:10CC800004D0C00702D128683844286009AFA068E2
:10CC9000008DB04243DD002E41DB01200F9007984C
:10CCA000CDE90007324605A92046069BFFF7D2FDD5
:10CCB0008246B8F1000F07D09DF81700C00703D1D6
:10CCC00028680999401A286006AB93E8070002AB70
:10CCD000019283E88300119800905346324605A9DB
:10CCE0002046FBF781FB56460D980BF0DBFC00203D
:10CCF0000D90B8F1000F03D09DF81700C00708D0C1
:10CD000028680999109A014402EB09000844286038
:10CD1000BDE7109A296802EB0900081AF7E7129993
:10CD20006FF04040814201D0834502D1204611F08E
:10CD300055FF00223021204612F00BFC13B0BDE855
:10CD4000F08F000070B504461248134E4FF40045B2
:10CD5000032C01D9032414E034B1032C11D0022C8C
:10CD600011D0012C01D009E0012400220821F5F79F
:10CD7000C0F9002229463046F5F7BBF90748047090
:10CD800070BD0122F2E700220821F5F7B2F9012275
:10CD9000F0E700000004024000000240880200208A
:10CDA00070B52DED028BB0EE408A054618EE100AE4
:10CDB00082B00C466FEAD05010F0FF0F2DD0B0EECD
:10CDC000C80A10EE100A2349884201DA9FED228A30
:10CDD000B0EEC80A10EE100AB0F17E5F37DBF9F74B
:10CDE00011FAF9F7D7F9BDEEC00A10EE102A521C5D
:10CDF000042A1BDBB0EE480AF9F7C4FA10EE100A59
:10CE0000F3F791FCCDE9000114A221462846F9F779
:10CE100083F902B0BDEC028B70BD02B02846BDECB8
:10CE2000028B10A2BDE87040F9F776B97AB1C2F171
:10CE3000040600BF18EE100AF3F775FCCDE90001F7
:10CE4000334609A221462846F9F766F9E1E70326A9
:10CE5000F0E700005F70893000000000252E30668A
:10CE6000000000002D2D0000252E2A660000000085
:10CE70002DE9F74F0546007F93464FF0000AC007A3
:10CE800060D14FF00108EC680026C1467CB9287FCC
:10CE9000C0F3C000401E304254D1B9F1000F51D050
:10CEA0000199284688474FF000080446C1460EB94C
:10CEB000261E47D0B8F1000F06D0214628465A4614
:10CEC00090470446B0423DD04FF00108002CDED020
:10CED000206810F0A1FB0006D8D427681FE00121CC
:10CEE000384610F077FFB0B12FB10121384610F06D
:10CEF00071FF0028CAD1E868A04223D0B0B128460B
:10CF000000F0F4FB0246E8681121006812F021FBF2
:10CF1000012817D106E038460FF002FF0746002F20
:10CF2000DDD1E8E7E868006811F053FA2846EC60C4
:10CF300000F0DCFB0246E8681021006812F009FBF3
:10CF4000012802D05046BDE8FE8FE868006811F065
:10CF500040FA296909B1284688470120F3E7000013
:10CF600013B54FF6FF73012269460248F6F7CCFF6E
:10CF700000981CBDAC06002010B5002821D0114B34
:10CF80000022001F196803E0814203D80A4649685D
:10CF90000029F9D152B11368841A9C4204D1006867
:10CFA00018441060104602E0506000E0186039B18B
:10CFB00002680B1A934203D10B681A440260496855
:10CFC000416010BDC803002070B5846C0546002C7C
:10CFD00016D0206820B10BF087FB20680BF062FBB5
:10CFE000E06908B106F0DDFD206A08B106F0D9FD60
:10CFF00060680BF057FB20460BF054FB0020A86440
:10D0000070BD2DE9F0411D46069C164607460CB141
:10D0100000202060002238460BF0ECFC002807D1ED
:10D0200023462A4631463846BDE8F0410BF0FBBBAB
:10D03000BDE8F0810D4810B5442101700C494160F4
:10D040000C4981600C49C160F3F782FF28B90022C6
:10D0500011460648F3F74CFF08B1012010BD034804
:10D060005430F8F7BDF9002010BD0000640800201E
:10D070007DD0000899D00008394302083EB50A2443
:10D080008DE81C000A46014601230248F5F700F925
:10D090003EBD00008C0400203EB50A248DE81C0033
:10D0A0000A46014601230248F5F7F4F93EBD0000A7
:10D0B0008C04002070B588B017F04BF9304C054651
:10D0C000002694F8510008B3606C281AB0F5AF7FC1
:10D0D0001CD9656494F8500003280ED2401C84F8D3
:10D0E000500069462046F8F7F7F80022BDF8001016
:10D0F000A4F15400F4F79CF908E0214884F850604A
:10D100005438F4F776F91E48F8F774F994F8520099
:10D1100048B1A06C281AB0F5117F26D984F8526066
:10D120001AF092FD21E094F8530048B994F83D00BC
:10D1300002281AD1E06C41F28831281A884214D9A9
:10D14000012084F8520084F853606A4607A90C480D
:10D15000E564F8F7C9F817F0FCF8A06408486A46D7
:10D16000BDF81C105438F4F763F9206C281A6428B1
:10D1700003D90120256408B070BD0020FBE7000042
:10D18000B8080020037A41EA432141EA023189B21A
:10D1900041F0800181800846704770B50146C06A41
:10D1A000CA6C12F0060F1AD0C2F34102022A18D03C
:10D1B000012A13D1D1E90E54AC4201DA04F5B4745A
:10D1C0004A6B0E6B1346B24201DA03F5B4722919A9
:10D1D00001EBD17149108E4206DA304470BD496BC3
:10D1E00000E0096B084470BD8A4201DD184470BD3F
:10D1F000084470BD2DE9F34F93B0064669460FF021
:10D200000DFD304610F0A0FD099030460FF038FDBE
:10D2100008900021304610F063FB83460021304621
:10D2200010F07FFB04460021304610F0A1FB0546BC
:10D230000021304610F027FB80460021304610F0D8
:10D240008BFB07460021304610F038FB07F0010148
:10D2500007EBD77201EB620100F0010200EBD07026
:10D2600002EB6000401C491C0D2900DB0D218946A2
:10D270000D2800DB0D2082460D2C00DB0D242746F7
:10D280000D2D00DB0D254046B8F10D0F00DB0D2004
:10D290008046002457E0306B00EB04110EA803F029
:10D2A00049FB0E98009A594658450EDCBBF10D0F0C
:10D2B00000DB0D21511A08440E900F98A8421ADC89
:10D2C00001980D2D05DA294604E0A2EB0A01084475
:10D2D000F2E70D21401A0F9908440F900998109910
:10D2E000C01B801E81420846009924DB08440D2F94
:10D2F00007DA394606E001990246A1EB090010441D
:10D30000EBE70D21084410900898119AA0EB080053
:10D310000199801E8242114411DB4046B8F10D0F85
:10D3200000DB0D200844119000220EA8149903F090
:10D330005EFC58B906E0014401EB0A00E3E701EBAB
:10D340000900F0E7641CB06BA042A4D8B06BA04207
:10D3500001D14FF6FF7415B02046BDE8F08F10F0F4
:10D360000F0000D1012070472DE9F0410E46040066
:10D370002CD066B304F1300080460DF06DFF58B13B
:10D38000006861680569284604F04CFE074622697A
:10D39000314628469047D8B1314604F1240012F0B6
:10D3A0002FFF050017D02969E06A084450F8046C83
:10D3B00040460DF051FF0246314640460DF0E7FF72
:10D3C00061682869BDE8F04104F02CBEFEE7FEE785
:10D3D0003846BDE8F0810020FBE72DE9F0474FF02B
:10D3E000000805461C4616460F464046C3F8008016
:10D3F00006E0E96B226851F82010401C11442160BE
:10D40000B042F6D30021284610F03BF90128284607
:10D4100015D00FF0CFFD2168081A206000212846A2
:10D4200010F070FA216808442060E96B51F826106A
:10D430000844401EA0600020C4F804801FE00FF0E4
:10D44000B9FD216808442060284610F07DFC814623
:10D450000021284610F074FA22680146A9EB020068
:10D46000401AA060E96B51F82610401A2060E2E7EC
:10D47000A96B626851F82010401C11446160B842E9
:10D48000F6D30021284610F085FA616808446060F0
:10D4900028460FF095FD6168081A6060A96B51F885
:10D4A00027100844401EE060BDE8F0872DE9F05FDA
:10D4B000894693468246002110F00CFA0546002169
:10D4C000504610F028FA80460021504610F04AFAE3
:10D4D00004460021504610F0D0F90646504610F0A0
:10D4E00033FC411BA1EB080750460FF0C9FB001BA2
:10D4F000801B8742504605DA10F026FC411BA1EB49
:10D50000080003E00FF0BCFB001B801B00EBD07099
:10D510004010DAF8141042190A44C9F80020021920
:10D52000DAF81810BBF1000F0A44C9F8042001D042
:10D53000CBF80000BDE8F09F0021852210F030BA42
:10D540000021862210F02CBA0021872210F028BA80
:10D55000032901D2012300E00023C01A03EB430397
:10D5600001EB8301891EC1EB41110C23B1FBF3F1E7
:10D5700011446422B0FBF2F2014401EB9001891ADC
:10D580004FF4C872B0FBF2F008440721B0FBF1F28F
:10D5900001FB1200C0B2704710B50446806C002831
:10D5A00004D144200DF07CFF08B1A06410BDFEE75B
:10D5B0002DE9FC47A9B1856900220427688AC0F3D8
:10D5C00008030CE0AE6802EB820456F8240007EB77
:10D5D0008404345B081A844206D8521C92B29342E7
:10D5E000F0D80020BDE8FC8702EB82041221AB6872
:10D5F00001EB84010026595C062702290BD04FF06D
:10D600000C0961B1274A08234FF0100C03290FD0F1
:10D61000012926D043E007EB8401595A3EE009EB8B
:10D62000840107EB840259589A5A085C161836E0B0
:10D63000ADF804000092A8680CEB840103EB8408A9
:10D64000425A50F80810022301A816F02DF930B301
:10D65000A96851F80820801A07EB84024010895A03
:10D660001CE0ADF804000092A8680CEB840103EB09
:10D670008408425A50F80810022301A816F014F941
:10D6800068B1A96807EB840351F80820801A09EBF8
:10D69000840240108A58C95A32F810000E183046D9
:10D6A000A0E7000009CE02082DE9F0410D4604462E
:10D6B00000F0C7F8071E17D0B86900212E1A3846A7
:10D6C00010F070FA0AF0E3FF05460021384610F02A
:10D6D0008DFA00EBD07106EB6101284491FBF0F06C
:10D6E000E16B814200D8481EBDE8F08170B5064666
:10D6F000002528460BE000BF0CF010F90128204659
:10D700000AD00CF0CDF8B04200D1254620460CF0EE
:10D71000CDF80400F0D1284670BD0000FEB5836945
:10D72000806900255B8AC4689B04A06826D4830FA7
:10D7300014D00123B3EB907F2CD1174826688DE8D5
:10D740000700A068042320F04042314601A816F0EB
:10D75000ABF8F8B1801B801061681AE00F482668AA
:10D760008DE80700A068022320F04042314601A85E
:10D7700016F09AF870B1801B4010EDE76368805C8A
:10D78000595C39B130B1637B2268491E11FB03211A
:10D79000401E0D562846FEBDA9F50008BDF500083F
:10D7A0002DE9FC5F0E461D46174682464FF40031B8
:10D7B0000FF046FF00EBD07044103F1B5046FFF7C0
:10D7C000ECFCBAF85C1001EB000909F15A0000B258
:10D7D00016F030F878434FEAE0380FFA89F016F087
:10D7E00029F87843C7134FF440394946504610F0A2
:10D7F00071F883464946504610F08DF8019049462D
:10D80000504610F0AFF800904946504610F035F8F9
:10D81000326820444244A2EB0B01091B29603268A4
:10D820000199424421441144A9607168CA190099C0
:10D83000511A091B6960716839440844E860BDE801
:10D84000FC9FC06A002802D000210FF038B9704751
:10D8500000210FF034B970B590F85C100024C906AF
:10D8600000D501240546002110F0EDF96FF040418C
:10D8700088420CD1002128460FF0BAFF6FF06041BA
:10D88000884204D1688D000501D444F0020420468A
:10D8900070BDB0F5806F01D201207047800A7047DB
:10D8A0002DE9F04104460F46618D00200426C1F3A6
:10D8B00005120FE0E36806EBC0055B59DD0108D5F2
:10D8C00023F07F43BB4204D1E16851F83000BDE84A
:10D8D000F081401C8242EDD84FF0806000EBB12017
:10D8E0004FEAB050608510F47C7F41D0C0F3051042
:10D8F000C100E06812F048FDE060C0B3608DC0F385
:10D9000005156D1E16D06FF003025300E06802EBA0
:10D91000C50141585FEAC11C0CD489010AD403EB4C
:10D92000C50C00EBC50184446D1EDCE9000CC1E9A7
:10D93000000CEBD1E068082100EBC5000DF0E9FE1A
:10D940000C200DF089FDE16841F8350013F0E1FE8F
:10D95000E26806EBC500115841F080711150E26891
:10D9600067F317011150E06850F83500AFE700E0A9
:10D97000FEE7FEE70969C06A0844001F704700001F
:10D980007FB516460A4690F83B5004462946104695
:10D9900006F0CCFA072D25D0082D25D0092D25D04D
:10D9A0000A2D25D00021626AD268A2EB8101B1FB69
:10D9B000F0F4B44200DD34460020134E0090029093
:10D9C00025460190681E03906A463221306905F0B1
:10D9D0002DFC684603F034F8A0420CDD6D1E002DCE
:10D9E000F0DC0AE00221DEE70421DCE71021DAE7BF
:10D9F0004FF48071D7E7002D02DC002004B070BD29
:10DA00000398401CFAE7000094520020491E01D5FB
:10DA1000401E0C310C2901DB401C0C3901290DD0B2
:10DA2000072091FBF0F200FB121000EBD07121F007
:10DA30000101401AC0F11F00C0B2704781070CD12C
:10DA40006421B0FBF1F201FB120149B94FF4C87136
:10DA5000B0FBF1F201FB120010B100201C30EBE72B
:10DA60000120FBE7136821B15B1E13600BD48068B3
:10DA700005E05B1C13608068018D8B4203DA00684F
:10DA800050F823007047002070472DE9FC411546EF
:10DA90000E4604460BF0F8FE0BF040FF01280AD0BA
:10DAA000032808D04FF6FF7005B1286006B130603A
:10DAB0000020BDE8FC810BF0E7FE69460BF002FF99
:10DAC0004FF0000855B320460FF074FA009947183C
:10DAD000002120460FF0D5FD01280BD06069002100
:10DAE0003F1A20460FF00EFF3A1A00204146C5F8B3
:10DAF000008010E0002120460FF022FF0146E0697F
:10DB0000401AC21BF1E7E36B53F8213018448242FC
:10DB100004DB491C2960E36A9942F4D3DEB1204654
:10DB20000FF04EFA01990844A169451A00212046D8
:10DB30000FF030FF2A1A00204146C6F8008007E0A7
:10DB4000A36B53F821301844824204DB491C316036
:10DB5000236B9942F4D30120ABE72DE9FF4F81B04D
:10DB60000546039880081E2800D91F2001278740FA
:10DB70001FFA81F86FEA080080B2009095F82A0039
:10DB800001F47F09C0F3C00A4FF0FF3600244FF0C4
:10DB9000040B1CE0E96801EBC400426892013DD52A
:10DBA000BAF1000F12D10BEBC4028958C1F307413F
:10DBB000090449450AD103685868384206D0DDE9AE
:10DBC0000312184613F081FD01282FD0641C688DC4
:10DBD000C0F30510A042DDD820E0E96851F8340018
:10DBE00042683A4219D00BEBC4028A58C2F307418B
:10DBF0000904494511D11FFA82FA009A1AEA020F64
:10DC00000BD1B24509DDDDE9031213F05EFD0128F9
:10DC100003D15046C24508D00646641C688DC0F347
:10DC20000510A042D9D8002E03DB012005B0BDE8C5
:10DC3000F08F0020FAE72DE9F04742F300061D4679
:10DC40000F4681465408761C15F0EFFDA7EB04083B
:10DC500000FB08F0C711484615F0ECFD00FB08F08A
:10DC6000C011002F06DD803F39120A1B32442144C7
:10DC70002A6005E0803739120A1B2144891B2A607B
:10DC8000A960002806DD80380012011B31442044C1
:10DC9000696005E080300012011B2044801B696030
:10DCA000E860BDE8F087002184220FF079BE2DE9FD
:10DCB000FF4F87B00746DDE917BA0D4609980AF00D
:10DCC000E6FC00EB0B0101EB0A000490FC6A0BEB95
:10DCD0000A006C43A1460025039053E07B6B53F888
:10DCE000241079B3FA6B0092002652F825E04FF029
:10DCF000040C401E0FE0A21953F8222072B11278D2
:10DD0000D2070BD005EB0608009A0CEB8808761CAE
:10DD100052F80880C64472198242ECD30878800712
:10DD200011D509980AF0B3FC00EB0B01049851449B
:10DD3000814206DD09980AF0AAFC00EB0B0101EB19
:10DD40000A0004901CE0DDE915010144AEEB01007E
:10DD50001499CDE9001000220292786B50F824103B
:10DD6000DDE9092305A8083114F000FC06990398A1
:10DD700008440499884200DC084634443544049041
:10DD8000641C6D1CF86A00EB0901A142A6D8049836
:10DD90000BB0BDE8F08F002189220FF001BE0021F9
:10DDA0008A220FF0FDBD2DE9FF410C4606460021F9
:10DDB0000FF0FEFE05464FF4802130460FF0F8FECE
:10DDC000074628460AF063FC054638460AF05FFC21
:10DDD0000746002130460FF00FFF0146781900EB8F
:10DDE000D07001EB600530460EF04AFFB16900EBE0
:10DDF000D07001EB600005EBD571A0EB61006060B5
:10DE00002844E060694630460EF008FF0098206024
:10DE10000298A060BDE8FF81F0B585B00446FFF729
:10DE200017FD06001DD04FF48027394620460FF01D
:10DE3000BFFE0546394620460FF0CCFE044630466C
:10DE40000CF052FA014600206FF06042CDE900026A
:10DE5000029023462A4603A814F088FB039805B0D5
:10DE6000F0BD0020FBE700002DE9F0411E461446FE
:10DE7000054601F47F07FFF770FE012829D08D2C9D
:10DE800002D21848005D05E01748006BA0B1A4F16C
:10DE90008D01405C10F0010F0ED00FB1002700E0A3
:10DEA0006D68EDB1298D3346394322462846FFF788
:10DEB00054FE01280DD0F3E797B9012C01D0022CB4
:10DEC0000ED128680AE0012C05D0C16929B10120D2
:10DED0003160BDE8F0818169F8E700680028F2D17F
:10DEE0000020F6E780DF0508945200202DE9F0417C
:10DEF00004460D46638D00200422C3F305110AE099
:10DF0000E66802EBC007F659B70103D526F07F4655
:10DF1000AE4202D0401C8142F2D8814204D0E16876
:10DF200001EBC000BDE8F0814FF0806000EBB32052
:10DF30004FEAB050608510F47C7F2FD0C0F30510FD
:10DF4000C100E06812F020FAE060608DC0F30510B7
:10DF5000401E0DD06FF00702E16802EBC00601EB36
:10DF6000C0030E44401ED6E90016C3E90016F3D1E3
:10DF70000821E0680DF0CDFB0C200DF06DFAE16892
:10DF8000086013F0C6FBE168486840F00070486024
:10DF9000E16865F317004860E068C3E7FEE72DE934
:10DFA000F041051E05D005F1300006460DF06DF973
:10DFB0000DE0FEE720686968006904F033F8074661
:10DFC00004F034F838B1214630460DF05BF9040016
:10DFD000F0D1BDE8F0813846FBE7000038B50F48C6
:10DFE0000D461446D0F8B0014FF0020190F824001D
:10DFF000C0074FF0120002D011F01AFF01E011F03B
:10E0000037FF2246294604F00DFE0090BDF80000BF
:10E010009DF8021040EA014038BD000094520020F3
:10E020002DE9F0474FF0000CDDE90964089DDDF8AB
:10E030002CA0E1466F1EF1B9052A03D0062A01D0B3
:10E04000042A02D10023012D01D0002107E0012282
:10E050005FF000019C4456F82180491CC444A94249
:10E06000F8D3ACEB0301072A21D2DFE802F0040762
:10E070000B201B130D00C4F8009018E0411A01EBAF
:10E08000D1710CE0411A0BE0411A91FBF7F3C4F88F
:10E0900000900CE0411A91FBF5F303EBD3714910AA
:10E0A000216004E0421A691C92FBF1F32360002115
:10E0B0000BE000BF54F8212056F821C0624404EB65
:10E0C000810C1A44491CCCF80420B942F2D304EB69
:10E0D000850106EB850251F8041C52F8042C11440A
:10E0E00022688A1ABAF1000F0DD0002109E000BFA2
:10E0F00054F8213056F82170C31ADB1B44F8213044
:10E10000491CA942F4D31046BDE8F0872DE9F0413F
:10E110008CB004466946F9F78BFD08A8102200214F
:10E120000DF0CBFA00210E46204612220FF038FCEB
:10E130000546314620460FF0F5FA0746314620469F
:10E140000FF0D8FA400700D53D4400212E460F4677
:10E15000204610220FF024FC0546394620460FF0D9
:10E16000E1FA8046394620460FF0C4FA800700D510
:10E17000454420460EF01EFF61693144081A0A909A
:10E1800020460EF01DFFA1692944081A00250B90B6
:10E1900007E0006808AA694650F8250001F060F819
:10E1A0006D1CA068018DA942F3D800980AF07AFA94
:10E1B00001980AF077FA02980AF074FA03980AF0C4
:10E1C00071FA002120460FF035FD0546002120465A
:10E1D0000FF0C9FA6FF040418D4201D0884202D160
:10E1E000204610F0FBFC00223021204611F0B1F94E
:10E1F0000CB0BDE8F081000070B504462E4E8AB028
:10E2000080074FF0000506D53046F7F7F3F886F89B
:10E2100054500AB070BDE00723D027488DF8045051
:10E220008DF800506A4601A95438F2F775FE22486D
:10E23000F7F7E0F89DF804109DF80000012219B1ED
:10E2400068B986F8542005E048B141B9014602207A
:10E2500086F85400012902D986F8512001E019F00E
:10E26000F3FC600713D514488DF81C506A4608A9C2
:10E270005438F2F75BFE07AB6A46BDF820100E4833
:10E28000F7F774F89DF81C0008B100F017F82007A4
:10E29000BFD5042016F050F86A4607A90648F7F7DC
:10E2A000B1F80028B5D004486A46BDF81C105438AF
:10E2B000F3F7BEF8ADE70000B8080020FEB507464A
:10E2C000254CC0074FF001064FF000050AD084F836
:10E2D000515084F8505084F85260483416F039F8A0
:10E2E00044F84809380704D594F8520008B184F876
:10E2F0005250B80726D594F831106A461648F6F7FA
:10E30000F5FF84F852509DF8000003280AD0124807
:10E3100001215438F2F728FFBDF80620BDF804109B
:10E32000012016E00C4800215438F2F71DFF218F20
:10E3300049B194F83A20002307483834F7F76CF8CD
:10E340002580E676FEBD16F004F8E064227B618944
:10E35000022019F07DFFFEBDB8080020704711684B
:10E36000090C41731168090E81731179C173918889
:10E37000090A0174002B03D0187840F010001870BF
:10E380007047002B03D0187840F0040018707047D5
:10E390007047017A491CC9B2072900D900210172CE
:10E3A00070477047002B03D0187840F002001870B7
:10E3B0007047002B03D0187840F0020018707047A7
:10E3C000F8B504461D461646684616F06CF99DF8E9
:10E3D000030084F83000002107E000BF56F8210058
:10E3E00004EB8102491CC9B250619DF803008842C8
:10E3F000F4D8227B61892046FEF738F984F8310091
:10E40000002D03D0287840F001002870F8BD704737
:10E4100070B5054C0025206D18B10EF031F825655A
:10E420006565257070BD0000CC0000202DE9F04727
:10E430000446C06A4FF4404103F061F994F9361084
:10E44000A08E0122FFF784F80546A06B08B30026D2
:10E450004FF002084FF00309AF1D4FF4004A15E0DA
:10E46000A06BA28E30F8261091420ED108EB8601E7
:10E47000425694F936108A4207D109EB860140567C
:10E480005246C119E06A03F003FC761CE06BB0420F
:10E49000E6D8A08E218E884210D194F9360094F9E6
:10E4A000321088420AD194F93300AD1D4119E06A57
:10E4B000BDE8F0474FF4804203F0EABBBDE8F087C7
:10E4C00010B502464B68127A097A40684FF0FF3463
:10E4D0008A4215D1012A01D05AB10EE0194613F033
:10E4E0009FF8002809D002DD4FF0010010BD204642
:10E4F00010BD984201D0FAD9F6E74FF0000010BDE8
:10E50000F5D9F1E770B5C56804461021284605F035
:10E51000ECFB10B1284605F044FB207A012804D119
:10E520006068BDE870400AF0BDB870BD2DE9F04FDD
:10E530000C46804687B00C2120460DF0FAF898F87A
:10E540001060D8F80C7016B93869002824D00AF089
:10E55000C7FFDFF818A15FEA000908F1140B1ED00D
:10E56000012E26D18DF80460009700226946DAF862
:10E57000200103F0C7FC050013D003F04EFD00F1AD
:10E5800008010EC984E80E00446900222946DAF821
:10E59000200103F072FD204607B0BDE8F08F012E88
:10E5A00007D10222394658460AF0F2F808B1002095
:10E5B000F2E72F4800900CF04FFE13E0286868B196
:10E5C000686858B10022114658460AF013FA2B68C1
:10E5D0002246414628469847012808D029460098F7
:10E5E0000CF04CFE0500E9D1012E16D018E0208970
:10E5F0000004000CF8D12088C0F30720142808D0AC
:10E6000004F0C4FAA18889B24843C01DC008208123
:10E61000EAE7A0880004C00BF9E758460AF064F85E
:10E62000B9F1000F1CD0012E1AD1CDB18DF80460C4
:10E63000384613F00BF80595009094E8070002ABFC
:10E64000544683E8070000226946DAF8200103F007
:10E650007EFC010006D00022D4F8200103F00DFD5D
:10E66000284699E700980AF01DF8A0E79452002088
:10E67000A453002010B502460B681279097900688E
:10E680004FF0FF348A4215D1012A01D05AB10EE071
:10E69000194612F0C5FF002809D002DD4FF0010035
:10E6A00010BD204610BD984201D0FAD9F6E74FF0D0
:10E6B000000010BDF5D9F1E70179012902D1006808
:10E6C00009F0F0BF704700002DE9F04F95B0834688
:10E6D0001EA8894690E84005B1F84810ADF818101A
:10E6E00099F84A008DF81A00106B0790506B08904B
:10E6F000244DD06A1C46174660B114B12068A84268
:10E7000008D1CDE9006806AB49465846D04715B058
:10E71000BDE8F08F98E80F000DF1080C8CE80F00B1
:10E72000706842423068414202A802F0EFFA04B930
:10E730000DAC25606560A560E560224602A93846FB
:10E740000AF0BAFC054694E80F000DF1240C8CE8A1
:10E750000F00D6E9001209A802F0D8FA012DD6D18F
:10E7600009AA414611A802F08CF90028E5D011A9A8
:10E7700009A8CDE9000106AB3A4649465846D047BC
:10E78000DBE70000010000E02DE9FF4FADB0C86AF3
:10E79000DDE93A970E4638B9316B4FF4807081420B
:10E7A00002D1716B814201D0012000E000201A905B
:10E7B000B06E08B1012500E00025D46A2C220021AA
:10E7C0002069169020891FFA80FA2088C0F3072B51
:10E7D00007A80CF072FF96F84C008DF8300096F800
:10E7E0004D00CDF824A000F00F008DF844001A98D9
:10E7F000284357D1BBF10E0F0ED096F84B00BBF15A
:10E80000140F24D002284DD81698CDF82C90CDE9BD
:10E8100007908DF828B03EE02D98494682686846FA
:10E8200002F02FF900283AD016980D900020089099
:10E83000CDE90F9A36F8480FADF83100B0788DF871
:10E84000330002208DF83800CDF81C9023E0022818
:10E8500028D8484602F0F4F80546484602F0FFF88A
:10E86000169908910D91CDF82C900AFB00F1A08823
:10E87000CDF81C9080B2B1FBF0F00D9900FB0510B3
:10E880000D904FEA5A00CDE90F9002208DF8380024
:10E8900012208DF8280007A92D9807F0DCF831B078
:10E8A000BDE8F08F1A9885434BD096F84B000228AC
:10E8B00047D8002219A8B16E0AF036FC0746012895
:10E8C0002ED1249860B30088C0F307200E2801D011
:10E8D000062825D1249D28690D90288980B21090A2
:10E8E00006F15400044602F0BAF8002800DA4C465B
:10E8F00068680022010C491E83B20091114602A8EB
:10E900005B1E02F010FA002003460090092202A9C3
:10E91000204601F0FFFE02A80F9002208DF838007B
:10E920001698CDF82C90CDE907908DF828B007A95E
:10E930002D9807F090F8012FB1D119A80AF094FB97
:10E94000ADE797E80F0020AC84E80F0020A80790FF
:10E95000484602F084F81790484602F071F8069095
:10E9600020A802F07CF8054620A802F069F880464D
:10E970005C46BBF1060F04D196F84B00022800D983
:10E9800010241A9838B10F2C0CD0112C0AD0122C4C
:10E990000AD0062C25D0204604F015F91990142C25
:10E9A00007D023E010241DE01424204604F00BF9C6
:10E9B000199005EB4500009011F024FD04F01CFBBC
:10E9C000870011F01FFD04F0FDFA04F0FCF8474346
:10E9D0000098B7FBF0F74046474500DD0746009832
:10E9E0001DE01524204604F0EEF81990204604F0AE
:10E9F000EAF86843039011F005FD04F0FDFA870082
:10EA000011F000FD04F0DEFA04F0DDF8474303984E
:10EA1000B7FBF0F74046474500DD074603987843CB
:10EA20000CF01AFD1590A8B108908DF82840239895
:10EA30001F90781E219926900844239020A80B90BF
:10EA4000142C08D00E2C17D0204604F0BCF86843D4
:10EA5000099086E1FEE769000991159A05FB07F127
:10EA600002EB41010D91CDE90F0502208DF8380030
:10EA700012208DF8280074E108990D91CDE90F0559
:10EA800002208DF83800B6F84800ADF8310096F84D
:10EA90004A008DF833000020089062E12098CDE90B
:10EAA0001B0122981D9023981E90D9F80400424221
:10EAB000D9F8000041421BA802F028F91A9878B151
:10EAC000159A3098CDE904B2CDE902600699CDE9F6
:10EAD000001ADDE916231BA92D9808F0BBFC9EE067
:10EAE00096F84B0002287CD31BA801F0A9FF07462B
:10EAF000BBF1060F16D0142C3DD00E2C3AD01C982A
:10EB00001B9A199900FB0AF002FB010116984FF0BD
:10EB100000080844149015981999019005FB01F01C
:10EB200003907AE0DDE91B120AFB021116984FF000
:10EB3000000E01444FF0FF08159A19E0002010E084
:10EB400002EB800311F800C083F802C011F800C086
:10EB500083F801C011F800C002F820C083F80380D8
:10EB6000401CA842ECDB02EB850251440EF1010E81
:10EB7000BE45E3DB53E04FEA5A011C98019148433C
:10EB800016991C9A01EB40011B984FF0000801EB0D
:10EB900040010291019901FB020206984143169837
:10EBA00000EB410010440590159803900D980490D7
:10EBB000680027901EE000BFDDE90210279A0CF0E4
:10EBC000C1FCDDE904012A460CF0BCFCDDE90110C2
:10EBD00000EB4100029005990198084405900398C4
:10EBE00000E084E000EB45000390049808F1010880
:10EBF00028440490B845DFDB11E0039A149901988A
:10EC00000CF0A0FC0199199808F1010805FB00100F
:10EC10001499019001EB0A001490B845EDDB96F8C9
:10EC20004B00022863D9B16C8046C0F1FF07019107
:10EC3000142C1ED0122C1CD00E2C7AD020A801F03F
:10EC400004FF01460198C2B212FB08F3C0F3072289
:10EC500012FB08F003900198C0F3074212FB08F280
:10EC6000DDF864C0002001FB0CF1DDF854E00591F3
:10EC70005DE0C1F3C40111FB08F014900198C0F3EA
:10EC80000720810811FB08F005900198C0F30740A8
:10EC9000C10811FB08F001901598009020A801F020
:10ECA000D4FE864600204FF4FC621EE0DDE900132E
:10ECB00031F810804FEAD82111FB07314FF4784327
:10ECC00003EAC10C059BC8F3451111FB073102EAA9
:10ECD000D1018C44149B08F01F0111FB0731009BEC
:10ECE0000CEB112123F81010401C7045DEDB20E0F6
:10ECF0001EF8001011FB07314FEA112C0EF800C06E
:10ED00000EEB0001DDF80CC091F8018018FB07CC78
:10ED10004FEA1C2C81F801C091F802C01CFB072CA3
:10ED20004FEA1C2C81F802C01999084405998142C8
:10ED3000DED807A92D9806F08EFE2398401C21905E
:10ED4000269908441F99239088420ADD2391142CA8
:10ED500007D120A801F074FE1599684301EB40002B
:10ED60000D9021991F9881427FF798AE159809F070
:10ED700099FC94E52DE9F0410446807A0D4640F077
:10ED80000200A0721E480026016DA14200D1466516
:10ED90002078012801D002282FD115B1606FA84238
:10EDA00001D1666715B1A06EA8420DD1A76E57B10B
:10EDB000224614213846A66610F0CBFB3A461421B1
:10EDC00020460AF0D3FD15B1E06EA84201D1E666F7
:10EDD00015B1206FA8420CD1206F48B122461421F2
:10EDE000266710F0B6FB3246142120460AF0BEFD1D
:10EDF00015B1A06FA84200D1A667BDE8F081000060
:10EE0000945200202DE9F041044690F83C0000F0B7
:10EE1000030001283CD1E16AA06BB1FBF0F0216B4B
:10EE2000B1FBF0F200FB1211A26B520802FB0011C1
:10EE3000B1FBF0F2216300FB1211A26B520802FB3E
:10EE400000116163204600210EF0B2FE054600214C
:10EE500020460EF0D1FE0746284609F018FC05466C
:10EE600020460DF0B9FE06462046FEF7F1FC0246AC
:10EE7000216BE819414306EBD67305EBD570BDE86D
:10EE8000F0415B10A3EB6000411A104610F085BD05
:10EE9000BDE8F08110B504460069B0B1A069A8B121
:10EEA0006068A0B103F0C6F8021D04F124002169D6
:10EEB00011F0BDF9002807D0042104F130000CF056
:10EEC000E8F90348E063012010BDFEE7FEE7FEE736
:10EED000A58A000810B504460069B0B1A069A8B1C0
:10EEE0006068A0B103F0A6F8021D04F124002169B6
:10EEF00011F09DF9002807D0042104F130000CF036
:10EF0000C8F90348E063012010BDFEE7FEE7FEE715
:10EF1000D181020870B50D4C064600200D460A4608
:10EF200020602121304610F014FB206858B1017890
:10EF300039B1294612F074FB28B13046216813F02C
:10EF4000B9FD002070BD012070BD00001803002035
:10EF50002DE9F0418CB01F4614460D4606460FF0D1
:10EF6000B1FA002839D0A54237D04FF4B4708542A9
:10EF700001DDA5F5B475844201DDA4F5B474F16A30
:10EF80000D440C44854201DDA5F5B475844201DDD4
:10EF9000A4F5B4740AAA04A93046FEF787FA3946E4
:10EFA00030460EF04DFB80463046394651220EF079
:10EFB000F7FC06A908B1012200E00022CDE90048D3
:10EFC000CDE902210A982B4682B2DDE9040104F062
:10EFD00077FA06A930460FF017FA0CB0BDE8F081B9
:10EFE00010B588B0044606AA04A9FEF75FFA6B467E
:10EFF00004A92046069AFEF7D3FB204600F0E8FA63
:10F00000011E03DD0246684601F02EFD69462046DA
:10F010000FF0FAF908B010BDF0B50646A1F57F4033
:10F020008DB00F46FF384DD0B06BB8424AD9306B27
:10F0300000EB071102A801F07DFC06A930460DF097
:10F04000EDFD002130460EF087FC044600213046DD
:10F050000EF034FC054630460DF0E6FD03F0C2FF2D
:10F060000A2190FBF1F2A24201DB90FBF1F490FB4C
:10F07000F1F2AA4201DB90FBF1F506980299021B1E
:10F0800011440291079A0399521B11440391049968
:10F0900008442044049007990598084428440590A2
:10F0A000306CB8420AD1706B30F81700400505D5B6
:10F0B00002A801F0C5FC0399081A039002A9304682
:10F0C0000FF0A2F90DB0F0BD2DE9FF470446006F27
:10F0D0000D46A84274D920460DF08FFD804620468B
:10F0E0000DF0A0FE064694F87400010705D500F067
:10F0F0000700012807D0022863D004B02046BDE8ED
:10F10000F0470FF066B9002120460EF014FB0746C9
:10F11000002120460EF0E7FB616938440844A0EB6B
:10F12000060920464FF4A02148220EF039FC06467D
:10F130004FF4003120460EF083FD074660690090D1
:10F14000A0690190E0690290206A03900199F0198A
:10F15000091A0191039908440390206F401EA842A8
:10F1600016D908FB05F1B1FBF0F202EB0901891B8E
:10F17000C91B6A1C009108FB02F1B1FBF0F101EB25
:10F180000900304438440290694620460FF03CF9AB
:10F19000002D3FD0681E08FB00F1206F401EB1FB20
:10F1A000F0F202EB0901891BC91B009108FB05F174
:10F1B000B1FBF0F101EB090030443844029025E046
:10F1C00028E0002120460EF07CFB8146206F08EBF2
:10F1D0000901B1FBF0F7002120460EF0ACFA82469F
:10F1E00007FB05F8002120460EF07DFB61695044C5
:10F1F00041444518694620460DF010FDA81B0090BB
:10F20000384400990290A1EB09000090694620461D
:10F210000FF0FAF8BDE8FF87044890F83D00022897
:10F2200001D000207047012070470000B80800207E
:10F2300070B505460EF088FD044628460DF020FD09
:10F24000844201DB012070BD002070BD28B10A2876
:10F2500003D00D2801D00020704701207047000026
:10F260002DE9F74F0D4686B00446CD490EF0B9FDA5
:10F2700000287CD12046FEF767F982462046FEF73B
:10F280008EFD5FEA000972D0BAF1000F6FD0204600
:10F29000FEF756F907462046FEF77DFD80462046DC
:10F2A000002188220EF07CFBC6B2204600218B2272
:10F2B0000EF076FBC0B20390296807EB0A006FF0EE
:10F2C000030303EB8000D5F808C051F82720095844
:10F2D0005CF800000844A0EB020B6A6808EB090028
:10F2E00003EB8000EB6852F82810125818581044AD
:10F2F000401A0290002120460EF0B1F9012806D1F3
:10F3000016B1022E02D002E0022600E0002604F12F
:10F310001400019001F0A3FB0090019801F090FB14
:10F320008246012E38D0022E4FD0032E4FF000011E
:10F33000204606D00EF041FA296851F827100844FB
:10F3400051E00EF03AFA296851F8271000EB010954
:10F35000002120460EF031FA0646002120460EF02C
:10F3600035FA3044ABEB00000090608D00E014E112
:10F3700040F400606085039801287CD002287BD08F
:10F3800003284FF00001204632D00EF028FA6A68B8
:10F3900052F828104718B8E000992046ABEB010955
:10F3A00000210EF00AFA0646002120460EF00EFA61
:10F3B0002968301A00EBD07051F8272009EBD97179
:10F3C000491001EB600010440DE020460EF0BCFC3B
:10F3D000296851F8272002EB0B010E1A0021204664
:10F3E0000EF0F4F9301A8146608D20F40060C1E718
:10F3F0000EF0F5F96A6852F82810471800212046E7
:10F400000EF0EDF90546002120460EF0CDF90299E7
:10F410002844A1EB000A608D40F48060608520469E
:10F420000EF092FC0099884204D120460DF028FC91
:10F43000504524D060690290A0690390E06904906F
:10F44000206A059020460EF0C4FFDDE9001001F0AF
:10F4500074FC5146019801F06BFC20460EF0B9FF98
:10F4600002AA2E21204610F074F820460DF058FC18
:10F470002246272101E021E039E010F06AF8204619
:10F4800000216A220EF08CFA0646204600216B22EB
:10F490000EF086FA054620460EF056FC82462046BF
:10F4A0000DF0EEFB3F4A0146C6F3417053104FF09A
:10F4B00080584FF0640C01282BD035E002980021D1
:10F4C000A0EB0A0620460EF08AF9074600212046E6
:10F4D0000EF06AF96A68381A00EBD07052F82810FA
:10F4E00006EBD672521002EB60000F180DE02046BA
:10F4F0000DF0C6FB6A68029952F8282011440D1AD3
:10F50000002120460EF050F92F1A608D20F4806003
:10F5100084E726F0C040904206DC404500DB181A24
:10F5200000FB0AF090FBFCF6C5F34170012809D1FD
:10F5300025F0C040904205DC404500DB181A4843E6
:10F5400090FBFCF5089A09EB0601781992681144C2
:10F5500062698D1A0899C9680844A169461A55EA72
:10F5600006001AD020460EF034FF6069284460611E
:10F57000E0692844E061A0693044A061206A304419
:10F58000206220460EF025FF09B03246294620466B
:10F59000BDE8F04F00230EF0C5BF09B0BDE8F08F05
:10F5A00001000600FEFFFF1F0A880368934201D096
:10F5B000981A704740684988401A70470A7803686B
:10F5C000934201D0981A704740684978401A7047B2
:10F5D0002DE9F0414FF4403604463C2231460EF00E
:10F5E000DFF905462046422231460EF0D9F905449E
:10F5F000314620460EF0EFF900283146204602DD64
:10F600000EF0E9F902E00EF0E6F940420544314619
:10F6100020460EF0E6F900283146204602DD0EF0C5
:10F62000E0F902E00EF0DDF94042054420463822C0
:10F6300031460EF0B5F9074620463B2231460EF022
:10F64000AFF93844854200DD2846BDE8F08170B549
:10F65000054608F095FD0446284608F095FD064647
:10F660000DF05EFB05462F2C01D02E2C0BD1002176
:10F6700030460BF0FFF9284616F072F82846BDE830
:10F68000704018F0A7BD70BD2DE9F0438DB007465E
:10F690001D46164689460846DDF850800DF0E6FA0C
:10F6A0000446414648460DF0B9FA22461146404606
:10F6B00001F0DAF907F11804022E05D0012E32D03C
:10F6C00000200DB0BDE8F08398E80E00D8F80C00DB
:10F6D00003908DE80E000022694648460EF0BCFA01
:10F6E0006A46214604A801F0CCF90028E9D004AC10
:10F6F00094E80F0008AC84E80F00022208A94846ED
:10F700000EF0AAFA08A94246084601F0BAF9002804
:10F71000D7D094E80F0085E80F000522114628464F
:10F7200001F0A2F90AE042462146684601F0A9F933
:10F730000028C6D09DE80F0085E80F000120C0E733
:10F74000F8B504460E46001D01F07AF90546201D65
:10F7500001F085F900960246217D2B46206804F0D1
:10F76000C0FB002800D1FEE7F8BD70B504460DF0DF
:10F77000E5F90646002506E0A068006850F8250077
:10F78000FFF7F3FF6D1CB542F6D3608DC1070CD0B7
:10F7900020F00100608520460FF020FA20460FF08F
:10F7A00049F916B120460BF0E3F9608D810708D5C1
:10F7B00020F0020060852046BDE8704000210EF078
:10F7C000A0BF70BD2DE9F0478046089D1F46A86A7E
:10F7D00000FB01F39B12002807DD934207DD00BF09
:10F7E00095F8340080070DD48BE09342F8DBCB19F9
:10F7F00043439B12002808DD934239DA95F8340020
:10F8000080077ED40120BDE8F0879342F6DC686A69
:10F81000521C504340F395000312C0B2FF2200284F
:10F8200028D000BF2E6BC0F1FF0404FB06F4A2EB4E
:10F83000242600BFA3EB0104A14636D0002C15DB23
:10F84000BC4213DAC0F1FF00C6F1FF014843A2EB4E
:10F850006020C1B295F83400800701D5C1F1FF01E5
:10F8600018F8040014F04EFB08F80400641C1CE0B7
:10F87000686ACEE74FF0FF06DCE7002C10DBBC42E5
:10F880000EDAA6EB6000C1B295F83400800701D50E
:10F89000C1F1FF0118F8040014F034FB08F804006B
:10F8A000286B641C361ABC4202DA286BB042E4DBD7
:10F8B000BC4218DA002C16DB686A70438012704371
:10F8C000C0F34721A86A002801DAC1F1FF0195F8C9
:10F8D0003400800701D5C1F1FF0118F8040014F0CD
:10F8E00011FB08F8040095F83400800707D5494655
:10F8F000B94506DC00290DDB404609E001E0641C47
:10F9000001D500207FE7BC4204DC391B08EB040072
:10F910000BF017FF022076E72DE9F05F06460A9FFD
:10F920008A461D46786A00FB02F18C12002800DD31
:10F93000641C97F83430544502DA980707D4D5E0B0
:10F940008C120AEB050CA44502DA98077ED483E0FA
:10F95000521C424341F3950142F395044FEA212999
:10F96000221204F0FF08C9B2A9EB0A04914505D0A0
:10F97000002803DA11B9FF219146641E914528D170
:10F98000002C0CDBAC420ADA01EB080041089807B6
:10F9900001D5C1F1FF01305D14F0B4FA305597F88C
:10F9A0003400641C800706D5A9EB0A01A9424DDA90
:10F9B0008EE030460AE0AC4200DD2C46002C45D0FB
:10F9C00006DD00BFA5EB040106EB04000BF0B9FE59
:10F9D00089E04FF0FF0B002844DAB86A4042484300
:10F9E0004FEAA028002C0DDBAC420BDA08FB01F03B
:10F9F000C0F34721980701D5C1F1FF01305D14F034
:10FA000081FA3055796AA8F1FF0041438812641EDB
:10FA100011D4AC420FDAC8F1FF014143ABEB6120D6
:10FA2000C1B297F83400800701D5C1F1FF01305D04
:10FA300014F068FA305597F83400A41C800709D5F3
:10FA4000A9EB0A01491EA9424DDC00E04EE0002965
:10FA5000AFDC48E0AC4202DD0120BDE8F09F002CA5
:10FA6000B0DA40E0C1F1FF00B96A41434FEAA12892
:10FA7000002C0EDBAC420CDA00FB08F0ABEB602094
:10FA8000C1B2980701D5C1F1FF01305D14F03AFA17
:10FA90003055796AC8F1FF0041438912641C0ED4C5
:10FAA000AC420CDA4843C0F3472197F83400800792
:10FAB00001D5C1F1FF01305D14F024FA305597F8FB
:10FAC0003400641C800707D5A9EB0A01A9420DDCAC
:10FAD0000029BFF66EAF06E0AC4200DD2C46002CDC
:10FAE00004D03FF76FAF4FF00200B6E74FF00000D1
:10FAF000B3E7FEB5C46A09F0C7FE054609F00EFF7C
:10FB000004280CD1216C204661640DF0B4F806463F
:10FB100009F0DAF818B10021304609F04AF9284610
:10FB200009F0FCFE012804D0284609F0F7FE03285E
:10FB300009D16946284609F0C5FE20460199FDF71E
:10FB4000B3FD20646064204607F0B2FF206B10B95B
:10FB500020460EF03EFC206C029002AA2021204696
:10FB60000FF0F7FCFEBD000010B5582109480BF05E
:10FB700090FB00222121084813F01AFC054CAC3CF4
:10FB8000C4F8A800A434F7F779FD00202070607055
:10FB900010BD000040530020AD7600082DE9F04173
:10FBA00005460F480E460024074616E00168A942A4
:10FBB00000D01DB94168B14209D046B1014638466E
:10FBC0000BF05CFB0028F1D12046BDE8F08116F077
:10FBD000FBFAF7F753FD012438460BF03DFBF1E744
:10FBE0004053002070B505460A480C4606460BF007
:10FBF00033FB0BE00168A94204D14168A14207D060
:10FC0000002C05D0014630460BF038FB0028F1D11E
:10FC100070BD00004053002010B50446582200215A
:10FC20000BF04BFD4FF4FA702063002060626420FB
:10FC3000E062012060640448206294F8540040F0BF
:10FC4000080084F8540010BDE5FC00082DE9F843D5
:10FC500004464FF48060174600901E46D4E90C20FD
:10FC600088460023089D19460BF02EFC33463A4681
:10FC70004146009503F046F8626AE16A891A4143F9
:10FC800002EBA120BDE8F88308B5B0F94E20009240
:10FC9000B0F94C30B0F94A20B0F94810FFF7D6FF60
:10FCA00008BD08B54FF4806300224FF4D77100936C
:10FCB000FFF7CCFF08BD08B54FF48061009140F21A
:10FCC000512300224FF4D771FFF7C0FF08BD08B5DC
:10FCD0004FF480610022009140F251231146FFF75A
:10FCE000B5FF08BD38B504464FF480600090D4E9F4
:10FCF0000C20002319460BF0E7FB626AE16A891ABF
:10FD0000414302EBA12038BDD0E90C128A4201DB4D
:10FD1000C06A7047406A70470020F7F7C7BC10B54B
:10FD2000029C20F8481F83804280C48010BD01617E
:10FD300070474942416370474161704701637047B2
:10FD400010F8542F61F3C30202707047416070478E
:10FD50000162704781637047C1637047C163704738
:10FD60004164704701647047C16070470163704728
:10FD7000C161704741624FF00041C0E90A1270470B
:10FD80000160704710B542F2107442F2F673A0425F
:10FD900000D91846A14200D91946A24200D91A46F4
:10FDA0000A23401D491D521DB2FBF3F2B1FBF3F1D2
:10FDB000B0FBF3F0120502EB8121084400F1004092
:10FDC00010BD000070B5054620480BF06AFA04002B
:10FDD00028D0582229460BF0B5FB2868A84200D14C
:10FDE00024601A48AC3890F8A51014F8540F61F349
:10FDF000410004F8040913F085FA01C414F8540909
:10FE000000071FD5A16939B120468847616A0144BE
:10FE10006162E16A0844E062204616F0F3FA68681D
:10FE200018B900E0FEE7A86810B1204616F00AFAFB
:10FE3000626812B1616A20689047A26812B12046D8
:10FE4000616A9047F7F71AFC204670BD40530020C6
:10FE500010B5D0E90E431B1B02E000BF03F5B473DD
:10FE6000002BFBDB4FF4B474A34202DBA3F5B473A5
:10FE7000FAE799420FDC03EBD372B1EB620FC16C6E
:10FE800002DA41F0080101E021F00801C0F84C104D
:10FE900041F0100117E0C3F5B474944203DCC16C67
:10FEA00041F00801F4E7C1F5B474944203DCC16C7D
:10FEB00041F0080105E01A448A4207DBC16C21F0D9
:10FEC000080121F01001C164012010BD002010BD07
:10FED00010B50C4687212D22C4E90E120020C4E97A
:10FEE0000B0149006163E16C21F00601E1641349F3
:10FEF0002164E16C606441F008016420C4E91201EE
:10FF000021F00100E0641001206513F0FBF9606549
:10FF1000606BA065E06C022120F01000E0642046D8
:10FF20000BF045FE4FF4447120460FF047F8204691
:10FF3000BDE810400D210FF02EBB00000080FFFF38
:10FF40002DE9F043BBB0044608F01EF905462046F3
:10FF500008F051F9814614AA31A92846FDF7A6FAFE
:10FF6000149800281ADD684603F093FA6A460021C7
:10FF700028460DF040FFDDE93101CDE90B01A96B09
:10FF8000E86A08440990E96BE86A08440A90149802
:10FF9000ADF834006946484603F048FA4FF400389B
:10FFA000414628460DF096FC0746414628460DF08E
:10FFB000B2FC0646414628460DF0D4FC04464146B4
:10FFC00028460DF05AFCB74201DD394600E03146C3
:10FFD000844201DD224600E00246914205DDB7423F
:10FFE00001DD384604E0304602E0844200DD204670
:10FFF00014990C1A002C19DD684603F04AFA6A4677
:020000040801F1
:10000000414628460DF0F7FEDDE93101CDE90B014F
:10001000D5E90B0108440990696BE86AADF83440F2
:1000200008440A906946484603F000FA36AB31A905
:100030002846149AFDF7B4FB15A805F0CDFA15AAC9
:100040004FF4403128460EF036F836AA15A9484636
:1000500005F0ACF83BB0BDE8F08300002DE9F04FAF
:1000600089B08A46FE480CF014FD01287DD1504627
:1000700008F086F80546504608F086F804464FF02A
:10008000640B4FF4B479022D13D0082D6ED0032DDC
:10009000FCD00E2D6BD00F2D6AD0132D69D0182DEA
:1000A00068D01A2D61D109B05046BDE8F04FFFF776
:1000B00047BF09F0E9FB050057D009F02FFC0128E4
:1000C00053D101A9284609F0FDFB05AA03A9204642
:1000D000FDF7ECF903990198401A019002990498F0
:1000E000081A029094F84C00C00731D14FF4003147
:1000F00020460DF0A5FA054605984FF48031401BC7
:10010000059020460DF066FE0028059806D1C1171F
:1001100000EB9171B5EBA10F00DA8D10401B05903B
:10012000012801DA012005900198029A404302FB60
:10013000020105984043814206DDE06C40F0010178
:10014000E16413F0DFF8606594F84C00C0070CD050
:10015000019911B90298002807D0D4E90E06864209
:1001600001DA06F5B476029805E0ABE0C0E0D9E02C
:10017000F6E0FBE061E100F075FEE16A401AA16B78
:10018000451A01E005F5B475002DFBDB48468542B4
:1001900002DBA5F5B475FAE705984FF41D714843E5
:1001A000B0FBFBF7322003F00BF94FF4B471484376
:1001B000B0FBF7F294F84C002946C0F3C007204684
:1001C000FFF746FE00287DD0A06BA26D311AA2EB8E
:1001D0000008A5EB0800002801DD024600E04242CD
:1001E0004FF48C739A4205DD94F84C20120709D520
:1001F000002508E0E26C5FEAC26C04D4120701D566
:100200004D4200E00D4677B1E16C0A071ED4CA06E4
:100210001CD4002800DC4042984217DD67F3C3017C
:100220000025E16412E08FB9E26C5FEA027C0DD533
:100230005FEAC26C0AD4002800DC4042C0F5B4700A
:10024000984203DD67F3C3020D46E264A5EB08059F
:10025000606D13F051F8216D41434FF47A70B1FB9A
:10026000F0F0854202DC4042854200DA0546D4E9DE
:100270001132A16BD01A771AFF0097FBF0F0001D26
:10028000C717454400EB177005EB2010256C009252
:10029000084432460BF018F9064694F84C00C0F3B7
:1002A0004100022803D1A06C811B606C0E18206CE9
:1002B000B04211D013F026F860653146204600F0B8
:1002C00018FA00E011E0AE4206D0002220212046BC
:1002D0000FF03FF9012808D1606CB04202D0A06C49
:1002E000B04202D113F00EF8606509B0BDE8F08F9E
:1002F000E06C20F001012046E1640CF0BCFC0546F6
:1003000008F0E2FC044609F0BFFA09F007FB0428F4
:10031000EBD1002CE9D009B02846BDE8F04F002110
:1003200008F047BD504607F05AFF256C132806D049
:10033000112804D0142804D0122802D005E0691C2A
:1003400000E0691E204600F0D4F9206CA842CCD011
:1003500009B02046BDE8F04F002220210FF0F9B887
:10036000504607F05BFF256C2918EBE7504607F075
:1003700053FF054603AA01A92046FDF797F8A06898
:10038000002600B1066A002120460DF059F980468A
:1003900003993044081A0299029A01440091019984
:1003A00003900B18121A091A04A800F0BCFC47F6B7
:1003B000FF7204A8296800F01AFC4FF0000AC0BBC5
:1003C0002868019A01684068891A029A801A00F028
:1003D00049FDE16A401AA16B471A01E007F5B477BD
:1003E000002FFBDB4846874202DBA7F5B477FAE72C
:1003F00003984FF41D714843B0FBFBF9322002F023
:10040000DFFF4FF4B4714843B0FBF9F239462046A0
:10041000FFF71EFD68B108EB4602114604A800F084
:1004200023FB47F6FF7204A8296800F0E0FB28715F
:100430005BE7FFE785F804A057E700210DF04AFAD3
:100440000746002120460DF066FA064600212046A8
:100450000DF088FA0546002120460DF00EFA01E065
:10046000C4E00508B74201DD394600E03146854267
:1004700001DD2A4600E00246914205DDB74201DD7A
:10048000384604E0304602E0854200DD28468046DA
:100490004FF44039494620460DF01CFA07464946BC
:1004A00020460DF038FA0646494620460DF05AFA25
:1004B0000546494620460DF0E0F9B74201DD3946D0
:1004C00000E03146854201DD2A4600E002469142C5
:1004D00005DDB74201DD384604E0304602E08542E2
:1004E00000DD2846801CA0EB08052046FFF770F8C9
:1004F0004419504607F090FE0168A14200DD0C4609
:100500000460F2E670B50C460546114600F076F838
:1005100021462846BDE8704000F0B6B870B50C46DC
:100520000546114600F006F821462846BDE8704011
:1005300000F032B870B505460C46B1F5B47F01DD68
:10054000A1F5B474D5E90E10421AA4EB010101D54E
:1005500002F5B472002901DA01F5B4718B1A002B8F
:1005600000DC531AB42B03DD28460DF032FF0DE0FA
:10057000914203DA00230246214604E08A4205DA6A
:100580000023224601462846FEF7E2FC2846EC639B
:10059000BDE870401DF08CB970B505460C46B1F54C
:1005A000B47F01DDA1F5B474D5E90E010A1AA1EBFF
:1005B000040101D502F5B472002901DA01F5B47124
:1005C0008B1A002B00DC531AB42B03DD28460DF0E8
:1005D00000FF0DE0914203DA00232246014604E0C9
:1005E0008A4205DA0023024621462846FEF7B0FC7F
:1005F0002846AC63BDE870401DF05AB970B5054699
:100600000C46B1F5B47F01DDA1F5B474D5E90C1049
:10061000421AA4EB010101D502F5B472002901DAF6
:1006200001F5B4718B1A002B00DC531AB42B03DDD7
:1006300028460DF0CEFE0DE04FF40033914202DA71
:100640000246214603E08A4204DA22460146284651
:10065000FEF77EFC2846FEF7C3FC28466C63BDE827
:100660007040FEF7BDBC000002E000BF01F5B471B0
:100670000029FBDB4FF4B472914202DBA1F5B471A7
:10068000FAE7C1620DF0A5BE70B505460C46B1F59E
:10069000B47F01DDA1F5B474D5E90C010A1AA1EB10
:1006A000040101D502F5B472002901DA01F5B47133
:1006B0008B1A002B00DC531AB42B03DD28460DF0F7
:1006C00088FE0DE04FF40033914202DA22460146E3
:1006D00003E08A4204DA024621462846FEF738FC47
:1006E0002846FEF77DFC28462C63BDE87040FEF7E7
:1006F00077BC036C8B420CD0826C8A4200DA1146C4
:10070000426C8A4200DD11468B4202D001641DF02A
:10071000CFB87047F0B50D688C68D1F80CE0641B59
:10072000D0E900654F68DDF814C0AEEB0707162A64
:1007300075D2DFE802F0C7C71A272D2F454D5D0B94
:100740006567757B7D8F97999B9DA1BD8268A2EBA4
:10075000060E0EF1010E621C0EEBDE7E4FEA6E0EEF
:1007600002EBD272AEEB620233E08068821B601C47
:10077000521C02EBD272521000EBD070A2EB60025E
:1007800000208AE08068621C801B401C821AF7E708
:1007900000220DE08268A2EB060E0EF1010E621C33
:1007A0000EEBDE7E4FEA6E0E02EBD272AEEB620211
:1007B000C06807F1010E401B401CA0EB0E006CE06E
:1007C000826804F1010E921B521CA2EB0E02EFE7AD
:1007D0000022C068A0EB050E0EF1010E781C0EEB96
:1007E000DE7E4FEA6E0E00EBD070AEEB600054E0A0
:1007F000826804F1010E921B521CA2EB0E02E8E784
:1008000000220AE08068821B601C521C02EBD2723C
:10081000521000EBD070A2EB6002F8433DE051E0D3
:100820008068621C801B401C821AF6E700220DE0E3
:100830008268A2EB060E0EF1010E621C0EEBDE7E4C
:100840004FEA6E0E02EBD272AEEB6202C068401B42
:10085000401C22E0826804F1010E921B521CA2EBA4
:100860000E02F3E7E2438BE7E243B2E7E2439FE79E
:100870008068821B00200FE08268C068921BA0EB9A
:10088000050E0EF1010E781C0EEBDE7E4FEA6E0EA9
:1008900000EBD070AEEB6000521C324428441A4486
:1008A0006044C1E9002022443844C1E90220F0BD7F
:1008B0008268C068921B401B07F1010E401CA0EB30
:1008C0000E00E9E700225BE70A6802604A684260BE
:1008D0008A688260C968C16070470A6802604A68B5
:1008E00042608A688260C968C16070470A680260B5
:1008F0004A6842608A688260C968C16070470A6855
:1009000002604A6842608A688260C968C160704754
:100910000A6802604A6842608A688260C968C16089
:1009200070470A6802604A6842608A688260C968E3
:10093000C16070470A6802604A6842608A688260E3
:10094000C968C16070470A6802604A6842608A6884
:100950008260C968C16070470A6802604A68426084
:100960008A688260C968C16070472DE9F0470C460B
:10097000064615461146204600F0E6F800285CD0F1
:1009800000222946204600F09CF800284FF0000085
:1009900051D1E76861682368A7EB010C6F68A26812
:1009A0007F1AA2EB0309002F05DD08C60F4486E875
:1009B00086000120361FE96862688A1AACEB0203E0
:1009C000002B0CDDE268914209DA06EB001C276877
:1009D000A2684CF8047B0B448CE80E00401C69684C
:1009E0006268914200DC1146EA68E3689A4200DBE3
:1009F0001A46531A2F682268BF1A002F0BDD002BEE
:100A000009DD06EB0018174448F8042B01EB030C32
:100A100088E88210401CAA682468151BA9EB05040D
:100A2000002C08DD06EB00151444C5E900210B4439
:100A3000C5E90243401CBDE8F0874FF0FF30FAE7FC
:100A4000C1684068081A401C704702688168891AAA
:100A5000C2684068101A401C491C484370478168AE
:100A60000068081A401C704703685B1A03608368BB
:100A7000194481604168891A4160C1681144C160AC
:100A8000704770B50B681468A34200DC234603600E
:100A90004D685468A54200DD2C4644608E68956818
:100AA000AE4200DA35468560C968D268914200DB03
:100AB0001146C1600120AB4201DC8C4200DD002008
:100AC00070BD7CB50D46044600680968164688422C
:100AD00038DB61686A68914234DBA268AB689A428D
:100AE00030DCE268EB689A422CDC4EB3CDE90001C1
:100AF00032466946284600F07AF8002821D0D4E929
:100B00000110CDE9000132466946284600F06FF831
:100B1000002816D0E1682068CDE900013246694618
:100B2000284600F064F800280BD0D4E90201CDE992
:100B3000000132466946284600F059F8002800D0E6
:100B400001207CBD00207CBD02688B689A420DDCD0
:100B500082680B689A4209DB4268CB689A4205DCDE
:100B6000C0684968884201DB012070470020704757
:100B70007CB50D460446806809681646884234DB19
:100B8000E0686968884230DB2168A86881422CDC13
:100B90006068EA68904228DC2EB3CDE90010324646
:100BA0006946284600F023F8E8B9D4E90110CDE9F8
:100BB000000132466946284600F019F898B9E16804
:100BC0002068CDE9000132466946284600F00FF85A
:100BD00048B9D4E90201CDE9000132466946284608
:100BE00000F005F808B100207CBD01207CBD2DE996
:100BF000FF4114460E460A68016805468A422EDB0C
:100C0000A86882422BDC72686B689A4227DBEF6827
:100C1000BA4224DC002C5DDD401A401C00EBD07091
:100C20004210F81A401C00EBD0704010824200DAEB
:100C30001046844200DD04460091286800222044CA
:100C400002906868019068683146204403906846C5
:100C5000FFF7CDFF38B102982044029032E0002027
:100C600004B0BDE8F081E8680022001B0190E8684C
:100C7000039031466846FFF7BAFF18B10298204446
:100C800002900DE0A8680022001B0090A868029066
:100C900031466846FFF7ABFF30B10098001B00906B
:100CA0000198001B019010E06868019068680022BC
:100CB0002044039031466846FFF799FF50B10098F1
:100CC000001B0090039820440390314668460FF0C3
:100CD0000FFAC5E70120C3E710B50C6813689C4202
:100CE00000DA234603604C6853689C4200DA2346CE
:100CF00043608C6893689C4200DD23468360C9682A
:100D0000D268914200DC1146C16010BD03680B44FB
:100D10000360836819448160416811444160C1687F
:100D20001144C160704710B5029C80E81E0010BDE0
:100D30004268491E1144C16070470268491E11444F
:100D40008160704742688A4201D80020704702687B
:100D50001AB1C06801FB00207047FEE770B5044679
:100D60000068002510B107F09DFC25606560A56056
:100D700070BD0021FFF7E6BF10B50446231D00201B
:100D800083E8070001FB02F00AF066FB2060002800
:100D900000D1FEE710BD70B5044600680D46A0B155
:100DA000D4E90101884203D12046091D00F00EF864
:100DB000D4E90001E26801FB020029460AF0C2FB07
:100DC0006068401C6060012070BDFEE770B50D4694
:100DD000C1680446694300680FF0D6FA30B1A560D7
:100DE00020606068A84200D9656070BDFEE7406879
:100DF000704700002DE9F04781468A46002012F036
:100E000049FB04464FF000080E4F16E0204612F052
:100E100041FB0546A068B8420ED1E66831684945F5
:100E20000AD17168514507D1204612F0E9FA3046DF
:100E300007F038FC4FF001082C46002CE6D1404664
:100E4000BDE8F087490E010870B5C568D5E90046D0
:100E500012F0D6FA284607F025FC3046A446BDE835
:100E6000704060470022002801DA01224042002938
:100E700001DA4942921C884207D9C1EB011101EB0A
:100E80004101B1FBF0F3103205E0C0EB001000EBC4
:100E90004000B0FBF1F30020D9B216290BD92C2960
:100EA00000D80120292900D8401C252900D8401C41
:100EB00020290BD90BE0022900D30120062900D3F9
:100EC000401C0A2900D3401C0F2900D3401C1844A1
:100ED000D10601D5C0F15A0091074FEAC27105D57C
:100EE00009B1B43005E0C0F1B40002E009B1C0F5C9
:100EF000B47080B27047C16000680DF06ABA0068D3
:100F00004FF0FF320168C26001F15002904202D1FD
:100F10008268CA6205E001F16002904201D18268F4
:100F20008A6300680DF055BA10B50C4600206421A4
:100F3000C4E90C01A063E062E06360642064A06423
:100F400094F8701021F03F0184F8701084F84C0080
:100F500004F15001204600F0A2F804F1600120469F
:100F600000F09DF8082120460EF028F810212046B8
:100F70000EF024F820460022BDE81040114600F093
:100F8000CDB810B50C46002104F15000FEF706FE66
:100F900004F16000BDE810400021FEF7FFBD000035
:100FA0002DE9F0410D462F480BF073FD01284FD17C
:100FB000284607F0E5F80446284607F0E5F880469D
:100FC000182C0AD0012C45D0082C43D01A2C3FD124
:100FD0002846BDE8F041F8F767BF4FF400310BF049
:100FE000CEF80446284607F017F905460068A042E7
:100FF00000DD0446002140462C600CF06EFC0746E4
:10100000002140460CF08AFC0646002140460CF0C8
:10101000ACFC0446002140460CF032FCB74201DA39
:10102000394600E03146844201DA224600E00246B9
:10103000914205DAB74201DA384604E0304602E070
:10104000844200DA2046002802DA2968081A28605B
:10105000BDE8F08108F13C014046BDE8F0410DF0EB
:10106000D3B90000E8E0050890F8700000F0070030
:10107000704790F8701001F00701022901D0006B51
:101080007047C16E491C01D0806E7047806B7047FD
:10109000C16D491C01D0806D7047C06A70470860FF
:1010A000002048608860401EC860704790F870104B
:1010B00001F0070101290AD1016B002907DA426B0F
:1010C000002A04DD806B884201D101207047002096
:1010D000704738B5134690F8702002F00702022AD4
:1010E0001BD1D0E90C428A4201DD0D4600E01546D5
:1010F000AC4201DD214602E08A4200DC1146C26AB0
:101100008A4200DA1146826B8A4206D0009300F1CF
:10111000600300F1380200F023F838BDF8B5C56A65
:1011200013468D421AD0D0E90C428A4201DD0E46A8
:1011300000E01646B44201DD214602E08A4200DCAE
:101140001146826B8A4200DD11468D4206D0009323
:1011500000F1500300F12C0200F002F8F8BD00008D
:10116000F0B597B007461C981C4616460D4668B366
:10117000E068401C40D0A068C4E901050021184681
:101180001560FEF70BFD6846FEF746FD21466846F2
:10119000FEF7F6FD19496846FEF7D8FD4FF4807258
:1011A00000216846FEF7E6FD15496846FEF7BFFDDB
:1011B0003846002164220CF0F3FB01466846FEF736
:1011C000BDFD6846FEF7FEFD17B0F0BD00211846D4
:1011D000FEF7E4FC4FF0FF30E060384635600DF07C
:1011E000F8F800212046FEF7D9FC17B02146384612
:1011F000BDE8F040FFF753BF3068BDE7F70E0108C8
:10120000FF0E010870B58C6C0D462CB1206C18B126
:1012100002F0C7FC002020642846BDE87040FBF7C0
:10122000D3BE00002DE9FF4F088C85B0C0F3072521
:10123000E81F1E460C46039003280BD9102D09D039
:10124000112D07D00F2D05D0122D03D0132D01D055
:10125000142D1ED1D4F848805FEA08001AD0D8F8BF
:1012600000000190284601F091FC81460798FFF7A5
:10127000F6FB8346207C01280FD000208246706850
:101280006FF06041C84231D10398032807D810207D
:1012900006E0002009B0BDE8F08F0C20EEE72846FC
:1012A00002900020009001235A46D8F8400002998D
:1012B00002F017FE070013D1D8F8400020B102F069
:1012C00070FC0020C8F84000002000900122594620
:1012D0005848029B02F024FC0700DAD0C8F840709E
:1012E000079907C986E80700F16006E0401C7060B6
:1012F000F068401CF060D8F8407007997068D7F823
:101300001080C9688842C4DC0399032946D80822A2
:10131000B2FBF9F13268B2FBF1F301FB1321029148
:101320000BFB09F10123C91D03EBD1010391636B91
:1013300002FB09F20AEB8301238D9BB200FB031031
:1013400000EBD209207C012810D0E068016901EB94
:10135000090600BFCDE900685B46216B2846029A6A
:10136000F7F75AFD207C012814D050E003980AF0CA
:1013700073F806000DD00020009032464946039BCA
:101380000198FBF73EFE0028E4D0304607F08AF9CA
:101390007FE7FEE7304607F085F938E0102D39D0B9
:1013A000112D37D00F2D35D0122D33D0132D31D034
:1013B000142DEDD139894FF000098DB2218D2B46C6
:1013C0008AB200FB02A031684246090100EBD1015C
:1013D000CDF800900198FBF714FE0028D8D1616A7F
:1013E0000C200A0C218D8BB202FB03007268C1F342
:1013F0004E0102FB0100316808EB050201445B4627
:10140000CDF800900198FBF7FCFD0028C0D1012029
:10141000E7623FE70BFB09F1CB08218D8AB200FBA5
:1014200002A03168424601FB09F100EBD101002026
:101430000090E7E78C53002038B50D46C968287C3A
:10144000144620B1012807D0022825D016E00C222E
:1014500020460AF077F824E0084607F07DF915A148
:1014600010F0DEF850B96B460C22214605F114004D
:1014700007F0D9F910B900980C2801D0002038BD28
:101480002078192802D0607019202070206820214F
:1014900041EA1040608004E00120A080E0800E203E
:1014A00060702068C1B2192902D0400C40006080F1
:1014B000012038BD62696E0010B507F0EFFD040031
:1014C00011D0094907F0DCFE0849204607F0DAFE92
:1014D0000749204607F0D2FE0649204607F0CCFE19
:1014E00005A0206110BDFEE739140108FD140108B4
:1014F000251201080512010842494E002DE9F04766
:1015000082464FF00008087C90B00C464546C14624
:10151000012801D088B34FE0E06807F01DF95EA113
:1015200010F07EF898B92046FCF736F806000ED089
:101530000C20A66409F090FF070007D00222E168A2
:1015400007F026F938B1384607F0ACF89FE00020E4
:1015500010B0BDE8F0873760216AC1F30720090C9D
:10156000090729D4C11F032923D90B3803285ED8C2
:1015700021465046F7F76CFB04E007E02146504651
:10158000F7F7F0FB8046012816D150E0E668306995
:101590000028DDD03088C0F30727206A000C000740
:1015A0000AD4F81F03280CD80846FBF7F5FF0028DB
:1015B000CED0E0790028E1D02046FBF705FD40467B
:1015C000C6E7A7F10B000328084604D8FBF7E4FFA1
:1015D0000028BDD0CCE7FBF7DFFF3168090CC90656
:1015E00001D5354609E000F1240530890004000CDE
:1015F00009D03146284602F021FBE5622889000423
:10160000000C11D012E01822314608A8EEF7A4FE13
:10161000384601F0BBFA099989B24843C01DC00899
:10162000ADF8280008A9E5E7208D28810125E76AA3
:101630005FB33946204607F0CBFD060027D0BE42F7
:1016400008D02046FBF7C0FC2046FBF7A5FFC6618B
:10165000E66201E0E062C5B9A079B0B907F096FC96
:1016600098B1207C8DF81000E0680390E26A02A92E
:10167000D06802905046A36C07F0D6FC38B1606485
:101680002046FBF789FFC0F81C90012060E7204648
:10169000FBF79AFC5BE7000062696E0010B50C4630
:1016A000102120460DF08AFC2046BDE810404FF482
:1016B00080610AF07CBA000010B5014603480AF0C8
:1016C000E1FD04460AF044FE204610BD0CE1050889
:1016D00070B50446806B154688420FD9606B30F8B0
:1016E0001120AA4320F811202046FDF795FC68053B
:1016F00004D52046BDE870400DF0B6BB70BD70B596
:101700000E460546002405E0324621462846FFF7EE
:10171000DFFF641CA86BA042F6D870BD084600210C
:101720004FF6FF728163C0E90F1201634163C1622A
:101730004164014900F0ECBA30E1050810B50146FA
:1017400003480AF09FFD04460AF002FE204610BD41
:101750004CE1050810B50C46086B06F0A3FF606B62
:1017600006F0A0FF00202063606310BD2DE9FE4F4E
:101770008A46FE480BF08DF9012833D1504606F019
:10178000FFFC0646504606F0FFFC00270446182ED4
:1017900002D02F2E48D02BE0E06BA146002821D0AC
:1017A0000025D9F82C800FE0D9F8340030F8150066
:1017B000400508D5E06BB8B120460BF00DFAE16B9F
:1017C000B0FBF1F111E06D1C58F82500002809D09C
:1017D000E7A10FF025FF002804D058F82500007875
:1017E0000028E1D1BDE8FE8F0021504606F095FDAE
:1017F0002E2E1DD04FF6FF75012E1BD0022E59D074
:10180000082E69D0062E7CD0032E7BD0102E7AD0E5
:10181000112EE7D0122EE5D00E2E75D01A2EE1D162
:101820005046F9F75BFADDE7E16A00F071FAD9E7B3
:101830002046F9E7504606F0A9FC06462046216CF2
:10184000FDF7EAFB08F020F808F068F8012801D05D
:1018500003281AD16946304608F034F86946204614
:10186000FBF7C8FC2564A842BCD0616B31F81010AE
:10187000C1F38012002AB5D1C1F300110029B1D102
:10188000014620642046FDF7C7FB206CA842A9D082
:10189000616B31F81000C0F340210029A2D1C0F3E0
:1018A000802166E0206C029002AA202120460DF0E3
:1018B00050FE97E7206CA84294D0504606F066FC94
:1018C000694607F0FFFF69462046FBF793FC216C51
:1018D000814287D0204659E0216CA9423CD0626BFE
:1018E00032F81100C0F3C013CBB1C0F38013B3B909
:1018F000C30503D594F84430DB0718D040F480705A
:1019000003E02EE040E044E08DE022F8110094F87E
:101910004400C00703D02046216C12F08EFA216CDF
:10192000606B30F81100C0F3402131B902E020F4BF
:101930008070E5E7C0F3802171B1C0F3801159B91F
:10194000C0F3001040B9206C029002AA202120466A
:101950000DF0FFFD0128ACD12046216CFDF75CFBAA
:1019600040E7206CA842A4D0616B31F81000C0F3AE
:10197000401100299DD1C0F38011002999D1C0F3F5
:10198000001000288ED02DE72046216CFDF744FB87
:1019900047E0A06B00288CD0504606F0F7FB0746C6
:1019A00007F0BCFF06462FB9002007F07FFF07F0C5
:1019B000B5FF064620460BF05EF907F085F9216C6D
:1019C000A942CDD1022E02D0042E2AD148B394F8D8
:1019D00044100020A26BC90701D113E0401C8242D1
:1019E0001DD9616B31F81010C1F30013002BF5D134
:1019F000C1F38013002BF1D1C1F300210029EDD0F8
:101A00000DE0401C82420AD9616B31F81010C1F31D
:101A10000013002BF5D1C1F380110029F1D120640E
:101A2000E0E62564DEE62046216CFDF7F5FA504637
:101A300006F0D5FB132813D0142835D004264FF018
:101A40000809122852D0112886D1002120460BF017
:101A500035FF8046206CA84274D12764626BA3E0F6
:101A6000206CA84202D13846276401E0401C206463
:101A7000A36B984200D32764666B226C07E0491C75
:101A80002164994200D32764206C90426DD0216C70
:101A900036F81100C0F3001CBCF1000FEFD1C0F309
:101AA00080100028EBD157E7206CA84201D12764B1
:101AB00000E000B9A06B401E20640346626B09E0A1
:101AC00019B1491E0846216402E0A06B401E206443
:101AD000984267D0216C32F81100C0F30016002E36
:101AE000EED1C0F380100028EAD135E7002120466E
:101AF0000BF0E4FE8046206CA84213D12764626B91
:101B000004E0491C2164A06B81424BD2216C32F865
:101B10001100C0F30013002BF3D1C0F38010002894
:101B2000EFD119E7216B01EB0010FEF798FF034698
:101B3000206C216B024601EB00152D6805EB630C50
:101B4000A36B25E03CE000BF06EB001506EB021797
:101B50004D59CF59BD421ADD01EB00152D68654581
:101B600015DC09EB00154F5904E01BE04CE10508BA
:101B70000A00000007EB0805654508DB656B35F8D2
:101B80001050C5F3801717B9C5F3001515B1401CE7
:101B90008342D9D8834245D8DEE6491C2164A06B34
:101BA000814201D32564D7E6216C32F81100C0F3DD
:101BB0000013002BF1D1C0F380100028EDD1CBE64B
:101BC000216B01EB0010FEF74AFF226C216B01EB49
:101BD00002131B6803EB600310B21EE006EB001556
:101BE00006EB02174D59CF59BD4214DA01EB00152F
:101BF0002F68A7EB08059D420DDC09EB00154D5938
